:10000000F01F001031C100002DC100002DC1000003
:100010002DC100002DC100002DC100000000000016
:100020000000000000000000000000002DC10000E2
:100030002DC10000000000002DC100005DB70000D0
:1000400085B7000085B7000085B7000085B70000C0
:1000500085B7000085B7000085B7000085B70000B0
:1000600085B7000085B7000085B7000085B70000A0
:1000700085B700002BC100002BC1000015B50000A2
:1000800045B700002DB7000015B70000FDB6000011
:100090002BC100008DB600002BC100002BC1000059
:1000A0002BC100002BC100002BC100002BC10000A0
:1000B0002BC100002BC100002BC100002BC1000090
:1000C0000223184A10B5116801240B431360202342
:1000D000154A164811680B431360154B1968014007
:1000E0001960196821431960124B13491A680240BC
:1000F0001A601A6822431A606C22104B1A60104B67
:1001000018680CF02FFA80220E4B120218600E4B6A
:1001100018600E4B20001A6080234022DB051A6015
:1001200010BDC0460480044080800440F8FCFFFFFE
:100130003040044034400440400D030018000040AB
:1001400018000010140000401000004000E100E022
:10015000802208201021094BD20510B511601860CB
:100160000023074814680C4201D0834204D105489B
:1001700098428041404210BD0133F3E7180000402F
:10018000FF0F0000FE0F0000802100222020134BF3
:10019000C90510B55A609A60DA600860104958685D
:1001A000012807D08A4203D1FFF7D2FF002010BDFB
:1001B0000132F4E78A42F7D000211A69013A5868FF
:1001C000FF2801D95868F2E71869904202D01A69ED
:1001D00059690A3158698142F1D1E5E718000010E8
:1001E000FF0F0000F8B5060003250C4B0C4C1F78E0
:1001F0000223A222A361013BE361E318DA77013312
:10020000DE77084BDF77FFF7BFFF0223FF3398420B
:1002100002D0013D002DEBD1F8BDC04668ED0000D5
:10022000180000101B000010064A537BD318D87327
:10023000537B0133DBB253735BB2002B01DA002333
:100240005373704728100010C143094A53699942FB
:1002500009D2591C08185169994200D27047516956
:100260008842FCD8F7E75169C91A8142FBD3F5E708
:10027000180000104023044A11680B431360012248
:10028000024B30331A707047808004401800001011
:10029000084B70B530331B7804000D00002B01D1E2
:1002A000FFF7E8FF182223689343236023681D4368
:1002B000256070BD180000100E4B70B530331B78F0
:1002C00006000D001400002B01D1FFF7D3FF701EB4
:1002D00002280AD8084B8000C25801231168AB409D
:1002E000012C04D10B43136070BD044AF5E7994318
:1002F0001160F9E71800001070ED0000FC3F00509D
:100300000F4B70B530331B7806000D001400002B26
:1003100001D1FFF7AFFF701E02280BD8094B8000F8
:100320001818C26801231168AB40012C04D10B439B
:10033000136070BD044AF5E799431160F9E7C046C0
:100340001800001070ED00000080005010B50C4C3B
:10035000606B002806D00220FFF744FF0238FF3808
:1003600043425841230038331A780A235106490F73
:100370004B430F210A4048349B186370E07110BD55
:1003800018000010F8B505000E000324A227094B41
:10039000B21C9A610022DA610133DF770133DD7725
:1003A000FFF7F2FE0223FF33984202D0013C002CFB
:1003B000EDD1F8BD1800001010B50120FFF712FFB5
:1003C0000223FF33984210D1094B01201A00383222
:1003D00014785863220706D0032203332240DA77C9
:1003E0000100FFF7CFFF200010BD01246442FAE7AF
:1003F0001800001070B50D4C636B002B13D0D5B2F4
:10040000E31CDD77130A251DDBB2EB77130CDBB29F
:10041000651D120E0634EB77E277FFF7B3FF023863
:10042000FF3843424341180070BDC0461800001019
:1004300010B5FFF7C1FF0220FFF7D4FE0223FF3300
:10044000984220D1104B1A00383212787F2A15D9E1
:100450005A6B002A12D01A000021082001242232EF
:100460009070D47051701170142226330638D970F0
:1004700018705C709A700731FFF784FF034A0421FB
:100480000920FFF7B7FF10BD1800001080808080A2
:10049000012210B510000B21FFF732FF00220B21C3
:1004A0000120FFF709FF012202210320FFF728FFA7
:1004B000002202210320FFF7FFFE10BD70B50600E9
:1004C0000024064D1835605D054B3100C01801341D
:1004D000FFF7DEFE0A2CF6D170BDC04670ED0000BD
:1004E00000400440F8B500240C4D22352B19665D00
:1004F0005F78012239003000FFF702FF023400224A
:1005000039003000FFF7D8FE142CEFD10020FFF7A0
:10051000D5FF0022024B5A65F8BDC04670ED0000C1
:1005200018000010F0B50125734B85B000900C0049
:100530009D6572B68022714B1202DA676C2200262A
:100540006F4B70481A60704B1968014019601A6847
:1005500004211A606D4B1A6802401A601A68002064
:100560001A602A00FFF7CCFE2A0004210020FFF7C2
:10057000A3FE2A0005210020FFF7C2FE2A00052164
:100580000020FFF799FE624B624D1E60FFF7AAFF45
:1005900031006148FFF77CFE31006048FFF778FECC
:1005A00031005F48FFF774FE31005E48FFF770FED0
:1005B00031005D48FFF76CFE5C4B1A685C4B1A60BB
:1005C000009B5A1E93413F225B429343594A9B181A
:1005D000594A13600423594A11680B431360584B5E
:1005E0002E601A685749584E0A401A602A680193CB
:1005F000A30700D47BE0EC235B0113432B60802333
:100600003360DB1833608023DB00336080235B01C1
:10061000336080231B013360009B002B52D00024E9
:100620004A4B4B4F1C604B4B21001C603800FFF7BE
:100630002FFE220009212000FFF762FE220009217F
:100640002000FFF739FE8021434A444813680B43DA
:10065000136007223B68763993433B603B68053A59
:1006600013433B60009B58430BF084FD03223C4B3B
:100670003C4918603C4B01981C603C4B1A603C4B59
:100680001A680A4080211A601A680A431A60802397
:1006900080229B0052023360326002687E391A4326
:1006A00002602A6813432B600123324A1360324AE6
:1006B0001160324A254913601460136010681842B3
:1006C000FCD00B6001222E4B52421A600A4BDB6DAC
:1006D000039362B630BFC046074B039ADB6D9A4264
:1006E00000D130BF0023044A936505B0F0BD8023DC
:1006F0001B0113432B608CE71800001004E100E09D
:1007000018000040F8FCFFFF304004403440044033
:100710000480044004820440084004400040044037
:10072000AC400440144004401C4004403882044063
:1007300034820440FF1800003082044010ED00E0D5
:10074000008204407FE2FFFF00E100E004C00040BF
:10075000644004400400014080800440841E000086
:1007600018C000400FF0FFFF08C0004014C0004058
:100770003CC0004078800440708004407480044095
:1007800008820440F7B50F4D6C6D002C18D1102075
:10079000FFF794FE0C4B22330193019B0022E65C91
:1007A0001B195F7830003900FFF7AAFD02340122DF
:1007B00039003000FFF780FD142CEED101236B656A
:1007C000F7BDC0461800001070ED000070B572B69D
:1007D00080248020802180250F4BC0001A1D6400DA
:1007E0004901D567D467D067D167C02252009D50B8
:1007F0009C5098509950094A094913680B4013605E
:10080000AC22084B52011A60FFF7BCFF0022064BD6
:100810001A6662B670BDC04600E100E00482044082
:100820007FEAFFFF0882044018000010F8B50700B7
:10083000FFF7A8FF002F09D0012207210220FFF7B0
:100840005FFD002207210220FFF736FD124E330024
:1008500030331B78002B01D1FFF70CFD0F4D012425
:100860002B681B0509D530363378002B01D1FFF7F3
:1008700001FD01242B68DB0A9C43002F09D00022D4
:1008800007210220FFF73CFD012207210220FFF78C
:1008900013FD2000F8BDC04618000010FC3F0050BA
:1008A000F0B5012089B0FFF7C1FF012304930028B0
:1008B0004FD104001D0004902A4E630001330393BE
:1008C000330037002233E25C1B195B780192190078
:1008D0002A0001980293FFF713FD00220299019864
:1008E000FFF7EAFC204B343630333C37069607934B
:1008F0003B787E780593079B1B78002B01D1FFF78F
:10090000B9FC059B032B0DD818000BF015FF022531
:100910002729164B2A00B2401B6813405A1E9341E8
:10092000002B02D16B461B7B0493039B023F0133D8
:100930000393069B9F42DBD1002202990198FFF7A7
:10094000DFFC02342A0002990198FFF7B5FC142C51
:10095000B2D1049809B0F0BD054BDBE7054BD9E7F0
:10096000054BD7E770ED000018000010FC3F005069
:10097000FC3F0150FC3F0250FC3F0350F8B54A00D9
:10098000070004001E48520D1518132D18DC002D09
:1009900009DACB0FDB070022691C01D119490B438F
:1009A0001900100017E0184E2E4132000A4014437F
:1009B00012D0802212032A415318B3430022EFE7DA
:1009C000332D0BDD8023DB009D4205D13A000B0067
:1009D00038000CF047FC07003800F8BD01260B4832
:1009E00076421218D6403E42F6D03322551B323A98
:1009F000AA40D219BA42A44164420B19B243CFE7CC
:100A000001FCFFFF0000F03FFFFF0F00EDFBFFFFC9
:100A100007B5002200280CD090231B0600920193FA
:100A200000980199802300225B050DF041FB03B083
:100A300000BD80235B05F1E707B5002200280CD03C
:100A4000F0231B060092019300980199E0230022F5
:100A5000DB050DF02DFB03B000BDE023DB05F1E766
:100A6000F0B5D34A4B0089B007000E000C005B08BC
:100A700093423CD9CF4A934200D8F5E1CE4A934203
:100A80000DD90B031B0B034304D002000B000CF029
:100A9000E9FB0EE000290EDA0027C84E0BE0C84A39
:100AA000C84B0BF07DFE002800D1DDE10020FFF7F0
:100AB000C3FF07000E003800310009B0F0BDC24A84
:100AC000C24B380031000CF0CDFB002200230BF0AC
:100AD00053FE0028E0D1BE4ABE4B380031000DF075
:100AE000E7FA002C00DAA8E00024BB4DA7E0BB4ADF
:100AF000934200D8C5E0BA4A9342ECD8B94ABA4BFF
:100B0000002900DA8FE00DF045FD012304000D00FF
:100B10000093B64AB64B02920393029A039B2000BD
:100B200029000DF037FD02000B0007000E00200029
:100B300029000DF02FFD029A039B0DF02BFD029072
:100B400003910022A44B380031000DF0B1FA04905B
:100B5000059102000B00380031000DF0A9FA0400E5
:100B60000D00A44AA44B0DF0A3FAA44AA44B0CF028
:100B700079FB22002B000DF09BFAA24AA24B0DF04C
:100B800009FD22002B000DF093FAA04AA04B0CF0B7
:100B900069FB22002B000DF08BFA9E4A9E4B0DF054
:100BA000F9FC22002B000DF083FA00229B4B0CF085
:100BB00059FB02000B0006900791049805990DF06F
:100BC00077FA02000B00002095490DF0E3FC0200CB
:100BD0000B0004900591069807990DF0DBFC049A30
:100BE000059B06900791380031000DF061FA020074
:100BF0000B0000208B490DF0CDFC02000B00069885
:100C000007990CF04BFE2B0022000DF051FA009BCF
:100C1000002B4CD102000B00380031000DF048FAD7
:100C200022002B003AE00CF01DFB01235B420093F5
:100C300004000D006D4A7C4B6DE700247B4D0200E3
:100C40000B00200029000CF00DFB0DF0EBFF0090D5
:100C50000EF01EF8634A644B029003910DF028FADF
:100C600002000B00380031000DF094FC5F4A0400D4
:100C70000D00029803995E4B0DF01AFA0290039151
:100C80004BE700216A4A0091934200D959E7694A2B
:100C9000694B31000CF0E6FA02000B000DF07AFC13
:100CA00002000B00380031000DF074FC01E7029ADD
:100CB000039B0DF06FFC3A0033000DF0F9F9029A36
:100CC000039B0DF067FC2B0022000DF063FC009BE2
:100CD00004000D0001330CD102000B00380031007C
:100CE0000DF058FC00223C4B0DF0E2F900223A4B8B
:100CF000DAE7009B012B26D10022504B380031004F
:100D00000BF03AFD002811D00022334B380031009F
:100D10000CF0A8FA02000B00200029000DF03AFCAC
:100D2000C02300221B060DF0C3F9C2E622002B00EF
:100D3000380031000DF02EFC02000B000CF092FA8E
:100D40000022364BA3E6009B1B050293009B013358
:100D5000392B0FD93A0033000DF01CFC02000B00B8
:100D600000202E490DF016FC029C00226318190089
:100D70002A4B99E7009B132B62DC8023009A9B038C
:100D800013410020254AD11A009001913A00330006
:100D9000200029000DF0FEFB02000B0000980199D5
:100DA0000DF0F8FB029C070063181E0083E6C046A6
:100DB00079684340412E8640FFFFEF7F0000F0BF7F
:100DC000EF39FAFE422E864059F3F8C21F6EA50194
:100DD000FE822B654715F73F0000E03F422ED63FCD
:100DE000B1A2F03F0000E0FE422EE63F763C7935AE
:100DF000EF39EA3D2DC3096EB7FD8ABE3952E6864A
:100E0000CACFD03EB7DBAA9E19CE143F8555FE1936
:100E1000A0015A3FF41011111111A13F0000F03F41
:100E20000000084000001840EF39EABD0000E0BFB4
:100E3000FFFF8F3C9C7500883CE4377E0000D0BFEC
:100E400000980E490022091A0B05200029000CF019
:100E500009FA02000B00380031000DF09BFB002264
:100E6000074B0CF0FFF99DE7002C00DA27E6054A56
:100E7000054B380031000DF01BF935E6FF0300008B
:100E80000000F03FFE822B654715F73FF0B54A00A2
:100E90005708914A89B005000C00CE0F97422DD912
:100EA0008E4A974211D90B031B0B034306D0020055
:100EB0000B00280021000CF0D5F910E0002E00D026
:100EC00006E12800210009B0F0BD854A854B0BF0F2
:100ED00067FC0190002805D00020FFF7ADFD05005C
:100EE0000C00EEE7804A814B280021000BF044FC07
:100EF000002807D00198FFF78BFDF0E77C4B9F425D
:100F000000D89BE07B497C4BF2008F426FD89F1842
:100F10003A6C7B6C280021000DF03CFB3B6D7C6D36
:100F2000012502900391AD1B04930594AB1B019323
:100F3000049A059B029803990DF02CFB05000C0008
:100F40002A002300280021000DF0B2F806000F004F
:100F50006A4A6B4B0DF0ACF86A4A6B4B0DF01AFB0A
:100F600032003B000DF0A4F8684A694B0CF07AF9A6
:100F700032003B000DF09CF8664A674B0DF00AFB0F
:100F800032003B000DF094F8644A654B0CF06AF9AE
:100F900032003B000DF08CF802000B00280021000D
:100FA0000DF0F8FA0B00020006000F0028002100E7
:100FB0000DF07EF8019B06900791002B53D1802302
:100FC0000022DB05300039000DF0E4FA02000B00CE
:100FD000069807990CF062FC2A0023000DF0DAFA5B
:100FE00002000B0000204F490DF0D4FA77E79E185D
:100FF00028004D4A4D4B21000DF05AF8326E736EA9
:101000000CF030F90DF00EFE01900DF041FE484A53
:10101000484B06000F000DF04BF802000B002800B3
:1010200021000DF0B7FA444A02900391434B30007F
:1010300039000DF03DF80490059179E7404B9F424F
:101040000CD8404A404B0CF00DF90022354B0BF008
:10105000A7FB002805D00022324B2AE7002301938A
:101060006EE701906CE7802132003B000020C9054B
:101070000DF090FA02000B00069807990CF00EFC98
:1010800002000B00049805990DF084FA029A039B64
:101090000DF080FA02000B00002022490DF07AFAD0
:1010A0002A4B019A9A4205DB019C0500260573181C
:1010B0001C0006E7FA25AD00AC46019C0022644402
:1010C000260573181900B8235B040CF0F1FF06E73E
:1010D00000252C00F5E6C046412E8640FFFFEF7F3D
:1010E000EF39FAFE422E864051302DD5104987C087
:1010F000422ED63FB1A2F03F70ED0000D0A4BE72E8
:101100006937663EF16BD2C541BDBB3E2CDE25AFD3
:101110006A56113F93BDBE166CC1663F3E5555558C
:101120005555C53F0000F03FFE822B654715F73F40
:101130000000E0FE422EE63F763C7935EF39EA3D8D
:10114000FFFFEF3D9C7500883CE4377E03FCFFFF0A
:10115000F0B5BA4B8DB00E00994223DC4B005B0812
:10116000034307D1002200230020B5490CF096FB71
:101170000DB0F0BD002906DA02000B000DF00AFAEE
:1011800000220023F2E7AF4B00220CF091FF362340
:101190000E005B42AC4A964206DD02000B000CF0EA
:1011A00061F8E5E70023F5E7A84C3215121936037C
:1011B000A74CD218330B02931C1980235B032340E6
:1011C000A44C029D5C401B159B18254300930022F4
:1011D000A04B29000DF0DEF9029B060002331B0331
:1011E0000F001B0B0022022B64DC00230BF0BEFA65
:1011F000002819D0009B002B00D11CE118000DF035
:1012000047FD954A954B04000D000CF051FF944AA0
:1012100006000F00934B200029000CF049FF02004C
:101220000B0030003900BAE78F4A904B300039008C
:101230000CF03EFF02000B0000208D490DF0AAF9D2
:10124000320004000D003B00300039000CF030FF8C
:101250000B000200290020000CF02AFF009B0290E6
:101260000391002B06D102000B00300039000DF075
:1012700091F97DE700980DF00BFD774A774B04005C
:101280000D000CF015FF764A00900191754B20007F
:1012900029000CF00DFF02000B00029803990DF0DD
:1012A00079F932003B000DF075F902000B0000984F
:1012B0000199DCE78023DB050BF0D4FF02000B0073
:1012C000300039000CF0EAFA0490059100980DF016
:1012D000DFFC049A059B06900791100019000CF0A2
:1012E000E7FE644A029B944663440B9302000B00A2
:1012F000089009910CF0DCFE04000D005E4A5F4B83
:101300000CF0D6FE5E4A5F4B0BF0ACFF22002B00C8
:101310000CF0CEFE5C4A5D4B0BF0A4FF22002B00CC
:101320000CF0C6FE5A4A5B4B0BF09CFF089A099BD7
:101330000CF0BEFE584A08900991584B2000290035
:101340000CF0B6FE564A574B0BF08CFF22002B00D8
:101350000CF0AEFE544A554B0BF084FF22002B00DC
:101360000CF0A6FE02000B00089809990BF07AFF1A
:10137000029A4F4B04009B1A0B9A0D001343002B4B
:1013800034DD00223A4B300039000CF091FE32007F
:101390003B000CF08DFE0290039102000B00200038
:1013A00029000BF05FFF049A059B0CF081FE009B67
:1013B00004000D00002B06D102000B0002980399D7
:1013C0000DF0E8F84FE7244A244B069807990CF0F3
:1013D0006FFE234A0090019106980799214B0CF06B
:1013E00067FE22002B000BF03DFF54E702000B00CC
:1013F000300039000DF0CEF8049A059B0CF058FE31
:10140000009B04000D00002B02D102000B002CE712
:10141000114A124B069807990CF04AFE104A0090A8
:101420000191069807990F4B0CF042FE02000B0049
:101430002000290033E70020002199E6FFFF0F007C
:10144000000050C300005043FFFFEF7F01FCFFFF8F
:10145000645F09000000F03F0000E0FE422EE63F1E
:10146000763C7935EF39EA3D555555555555D53FBB
:101470000000E03F86EBF9FF44523EDF12F1C23F2D
:10148000DE03CB966446C73F599322942449D23F4A
:10149000935555555555E53F9FC678D0099AC33F9A
:1014A000AF788E1DC571CC3F04FA97999999D93FB1
:1014B00051B80600434218434900C00F4908014390
:1014C0000348401A414201430120C90F401A7047A6
:1014D0000000F07F03004042184349004908C00F54
:1014E00008430249081AC00F7047C0460000F07F49
:1014F000564BF0B51A0085B005000C000A409A4220
:101500000FD102000B000CF0D3FD02000B002800ED
:1015100021000BF0A7FE05000C002800210005B0FB
:10152000F0BD0200002910DC4B005B080343F4D03F
:101530000020814200D180E00B0028000DF02AF845
:1015400002000B000CF0AAF9E5E7081575D0404B36
:101550000903C0188023090B5B031943C30703D594
:10156000D30F4900C91852000024431049000393C7
:10157000D30FCB188021162520005200890346186E
:101580009E4202DC70189B1B6418D60F5B00013D65
:101590009B1952004908002DF1D1202680272900EF
:1015A00001963F067E19B446834202DC14D196426E
:1015B00012D865466646ED190290002E03DAEE4316
:1015C000F60F861902961B1A6245804140421B1A8B
:1015D0006046121A0298C919D60F5B00F318019ED3
:1015E0005200013E7F080196002EDBD1134303D049
:1015F0004B1C27D131000134164B6010C01849082C
:10160000E30702D580231B061943039B0D001C052D
:1016100023181C0081E7D10A153B52050029FAD096
:101620008024640321420AD020241600241AE640B4
:10163000451E82403143581B89E70023EEE74900ED
:101640000130EFE7012301319943D5E70000F07F36
:1016500001FCFFFF0000E03FF0B54F005E008DB0E1
:101660007F087608B74205DA3C0037002600040000
:1016700010002200330000920193F0223900040090
:101680003D00BB1B9204934206DD009A019B0BF0C8
:10169000E9FD04000D0017E0804B9F4200DCA1E053
:1016A0007F4B9F4214DD3F033F0B074305D0009A59
:1016B000019B0BF0D7FD04000D007A4B5E40009BB0
:1016C0001E4301D1009C019D200029000DB0F0BDFA
:1016D000754BF618FF18009A019B33000092019396
:1016E00096233D009B000893704B9E421BDC704B81
:1016F0009E4200DD78E0009B3343E5D000980199DD
:1017000000226C4B0CF0D4FC002200900191694B3C
:10171000200029000CF0CCFC674A040094460D0020
:10172000089B63440893009A019B200029000CF059
:1017300031FF0200099102900B0004910098019979
:101740000BF01AF8002200285ED03B001000390090
:1017500016000CF0ADFC009B049005919C46009A8D
:10176000019B8020614600068446029101996144F4
:101770000391029803990CF09BFC320000900191B8
:101780003B00200029000BF06DFD32000290039118
:101790003B00200029000CF0FDFE02000B00029827
:1017A00003990CF085FC02000B00009801990CF0E5
:1017B000F1FE02000B00049805990CF0EBFEFFF718
:1017C00097FE089B04000D00002B00D17CE7002051
:1017D0003A4A1B0599180B000200290020000CF062
:1017E00067FC56E700237EE79623354A9B0594461F
:1017F000FF18F618089B3D0063440893009A019B6C
:101800003300009201938EE7330080210692079304
:10181000002249037B180698079916001F000CF058
:1018200047FC0A900B918020000684460299049B95
:1018300004910999029A61440591049805990CF064
:1018400037FC2200029003912B00200029000BF0AE
:1018500009FD32003B000CF09DFE009A019B0CF04C
:1018600027FC069A079B04000D00009801990CF0D4
:1018700091FE32003B000CF01BFC02000B0020002C
:1018800029000BF0EFFC02000B00029803990CF00A
:1018900081FE02000B000A980B998EE70000305F72
:1018A000FFFFEF7F0000F07F000080DAFFFFAF2036
:1018B000FFFF0F000000D07F02FCFFFF0000F03FA1
:1018C000A8FDFFFFF0B589B002920393464A4B0092
:1018D00005000C005B08934203DC0DF0A3F900281F
:1018E0004CD02A002300280021000CF0E1FB060068
:1018F0000F0002000B00280021000CF0D9FB3B4A2E
:10190000009001913A4B300039000CF0D1FB394A7C
:10191000394B0CF03FFE32003B000CF0C9FB374A5C
:10192000374B0BF09FFC32003B000CF0C1FB354AFB
:10193000354B0CF02FFE32003B000CF0B9FB334B63
:10194000334A0BF08FFC0E9B04900591002B19D1AC
:1019500002000B00300039000CF0AAFB2D4A2E4B80
:101960000CF018FE009A019B0CF0A2FB02000B0089
:10197000280021000BF076FC05000C002800210057
:1019800009B0F0BD002202980399244B0CF090FBA3
:10199000049A059B06900791009801990CF088FB2A
:1019A00002000B00069807990CF0F4FD32003B0092
:1019B0000CF07EFB029A039B0CF0ECFD154A06002E
:1019C0000F0000980199144B0CF072FB02000B0001
:1019D000300039000BF046FC02000B00280021000B
:1019E0000CF0D8FDC8E7C046FFFF3F3E7CD5CF5A7C
:1019F0003AD9E53DEB9C2B8AE6E55A3E7DFEB15790
:101A0000E31DC73ED561C119A0012A3F1111813FD5
:101A1000A6F81011495555555555C53F0000E03FF2
:101A2000F8B50022324B0CF043FB002200230600E5
:101A30000F000AF09BFE002854D100222D4B3000ED
:101A400039000AF093FE00284FD132003B003000ED
:101A500039000CF02DFB04000D00274A274B0CF039
:101A600027FB274A274B0CF095FD22002B000CF09A
:101A70001FFB254A254B0BF0F5FB22002B000CF039
:101A800017FB234A234B0CF085FD22002B000CF0A2
:101A90000FFB214A214B0BF0E5FB22002B000CF041
:101AA00007FB1F4A1F4B0CF075FD22002B000CF0AA
:101AB000FFFA1D4A1D4B0BF0D5FB22002B000CF04A
:101AC000F7FA1B4A1B4B0CF065FD22002B000CF0B3
:101AD000EFFA194A194B0BF0C5FB32003B000CF032
:101AE000E7FAF8BD00200021FBE700201449F8E7E1
:101AF0000000E03F0000D03F98456D69B8D1B93F84
:101B0000722CC67097F7E63FA79ED5E9358F0E4039
:101B10000CD7D1DD74302E40CB905148830745401F
:101B2000437562CE2C2D53406EAA7567BC66544037
:101B300052BE25E6BCAB4440182D4454FB2119404D
:101B40000000F03FF8B505000C00FFF7B3FC0028DB
:101B500000D0E3E000220023280021000AF00CFE60
:101B600000280BD0280080252D066119FFF7EAFF19
:101B70004919002200230BF075FBF8BD0022002359
:101B8000280021000AF0F2FD061E02D0002001000C
:101B9000EFE70022644B280021000AF0E7FD00284F
:101BA00000D0BEE00022614B280021000AF0DEFDDB
:101BB0000028EBD15E4A60002300400890420BDD14
:101BC0002A00280021000BF04DFB02000B000BF057
:101BD00065FE05000C000FE08027E20F2900D20708
:101BE000FF05B84215DC07D1002D12D1D20FD3006A
:101BF000504AD218156F546F00224B4B2800210019
:101C00000AF0C4FD002857D028002100FFF708FF84
:101C1000AFE780241B031B0B64031C43464B0015DA
:101C2000C018464BE318002816D1002B00DA230019
:101C30001C0001200C43D9D0414CA3421ADD414C79
:101C4000A0421DDB3D4C0D001B191A433E4BC01832
:101C5000000502431400CFE7002B05DA6400CB0F28
:101C60001C1949000138DCE71C000C43BED05B00A6
:101C7000CC0FF5E7CD0F5B005B1949000138DCE7BD
:101C8000241A142C0ADC314DE14040191D00854016
:101C900023410D431A43110028009AE71F2C07DC4B
:101CA000E1402A4C001983400B431D001300F1E76B
:101CB0002749081A0341F8E700221C4B280021009D
:101CC0000AF064FD002806D02A00230000201749EE
:101CD0000CF060FC9AE700221E4B280021000AF05D
:101CE00055FD002200280AD0280021000F4B0CF0DF
:101CF00051FCFFF795FE80231B06C91839E78023A6
:101D00002800DB0521000AF041FD002800D13DE755
:101D100080212A0023000020C905E8E700200E49A1
:101D200027E73000014924E70000E03F0000F03FD2
:101D3000FFFFEF7F70ED000000FCFFFF0000F0FFF1
:101D4000FFFF0F0002FCFFFFFF0300001E04000066
:101D5000E2FBFFFF0000F83F0000F87FF0B587B01E
:101D6000049205934B005B080093009A484B0500D2
:101D70000C009A4204DC0CF055FF002800D184E0EE
:101D80002A002300280021000CF092F90022414B88
:101D900006000F000CF08CF93F4A029003913F4B74
:101DA000300039000CF084F93D4A3E4B0BF05AFAF2
:101DB00032003B000CF07CF93B4A3C4B0CF0EAFB58
:101DC00032003B000CF074F9394A3A4B0BF04AFAF6
:101DD00032003B000CF06CF9374A384B0CF0DAFB60
:101DE00032003B000CF064F9354A364B0BF03AFAFE
:101DF00032003B000CF05CF932003B000CF058F96B
:101E0000049A059B06000F00280021000CF050F9F1
:101E100002000B00300039000CF0BCFB2A4B009A8A
:101E200004000D009A420DDC02000B000298039999
:101E30000CF0B0FB020000200B0024490CF0AAFBC0
:101E400007B0F0BD224B009A00269A421BDC13001B
:101E5000204A944663441F0032003B0000201B4987
:101E60000CF098FB320000900191029803993B001E
:101E70000CF090FB22002B000CF08CFB02000B00FE
:101E800000980199DAE7144FE6E700200F49D7E7F9
:101E9000FFFF3F3E0000E03FD43888BEE9FAA8BD0E
:101EA000C4B1B4BD9EEE213EAD529C804F7E923EA9
:101EB0009015CB19A001FA3E7751C1166CC1563F5F
:101EC0004C5555555555A53F3233D33F0000F03F93
:101ED0000000E93F0000E0FF0000D23F70B51400B1
:101EE0004A000B00520D0DD14B005B0803430FD08D
:101EF000224B00220CF0DCF8214B9C4209DA214AEB
:101F0000214B17E0214DAA4207D102000BF0AAF99C
:101F100070BD0B004A00520D363A1D4DAC420CDD2F
:101F2000C90F1C48C907084303001B4A19001000C9
:101F3000184B194A0CF0BCF8EAE7A218174CA24259
:101F4000EEDC002A05DD164C120523401343190070
:101F5000DEE71400353408DAC90F0B48C907084317
:101F60000300084A19001000C9E70D4C363223401F
:101F700012051A4311000B4B0022DBE7000050430F
:101F8000B03CFFFF59F3F8C21F6EA501FF07000028
:101F900050C300003CE4377E9C750088FE070000BB
:101FA000FFFF0F800000903CF0B54B00394A5B0DFD
:101FB00085B09E180D0004000390132E33DC002E14
:101FC00014DA354A354B0BF04DF9002200230AF0A4
:101FD000E7FB002807D0002D58DA6B005B081C4394
:101FE00001D000242E4D2000290026E02D4F37413E
:101FF0003B000B40034320D000900191264A274B21
:10200000009801990BF02EF9002200230AF0C8FB7A
:102010000028E8D0002D03DA80235B033341ED185C
:10202000BD430024DFE7332E09DD8023DB009E4221
:1020300003D102000B000BF015F905B0F0BD01272C
:10204000194A7F429B18DF403842F6D00090019138
:10205000114A124B009801990BF004F90022002359
:102060000AF09EFB0028BED0002D02DA142E02D109
:102070000135BC43B7E734239E1B333BB340E41820
:10208000039B9C429B415B42ED18F2E70024250034
:10209000A9E7C04601FCFFFF9C7500883CE4377E41
:1020A0000000F0BFFFFF0F00EDFBFFFFF0B5D14CCC
:1020B000A54408900991D01E1821140002930AF03B
:1020C00051FA1823421C5B4253431B19002400930E
:1020D000029B05905D1EDF1C451BC74BAE00F6182A
:1020E000EC4200D5F1E0A300F0580CF0D1FDE30084
:1020F00022AAD318013418605960A742F0DA0024EC
:10210000029BDB00D3180793079B00261D190023B1
:1021100000270693069B089ADB00E91A0839D318B2
:102120001A685B68086849680BF0C2FF02000B0080
:10213000300039000BF096F8069B06000133069339
:10214000069A029B0F009342E4D172AB1B1908342C
:102150001E605F60282CD7D10426059BA64A9B00F1
:102160009B180A93370072AAF300D3181C685D68A5
:102170000EA9B3005B1805930B9200229F4B200021
:1021800029000BF095FF0CF04DFD0CF081FDBB001C
:102190005B42079300229A4B029003910BF088FF59
:1021A00002000B00200029000CF0F4F90CF03AFDBD
:1021B000059B079A013F98500B9AFB00D3181A68A9
:1021C0005B68029803990BF04DF804000D00002F96
:1021D000D3D1009AFFF782FEFF2300229B05040063
:1021E0000D000BF065FFFFF7DFFE0022854B0BF0C3
:1021F0005FFF02000B00200029000CF0CBF90D005E
:1022000004000CF00FFD07900CF042FD0B000200E3
:10221000290020000CF0BEF9009B04000D00002BEB
:1022200056DD721E92000EAB9B5818211F000098BD
:10223000091A0F410798C0198F40DF1B0EAB9F5042
:102240001723009A07909B1A1F410597059B002BA7
:102250004FDD079B00270133079380235B043A007F
:102260009C4691000EABCB58002F00D0A5E0002B70
:1022700004D06746FB1A0EAFCB51012701329642BC
:10228000EFD1009B002B05DD012B00D19AE0022B42
:1022900000D1A1E0059B022B2BD122002B000020B6
:1022A00059490CF077F904000D00002F21D0009A55
:1022B00000205549FFF712FE02000B002000290004
:1022C0000CF068F904000D0013E0002000210EE777
:1022D000009B002B06D1731E9B000EAAD758FB153E
:1022E0000593B3E70022494B0AF064FA002861D154
:1022F000059700220023200029000AF037FA002861
:1023000000D1E0E00022731E0293013B022B00D0BB
:102310006AE0002A00D19BE0009B0EAA183B0093C4
:10232000029B9B009B58002B00D1C8E0009A002024
:102330003549FFF7D3FD06000F00029C002C00DB9F
:10234000FCE00025029B324FDC0072AB1C19029BA3
:102350005B1B00D40AE100263500029C002C00DB48
:1023600029E1059B2900002B02D080231B06E918D8
:102370000B003200099901240A604B604A984B997E
:102380002B000CF007F9029BA34200DB20E1059B28
:10239000002B02D080231B06C91802000B00072067
:1023A00009998A60CB60079B034018009B239B0020
:1023B0009D44F0BD022305934BE71648C31A0EA8AF
:1023C0000B505BE7721E92000EAB9B5802935B02B0
:1023D0005B0A0EA98B505DE7721E92000EAB9B58F4
:1023E00002939B029B0AF4E799000EA8091849681A
:1023F0000A438AE794FDFFFF98F600000000703E54
:1024000000007041000020400000F03F0000E03F6D
:10241000F0ED0000FFFFFF0001339A008A1A1269F5
:10242000002AF9D0721C0292069A00249219D20056
:102430000792079922AA8C4662440C92F318F20084
:102440000D920593029B059A934204DD160089E6DE
:1024500001230EA9E1E7079B0A9A1D1922AB5D191A
:10246000029B00269B00D0580CF012FC002728602D
:10247000696000250C9B1B190B93089AEB00D1187F
:102480000B9A08684968D31A1A685B680BF010FE4B
:102490000B000200390030000AF0E4FE069B013513
:1024A00006000F00AB42E8D10D9B72AA1B19D3188E
:1024B0009E60DF60029B083401330293C2E7029BF7
:1024C000013B029328E7009B20005A422900FFF7B6
:1024D00005FD0022434B04000D000AF06BF90028B3
:1024E00023D00022404B200029000BF0E1FD0CF02E
:1024F00099FB07000CF0CCFB00223A4B0BF0D8FD07
:1025000002000B00200029000CF044F80CF08AFBBC
:102510000EABB200D050731C0293009B0EAA18336E
:102520000093029B9B009F5000E7200029000CF0C5
:1025300079FBB7000EABF8500296F7E6E50072ABF8
:102540000EAA5D19A30098580CF0A2FB32003B00C4
:102550000BF0AEFD002228606960234B300039008B
:102560000BF0A6FD013C06000F00E7E60022002369
:10257000002600920193B54213DBF300F918E3182B
:102580001A685B68086849680BF092FD02000B004E
:10259000009801990AF066FE013600900191052E1F
:1025A000E9D1EB004AAAD31801350099019A083CF9
:1025B00019605A60CBE6E3004AAAD31830001A68C3
:1025C0005B6829000AF04EFE013C06000D00C5E6DE
:1025D000E3004AAAD3181A685B680AF043FE013484
:1025E000D1E6C046000070410000703E49004B0833
:1025F00019007047F7B54B005B080193019A3F4BF8
:102600009A4204DD02000B000BF052FD2BE03C4B24
:10261000019A9A422DDCFFF7E9FFFEF721FA00222A
:10262000384B06000F000AF01DFE374B019A0400DC
:102630000D009A4219DD32003B00300039000BF0EA
:1026400037FD220006000F002B00200029000AF0B1
:1026500009FE02000B00300039000BF01FF90022C8
:10266000284B0AF0FFFD04000D002000290003B0F4
:10267000F0BD264B019A9A4216DCFFF7B7FFFEF732
:1026800005FC0022224B04000D000BF011FD22007E
:1026900006000F002B0000201D490BF0FFF8020080
:1026A0000B0030003900DCE71A4B019A9A4206DC35
:1026B000FFF79CFFFEF7EAFB0022154BA4E7164B41
:1026C000019A9A4205DD154B9A4213D1144A904261
:1026D00010D8FFF78BFF00220D4B0BF0E9FCFEF743
:1026E000D5FB04000D000022094B0BF0E1FC220099
:1026F0002B0089E70020FEF79FF9B4E7FFFFEF7F8B
:10270000422ED63F0000F03FFFFF7F3CFFFF3540E9
:102710000000E03F412E8640CD338640CE338640D8
:102720007DF8B98FF0B54C4A4E0085B005000C001D
:102730000B007608964208DD02000AF093FD0500C2
:102740000C002800210005B0F0BD0022002944DA69
:10275000424B00920193424B9E424FDC414B9E42C2
:102760000BDC414A414B280021000AF07BFD00228E
:102770003F4B0AF015F80028E3D128002100FFF7AD
:1027800035FFFEF76DF93B4B04000D009E4226DC41
:1027900002000B000AF066FD2200029003912B005C
:1027A000200029000BF084FC002206000F00304BB3
:1027B000200029000AF056FD02000B00300039000D
:1027C0000BF06CF802000B00029803990BF0E2FE8C
:1027D000009A019B0BF06CFCB1E7274BB9E7002294
:1027E000234B0AF03FFD02000B00200029000BF0F4
:1027F00055F822002B000AF035FDE9E71F4B9E42F9
:1028000006DC28002100FFF7F1FEFEF73FFBDFE7C3
:102810001B4B9E4205DD1B4B9E4217D11A4A954227
:1028200014D828002100FFF7E1FE0022124B0BF024
:102830003FFCFEF72BFB04000D0002000B0000988C
:1028400001990BF035FC22002B00C3E7064A074B29
:1028500028002100BEE7C046FFFFEF7F0000E0BF79
:10286000FFFF3540FFFF2F3E3374AC3C1F7BAC7F36
:102870000000F03FFFFFEF3F0000E03F412E8640A9
:10288000CD338640CE3386407DF8B98FF7B517003B
:102890001E0004000D00FFF7A9FE00221B4B09F0EB
:1028A00075FF00280CD020002900FFF7A3FE386038
:1028B000796020002900FFF735FF30607160F7BDB7
:1028C00020002900FEF7E2FA04000D0002000B00D0
:1028D00000200E490AF0E2FF0022009001910B4B0C
:1028E000200029000BF0E4FB009A019B04000D007E
:1028F0000BF050FE220030607160009801992B00AF
:102900000AF0B0FC38607960D9E7C0460000E03FCB
:1029100082B0F0B58BB00190109211930022129802
:102920001399002309F022FF0022002300283ED043
:102930001098119909F01AFF00280CD012981399D9
:10294000002200230BF0B4FB002200230AF08AFCD3
:10295000129C139D19E010981199FFF747FEFEF79E
:10296000C7FD0022002304000D001098119909F002
:1029700003FF00220023002812D0200029000BF0C2
:1029800097FB002200230AF06DFC019B1860596040
:102990009C60DD6001980BB0F0BC08BC02B0184729
:1029A000129813990BF084FB22002B00CEE71098AD
:1029B000119909F0DBFE002830D012981399FFF727
:1029C00015FE0022764B0BF073FBFEF791FD002203
:1029D000002305000C000BF06BFB002206000F002B
:1029E00012981399002309F0DBFE32003B00002807
:1029F00004D0280021000AF035FC06E02800210060
:102A00000BF0C8FD80231B06E418019B2A00186008
:102A10005960230001998A60CB60BBE71098119937
:102A2000FFF7E4FD00225F4B09F0BAFE00280AD14F
:102A300012981399FFF7DAFD00225A4B09F0B0FE05
:102A4000002800D175E0109811990022564B0BF028
:102A50002FFB0022544B04000D00129813990BF029
:102A600027FB8023002202900391DB05049205934B
:102A700002980399002200230BF01AFB22002B007E
:102A80000AF0F0FB029A039BFEF7E6FD0022444B9E
:102A90000BF00EFB002206900791414B200029000D
:102AA0000BF006FB002206000F00029803993C4B36
:102AB0000BF0FEFA00220890099100232000290063
:102AC00009F06EFE32003B00002846D006980799B8
:102AD0000AF0C8FBFEF70CFD02000B0006000F0019
:102AE000089809990AF0DAFEFFF780FD049A059B21
:102AF0000BF0DEFA32003B0005000C00049805994B
:102B00000BF0D6FA06000F00002200232800210057
:102B10000BF0CEFA0022049005910298039900234D
:102B200009F02AFE049A059B002835D030003900B0
:102B300066E70022109811991C4B0BF0B9FA00229D
:102B40001A4B04000D00129813990BF0B1FAF923F7
:102B50000290039100229B0588E7069807990BF0E5
:102B600019FDFEF7C5FC02000B0004000D000898DB
:102B700009990AF093FEFFF739FD049A059B0BF0C3
:102B800097FA22002B0006000F00049805990BF01D
:102B90008FFA05000C00B7E7300039002BE7C0467C
:102BA0000000E03F000010400000D03F0000504314
:102BB000F0B593B002920393039B0E0002995D005F
:102BC00004930B006D0807002B4319D180210903E2
:102BD000714002000B0092185B419B498B4206D862
:102BE00001D000F0C7FC002A01D100F0C3FC029A1A
:102BF000039B380031000AF035FB009001917CE026
:102C0000924B74000896009064089C469C4207DC36
:102C100001D1002804D1654502DC0CD100290AD07D
:102C20008B4BF3183B43E2D18021039809034840C2
:102C3000029A0300CFE700230693002E17DA854A95
:102C400095424BDC844A954211DD844B2A15D218FB
:102C5000142A23DD3420821A0298D04003009340C6
:102C60008B4204D1012210409218131A06930029B6
:102C70005ED1654521D1764BE3181F4301D100F0A9
:102C800079FC754B9C422BDD049B002B01DA00F094
:102C900075FC029B039C009301942EE0002947D110
:102CA00014239A1A2B00134119009140A94204D110
:102CB000012213409218D31A0693694B9D4220D1EA
:102CC00038003100049B00900191002B15DA3A0086
:102CD0003300002062490AF0E1FD8EE70223C5E7D8
:102CE000049B002B01DB00F049FC80221206944675
:102CF000029B0093039B634401930098019913B0D6
:102D0000F0BD8023049ADB059A4206D13A003300D5
:102D1000380031000BF0CCF96FE7524B049A9A421D
:102D200006D1002E04DB38003100FEF7E1FB64E73A
:102D300038003100FFF75AFC00900191002F2ED18E
:102D4000002C04D0464AB3009B08934227D1049B31
:102D5000002B07DA009A019B002041490AF09EFDF2
:102D600000900191089B002BC7DA394BE418069BB1
:102D70001C4308D1009A019B100019000BF00AFCBB
:102D800002000B00A7E7069B012BB6D1009880211B
:102D9000020001980906431800920193ADE7F20F73
:102DA000069B013A134304D13A0033003800310046
:102DB000E4E7069B013B13430022002B14D0284B71
:102DC000069207938423DB059D4200DC0AE1264B33
:102DD0009D4212DD204B9C4208DC049B002B08DA4C
:102DE0000020FDF729FE08E7204BE9E7049B002BB4
:102DF000F6DC0020FDF70CFEFFE61D4B9C420FDCCD
:102E0000069807990023002209F0B6FC431E98415A
:102E100001244042049B04402000002BEADAE0E752
:102E20000F4B9C4226DD069807990023002209F0EB
:102E3000A3FC431E984101244042049B044020000F
:102E4000002BCEDCD6E7C0460000F0FF0000F07F8C
:102E5000000010C0FFFF3F43FFFFEF3F01FCFFFFFB
:102E60000000F03F0000E03F0000F0430000F0BF32
:102E7000FEFFEF3F0098019900224F4B0BF08AFBB9
:102E8000C0224E4BD20506000F000BF011F94C4A40
:102E9000049005914B4B300039000BF009F90022EA
:102EA00000900191484B300039000BF001F902000D
:102EB0000B00464846490BF06DFB32003B000BF01F
:102EC000F7F802000B00002042490BF063FB3200D0
:102ED00004000D003B00300039000BF0E9F802005F
:102EE0000B00200029000BF0E3F83B4A334B0BF0BA
:102EF000DFF802000B00009801990BF04BFB020079
:102F00000B0004000D00049805990AF0ABF9049A2F
:102F1000059B0020009001910BF03CFB02000B0090
:102F2000200029000BF036FB029C039D00240600C4
:102F30000F000298039922002B000BF02BFB009A44
:102F4000019B0BF0B5F8029A039B049005913000A9
:102F500039000BF0ADF802000B00049805990AF057
:102F600081F922002B0002900391009801990BF047
:102F70009FF806000F000B000200029803990496C8
:102F800005970AF06FF9154B05000C00089199425E
:102F900000DCCAE2124BCB18034300D1CCE1069807
:102FA00007990023002209F0E7FB431E9841012402
:102FB00040420440200014E70000F03F4715F73F6F
:102FC00044DF5DF80BAE543E0000D03F55555555DB
:102FD0005555D53F0000E03FFE822B65FFFF8F4037
:102FE000000070BFBB4B00229C420ADC0098019994
:102FF0000022B94B0BF05CF8352200900191019C46
:103000005242B64923155B189B182403B44DB54AA8
:103010000E93230B1D430024934209DDB24A013471
:10302000934205DD0E9B1B1900240E93AF4BED1848
:10303000009801992900AE4AE300D3180F931A6C47
:103040005B6C0C900D910A920B930BF0A3FA0C9A07
:103050000D9B06000F000A980B990AF003F9020075
:103060000B0000209E490AF019FC109011910200FB
:103070000B00300039000BF01BF808900991089AFA
:10308000099B802104920593002389056D100D434F
:1030900080210493049A059B009201930022090366
:1030A0006D18A4042B190098019914001D000AF052
:1030B000FFFF02000B00300039000BF06BFA0A9A98
:1030C0000B9B06000F00200029000BF063FA0200A2
:1030D0000B000C980D990BF05DFA009A019B0AF019
:1030E000E7FF02000B00300039000BF053FA109A92
:1030F000119B0AF0DDFF089A099B0A900B911000C2
:1031000019000AF0D5FF06000F007A4A7A4B0AF040
:10311000CFFF7A4A7A4B0AF0A5F832003B000AF05A
:10312000C7FF784A784B0AF09DF832003B000AF05E
:10313000BFFF764A764B0AF095F832003B000AF062
:10314000B7FF744A744B0AF08DF832003B000AF066
:10315000AFFF724A724B0AF085F8320004000D008E
:103160003B00300039000AF0A3FF02000B002000F2
:1031700029000AF09DFF009A019B04000D000898A9
:1031800009990AF06FF80A9A0B9B0AF091FF220046
:103190002B000AF067F8009A019B0C900D9110002B
:1031A00019000AF085FF00225E4B04000D000AF0B2
:1031B00059F80C9A0D9B0AF055F8049E0F00320046
:1031C0000B00009801990AF073FF00220090019112
:1031D000544B300039000BF0DDF922002B000BF0CE
:1031E000D9F902000B000C980D990BF0D3F9089A4D
:1031F000099B0AF05DFF320004000D000A980B994C
:103200003B000AF055FF02000B00200029000AF0E5
:1032100029F804000D0002000B00009801990AF043
:1032200021F8E022049E12063F4B30000F000AF006
:103230003FFF08900991009A019B300039000BF084
:10324000A9F902000B00200029000BF0A3F9374A6E
:10325000354B0AF02DFF364A04000D00354B300087
:1032600039000AF025FF02000B002000290009F0B8
:10327000F9FF0F9B1A6D5B6D09F0F4FF0A900B913B
:103280000E980BF005FD04000D00089809990F9B9E
:103290001E6E5F6E0A9A0B9B09F0E4FF32003B0042
:1032A00009F0E0FF22002B0009F0DCFF0498220067
:1032B0002B00009001910BF06DF932003B000BF0F8
:1032C00069F9089A099B0BF065F902000B000A984E
:1032D0000B9927E6FFFF0F000000404301FCFFFFB2
:1032E0000000F03F8E98030079B60B000000F0FF5D
:1032F000F0ED0000EF4E454A287ECA3F65DBC993DA
:103300004A86CD3F01411DA96074D13F4D268F51A2
:103310005555D53FFFAB6FDBB66DDB3F0333333322
:103320003333E33F0000084009C7EE3FFD033ADCBA
:10333000F5015B14E02F3EBE924A934B029803992D
:1033400009F090FF3200009001913B00280021001D
:103350000BF020F902000B000098019909F020FA07
:10336000002800D01BE60021884A63005B0800911A
:10337000934225DD864A1B159B18802252039446F2
:103380001A4114196000834B400D834DC01805414C
:103390002100A9430B0061462403240B214314247C
:1033A000201A0141009108990022002902DA0099AF
:1033B00049420091300039000BF0ECF8049005917F
:1033C000029A039B04980599002609F04BFF0022FE
:1033D000724B30000F000AF06BFE049A059B0890B8
:1033E0000991300039000BF0D5F802000B0002986B
:1033F00003990BF0CFF86A4A6A4B0AF059FE6A4A01
:1034000004000D00694B300039000AF051FE020043
:103410000B002000290009F025FF04000D00020028
:103420000B000898099909F01DFF089A099B0600EE
:103430000F000BF0AFF802000B00200029000BF08A
:10344000A9F83200029003913B00300039000AF0E5
:103450002FFE04000D00564A564B0AF029FE564A2C
:10346000564B0BF097F822002B000AF021FE544A2D
:10347000544B09F0F7FE22002B000AF019FE524AC5
:10348000524B0BF087F822002B000AF011FE504A35
:10349000504B09F0E7FE22002B000AF009FE020063
:1034A0000B00300039000BF075F804000D0002002D
:1034B0000B00300039000AF0FBFD802304900591D9
:1034C0000022DB05200029000BF064F802000B004D
:1034D000049805990AF0E2F9029A039B04000D0092
:1034E000300039000AF0E4FD029A039B09F0BAFEAD
:1034F00002000B00200029000BF04CF832003B00CA
:103500000BF048F802000B00002033490BF042F8A2
:10351000009B1B055B181A15002A29DC009AFEF790
:10352000DDFC069A079BFFF7F5FB2C4A4B005B0876
:10353000934200DC17E72A4BCB1803430CD00698C4
:1035400007990023002209F017F9431E984101242E
:103550004042044020004DE432003B000BF01AF8DA
:10356000029A039B09F026F9002800D1FBE6E6E762
:103570001900D6E70023184CFFF78DFB0023002429
:10358000FFF789FBFE822B654715973C0000E03F63
:1035900002FCFFFF01FCFFFFFFFF0F00432EE63F91
:1035A000EF39FAFE422EE63F396CA80C615C20BE72
:1035B000D0A4BE726937663EF16BD2C541BDBB3E39
:1035C0002CDE25AF6A56113F93BDBE166CC1663F17
:1035D0003E5555555555C53F0000F03FFFCB904037
:1035E00000346F3FF0B5984B85B04E0004000D00DD
:1035F000039176089E4218DD944B9E4202DC0AD16C
:10360000002808D022002B002000290009F02AFE03
:1036100004000D0005E0039B8D4C002B00DC10E145
:103620008C4D2000290005B0F0BD8B4B9E420FDC75
:103630008A4B9E4209DC8A4A8A4B09F013FE00221B
:10364000894B09F0ADF80028EBD101235B4225E05E
:10365000FEF7CCFF854B04000D009E4200DDAAE082
:10366000834B9E4200DD90E002000B0009F0FAFD62
:1036700000227D4B0AF08EFF802306000F000022FF
:10368000DB052000290009F0EDFD0B0002003900E8
:1036900030000AF003F9002304000D000293220019
:1036A0002B00200029000AF003FD02000B0000900F
:1036B00001910AF0FDFC06000F006E4A6E4B0AF005
:1036C000F7FC6E4A6E4B09F0CDFD32003B000AF06C
:1036D000EFFC6C4A6C4B09F0C5FD32003B000AF070
:1036E000E7FC6A4A6A4B09F0BDFD32003B000AF074
:1036F000DFFC684A684B09F0B5FD32003B000AF078
:10370000D7FC664A664B09F0ADFD009A019B0AF0B2
:10371000CFFC644A00900191634B300039000AF0FD
:10372000C7FC624A624B0AF035FF32003B000AF0E8
:10373000BFFC604A604B0AF02DFF32003B000AF0EC
:10374000B7FC5E4A5E4B0AF025FF32003B000AF0F0
:10375000AFFC5C4A5C4B0AF01DFF32003B000AF0F4
:10376000A7FC02000B000098019909F07BFD2B00DB
:1037700022000AF09DFC029B013343D102000B00A2
:10378000200029000AF006FF42E70022364B0AF02B
:1037900001FF002206000F00334B2000290009F032
:1037A00061FD0B000200390030000AF077F80123B8
:1037B00004000D0072E7454B9E4219DC0022444B89
:1037C0000AF0E8FE002206000F00414B200029000D
:1037D0000AF06EFC0022244B09F044FD0B000200AD
:1037E000390030000AF05AF8022304000D0055E7B2
:1037F0000B000200374900200AF050F803230400B0
:103800000D004BE7029B344FDE00344BBF199E196D
:10381000326973690AF0BEFE22002B000AF0BAFE7C
:103820000B000200386F796F0AF0B4FE039B0400AE
:103830000D00002B00DBF4E6802109066B181D004B
:10384000EFE6274DEDE6C046FFFF0F440000F07F96
:10385000182D4454FB21F93FFFFFDB3FFFFF1F3EC4
:103860009C7500883CE4377E0000F03FFFFFF23F8C
:10387000FFFFE53F11DA22E33AAD903FEB0D7624EE
:103880004B7BA93F513DD0A0660DB13F6E204CC58A
:10389000CD45B73FFF8300922449C23F0D55555592
:1038A0005555D53F2F6C6A2C44B4A2BF9AFDDE5209
:1038B0002DDEAD3F6D9A74AFF2B0B33F711623FEAB
:1038C000C671BC3FC4EB98999999C93FFF7F0340EB
:1038D0000000F83F0000F0BFF0ED000070EE0000C7
:1038E000FB21F9BFF7B554425E001443484F7608F8
:1038F000E40F00933443BC4209D844424D000443D2
:103900006D08E40F009101902C43BC4203D909F0EB
:10391000A9FC03B0F0BD3F4C1C19144302D1FFF7C2
:1039200061FEF6E79C17A446022467463C40009FD0
:10393000FF0F3C43019F2F4306D1022C62D0032C82
:10394000E7D135483549E4E73700174305D1009BF7
:103950003148002B59DA3249DBE72D4FBE421BD1EB
:10396000B5420ED1022C06D0032C07D02A48012CD8
:1039700046D12C49CDE72C482C49CAE72A482C4986
:10398000C7E7022C3ED0032CDBD000200021012C05
:10399000BFD180210906BCE71D4FBD42D7D0AD1B6A
:1039A0002D153C2D16DC002B01DA3C3515DB09F01A
:1039B00075FFFEF71BFEFFF715FE012C10D0022C41
:1039C00013D0002CA5D01B4A1B4B0AF0E3FD124A72
:1039D0001A4B12E010481A49EFE700200021ECE7EB
:1039E000802424060B19190093E7124A124B0AF09F
:1039F000D1FD02000B00084810490AF0CBFD88E712
:103A0000104986E704480D4983E70D4981E7C04620
:103A10000000F07F000010C0182D4454FB2109C0A5
:103A2000FB21F9BFFB21E9BFD221337F7CD90240C2
:103A30007CD902C0075C143326A6A13CFB210940B7
:103A4000FB21F93FFB21E93F82B0F0B589B00E922E
:103A50000F93019000220E980F99002308F086FE24
:103A6000002808D0109811990022704B08F098FE99
:103A7000002800D0CCE00E9A0F9B100019000AF02D
:103A800017FB0290039102000B00002067490AF027
:103A900081FD109A119B04000D00100019000AF01E
:103AA00007FB02000B00200029000AF073FD0E9AAC
:103AB0000F9B04000D001000190009F0D3FB220039
:103AC0002B00FFF70FFF0022594B0AF0F1FA594A79
:103AD000594B0490059109F0E1FE002200230400F7
:103AE0000D0008F067FE0022514B002800D18AE04B
:103AF0002000290009F0B6FB00224C4B04000D0009
:103B0000109811990AF046FD02000B000AF0D0FA55
:103B1000029A039B09F0A6FB00220023069007915E
:103B200008F024FE002800D072E0290020000BF0ED
:103B300079F80BF0ADF8002206000F0010981199EB
:103B40003A4B09F08FFB02000B000AF0B1FA029A1F
:103B5000039B09F087FB069A079B09F09FFEFDF780
:103B6000F7FA0022354B0AF0A3FA354A0290039186
:103B7000344B300039000AF09BFAA82206900791D6
:103B8000D2052D4B300039000AF092FA02000B00EA
:103B9000049805990AF0FEFC802204000D005205ED
:103BA000294B300039000AF083FA02000B00200094
:103BB00029000AF0EFFC002206000F00029803998A
:103BC00000230AF075FA069A079B04000D003000E6
:103BD00039000AF0DFFC02000B002000290009F088
:103BE00041FB019B00221860596002980399002351
:103BF00009F038FB019B9860D960019809B0F0BCCE
:103C000008BC02B01847200029000AF0C3FC73E783
:103C10000E4B0198196B5A6BDC6B9B6B0160426019
:103C2000029303948360C460E7E7C0460000F03F5E
:103C30000000E03F182D4454FB2109400000D03F14
:103C40006EC0453163626A3C460B213E70EE000057
:103C500082B0D3B5069207930400089A099B069890
:103C60000799FDF7F9FCFDF773FA069A079B009098
:103C7000019108980999FFF735FE002200230600FC
:103C80000F000AF015FA009A019B09F0EBFAA66002
:103C9000E760206061602000D6BC08BC02B0184715
:103CA00082B0F0B593B004001A981B99189219933A
:103CB000002200230AF0FCF9189A199B09F0D2FAA5
:103CC00000260200002700200B00454902960397BA
:103CD000049005911A981B99009001910EA808F084
:103CE00073FD0E9A0F9B08920993109A119B0A92EA
:103CF0000B93189A199B1000190009F0B3FA1A9A3D
:103D00001B9B0AF0D5F90D00079032003B00079885
:103D100029000AF0CDF91A9A1B9B06000F0018988B
:103D200019990AF037FC1A9A1B9B0C900D91189860
:103D3000199909F097FA02000B000C980D990AF0F6
:103D4000B7F932003B0009F08DFA02000B000020A9
:103D500023490AF01FFC32003B000AF01BFC8023C1
:103D60001B06ED180B0007990200019500910EA8A3
:103D7000FEF7CEFD0E9A0F9B0898099909F072FA8A
:103D8000109A119B06000D000A980B9909F06AFA27
:103D900032002B00019100900EA8FFF759FF00227E
:103DA000104B0EA804920593802300221B0602925A
:103DB0000393109A119B009201930E9A0F9B08F0A7
:103DC00003FD0E9A0F9B200022606360109A119BE6
:103DD000A260E36013B0F0BC08BC02B01847C04654
:103DE0000000F03F0000F0BF82B0F0B589B00F9343
:103DF000159B0E9207930600109A119B0E980F992F
:103E0000FDF72AFC00220023149F0290039108F082
:103E1000ADFC002810D0474B196C5A6CDC6C9B6CC5
:103E200031607260009301943000B360F46009B0B7
:103E3000F0BC08BC02B01847079B10981199069374
:103E40000E9A0F9BFFF74EFD129A139B049005915B
:103E500002980399FEF7ACFE374A0090019104984E
:103E60000599364B09F01AFD02000B0012981399C0
:103E70000AF01EF9002204000D0000233800069904
:103E800008F074FC00282AD1049A059B80200006C3
:103E900084460799049761440591049805990AF0AE
:103EA00007F9FCF7F3FF02000B00009801990AF0F4
:103EB000FFF80090019102980399FDF749F93A0043
:103EC000069B0AF0F5F81C4A1C4B09F0E7FC0200BF
:103ED0000B002000290009F0C5F904000D002000A6
:103EE0002900FDF72FFE009A019B0AF0E1F822005D
:103EF0002B0002900391002011490AF04BFBFDF7C3
:103F000021FE02000B00009801990AF0D1F800226E
:103F100004000D000298039900230AF0C9F80B0071
:103F200002002900200009F09DF9029B039C3060EB
:103F3000716079E770EE0000182D4454FB210940B0
:103F40000000E03FF0B58FB000934B005B08069394
:103F50000292D34B069A05000C000B919A425DDC4D
:103F60000AF060FE0490002800D07CE0149B069AC2
:103F700001332B4313430FD128002100FEF736FBFA
:103F800002000B000020C74909F088FC05000C0066
:103F9000280021000FB0F0BD149B012BF8D0029A2D
:103FA000009B2800210009F05DF9020004980B0035
:103FB000069007910020BC4909F070FC2A00089087
:103FC000099106980799089E099F23000AF0E2FAD2
:103FD000049E02000B00029800990AF0DBFA3200FE
:103FE0003B000AF065F8320004000D0006980799BE
:103FF0003B000AF05DF80022AA4B09F033F90200F9
:104000000B002000290009F02DF9089A099B0AF0FD
:104010004FF832003B0009F025F9B7E7A34B069AA9
:104020009A4220DD002907DA802109068C466318B0
:104030001C00009B634400932A0023009C489D4978
:104040000AF0A8FA06000F00029A009B9A489B49C2
:104050000AF0A0FA3B00320009F004F90023050041
:104060000C00029300932A002300280021000AF08C
:104070001FF802000B00049005910AF019F8049A49
:10408000059B06000F00280021000AF011F88C4A59
:10409000089009918B4B300039000AF009F88A4AE0
:1040A0008A4B09F0DFF832003B000AF001F8884A39
:1040B000884B09F0D7F832003B0009F0F9FF864A37
:1040C000864B09F0CFF832003B0009F0F1FF844A3B
:1040D000844B09F0C7F832003B0009F0E9FF824A3F
:1040E000824B09F0BFF8049A059B09F0E1FF804A72
:1040F0000C900D917F4B3000390009F0D9FF7E4ABA
:104100007E4B09F0AFF832003B0009F0D1FF7C4A4A
:104110007C4B09F0A7F832003B0009F0C9FF7A4A4E
:104120007A4B09F09FF832003B0009F0C1FF784A52
:10413000784B09F097F832003B0009F0B9FF764A56
:10414000764B09F08FF802000B000C980D9909F0DE
:1041500089F8089A099B09F0ABFF029A009B09F0C5
:1041600081F8049A059B09F0A3FF029A009B09F0CD
:1041700079F806000F0008980999694A694B09F017
:1041800097FF32003B0009F06DF8029003910200A6
:104190000B002800210009F065F8444B069A060040
:1041A0000F009A423DDD14980AF072FD3200009033
:1041B00001913B003000390009F07AFF009A019B21
:1041C000049005913000390009F04CF802000B0012
:1041D0000498059909F062FB029A039B0AF0DAF948
:1041E00002000B00280021000AF0D4F902000B00A5
:1041F00009F038F802000B00009801990AF0CAF99A
:104200000B9B0400981702231840013B181A0D005D
:104210000AF03EFD02000B002000290009F048FFD3
:10422000B4E6149B012B37D000230096019700932E
:10423000009A019B0492059302000B0000201A498A
:1042400009F02CFB2A000690079104980599069E18
:10425000079F23000AF09EF9009E02000B000298BF
:1042600003990AF097F932003B0009F021FF320070
:1042700004000D00049805993B0009F019FF002285
:10428000084B08F0EFFF02000B002000290008F0A7
:10429000E9FF069A079BBAE605000C0078E6C046DF
:1042A000FFFF2F3E0000F03F0000F0BF2794E53FE6
:1042B000182D4454FB21E93F075C143326A6813CAA
:1042C000D47ABF74702AFB3EE9A7F0320FB8123FD0
:1042D00068108D1AF726303F1583E0FEC8DB573F84
:1042E00093846EE9E326823FFE41B31BBAA1AB3F44
:1042F000735360DBCB75F3BEA69237A0887E143F64
:104300000165F2F2D844433F280356C9226D6D3F40
:1043100037D60684F464963F7AFE10111111C13F1E
:10432000635555555555D53FF0B54B008FB05B08DB
:1043300000931700DA4B009A040007919A4209DCB7
:1043400002000B003A607B6000220023BA60FB6031
:10435000002624E0D34B009A9A4200DD6DE0D24A59
:10436000002935DDD14B0AF015F9009B04001A0035
:10437000CE4B0D009A4215D0CD4ACE4B0AF00AF929
:1043800002000B0020003A607B6029000AF002F96D
:10439000C74AC84B0AF0FEF80126B860F960300041
:1043A0000FB0F0BDD322C34B52050AF0F3F8C24A56
:1043B000C24B04000D000AF0EDF802000B002000D3
:1043C0003A607B6029000AF0E5F8BB4ABB4BE1E7A5
:1043D000B64B08F047FF009B04001A00B34B0D00DA
:1043E0009A4214D0B24AB34B08F03CFF02000B00D3
:1043F00020003A607B6029000AF0CCF8AC4AAD4B53
:1044000008F030FF0126B860F9607642C7E7D32292
:10441000A84B520508F026FFA74AA84B04000D0040
:1044200008F020FF02000B0020003A607B602900AA
:104430000AF0B0F8A04AA14BE2E7A14B009A9A42D9
:1044400000DDD0E0FEF7D2F89E4A9F4B04000D003D
:1044500009F02EFE00229D4B08F004FF0AF0E2FB5B
:1044600006000AF015FC904A904B0490059109F063
:104470001FFE02000B00200029000AF08BF88C4A76
:1044800002900391049805998A4B09F011FE0400EB
:104490000D0002000B00029803990AF07BF81F2E12
:1044A00028DC8B4A731E9B009B58009A934221D0B4
:1044B00002000B003A607B60029803997B683A68BF
:1044C0000093009B0AF066F822002B000AF062F8C5
:1044D0000B000200BA60FB60079B002B00DB5EE76D
:1044E000802212069446009B891863447B60B86062
:1044F000F9608AE7009B1B150693069A4B005B0D3B
:10450000D31A102BD4DD04980599D322694B520598
:1045100009F0CEFD04000D0002000B000298039983
:104520000AF038F802000B000090019102980399FC
:104530000AF030F822002B000AF02CF804000D00DD
:10454000049805995C4A5D4B09F0B2FD22002B00EE
:104550000AF020F802000B0004000D0000980199F9
:104560000AF018F8069A4B005B0DD31A312B08DCC1
:1045700002000B003A607B60009A019B0292039359
:104580009AE7B8220498059992054C4B09F090FDE2
:1045900004000D0002000B000098019909F0FAFFD9
:1045A00002000B00029003910098019909F0F2FFBC
:1045B00022002B0009F0EEFF04000D00049805997D
:1045C000444A454B09F074FD22002B0009F0E2FF3C
:1045D00002000B0004000D000298039909F0DAFFB5
:1045E0003860796068E73D4B009A9A4208DD020026
:1045F0000B0009F0CFFFB860F96038607960A7E67A
:10460000009B374A1B159B18009A02931B05D51A6D
:1046100029000AF007FB0AF03BFB02000B00200018
:1046200029000892099309F0B5FF00222D4B09F0EB
:104630003FFD04000D000AF0F5FA0AF029FB020024
:104640000B0008AEB260F3602000290009F0A2FF61
:104650000022244B09F02CFD032430617161651E9A
:10466000EB00F318186859680022002308F07EF860
:10467000002813D123003000029A3900FDF716FDFF
:10468000079B0600002B00DB89E680227B68120670
:104690009B187B60FB689B18FB60B6E62C00DEE78E
:1046A000FB21E93F7BD9024000004054FB21F93F48
:1046B0003163621A61B4D03D7370032E8A19A33B33
:1046C000FB21394183C8C96D305FE43F0000E03F02
:1046D00018F60000C14920259A837B39FFFFEF7F40
:1046E000EAFBFFFF0000704130B5204A4B0087B065
:1046F0005B08934206DC0023002200930023FDF7B1
:10470000E1F806E01A4A934205DD02000B0009F0C9
:1047100041FF07B030BD02AAFFF706FE049C059DCD
:1047200003230340012B0AD002980399022B0DD0DA
:10473000002B15D10133009322002B00DFE722006C
:10474000029803992B00FDF709FBE2E70123220001
:1047500000932B00FDF7B6F880231B06C918D8E795
:1047600022002B00FDF7FAFAF6E7C046FB21E93FED
:10477000FFFFEF7F30B51E4A4B0087B05B089342C6
:1047800004DC00220023FDF7E9FA06E0194A93420F
:1047900005DD02000B0009F0FDFE07B030BD02AAE6
:1047A000FFF7C2FD049C059D03230340012B08D0A5
:1047B00002980399022B0FD0002B12D122002B005C
:1047C000E1E700932200029803992B00FDF77AF8A5
:1047D00080231B06C918E0E722002B00FDF7BEFA74
:1047E000F6E70123220000932B00FDF76BF8D4E7D6
:1047F000FB21E93FFFFFEF7F82B0D0B586B0040018
:104800000C980D990A920B9304AA02ABFEF73EF89E
:104810000A980B99FFF7AEFF029A039B09F048FC38
:1048200006000F000A980B99FFF75EFF049A059B9C
:1048300009F03EFC00220090019100233000390075
:1048400009F036FC02000B000098019908F00AFDFF
:10485000206061602000A660E76006B0D0BC08BCA4
:1048600002B0184782B0D3B50692079304000698A9
:104870000799FCF70BFB06000F0008980999FFF752
:1048800033FF32003B0009F013FC009001910898BF
:104890000999FFF76FFF32003B0009F009FC002285
:1048A00006000F0000980199002309F001FC0200A6
:1048B0000B003000390008F0D5FC009A019B206005
:1048C0006160A260E3602000D6BC08BC02B018475B
:1048D00082B0F0B50026002797B01D931E9B1F9D48
:1048E0000E9304001C923B0032000E98290006959E
:1048F00007F03CFF002821D01C981D9932003B0096
:1049000007F044FF002819D01C981D99FDF74CFBB7
:104910001C9A1D9B07F02AFF00280FD032003B0095
:1049200000208B4908F0BAFFA660E7602060616054
:10493000200017B0F0BC08BC02B0184780231C98B8
:104940001D991B06EB180F930022824B07F014FFF2
:10495000002854D01C981D997F4A804B09F0A8FB71
:104960007D4A06000D007D4B0E98069909F0A0FBCC
:1049700032002B000191009012A8FFF73DFF149A1E
:10498000159B129E139F069207931C9A1D9B002055
:104990006F4909F0FFFD0B000F99020001910E997C
:1049A00012A80091FFF794FF149A159B12A8049285
:1049B0000593129A139B02920393069A079B009207
:1049C000019332003B0007F0FFFE149A159B0492FE
:1049D0000593129A139B029203930022002312A8BC
:1049E000009201935C4A5D4B08F062F9129A139BA6
:1049F00022606360149A159BA260E36098E700222E
:104A00001C981D99524B09F0C5FD002200230C9201
:104A10000D93012201254E4B089009910A920B93A8
:104A20004F4B50331093109AEB00D3181E685F68F9
:104A30000E9A069B2800049205930AF029F9089A19
:104A4000099B08F00FFC00220023029003910092C2
:104A5000019312A832003B0008F02AF9129A139B26
:104A60000A980B9908F0FEFB149A159B0A900B917B
:104A70000C980D9908F0F6FB01350C900D910B2D5B
:104A8000D1D1089809990022364B08F0EBFB00229F
:104A9000304B08F0E7FB0500109111912E48324988
:104AA000FCF726FD002206000F0008980999294B03
:104AB00008F0D8FB0E9A069B02900391049205938E
:104AC000069B2A0001930E9B12A80093119BFFF7EF
:104AD0008BF91298139932003B0009F0E9FA320081
:104AE00006900791149815993B0009F0E1FA80228D
:104AF000120694460F0006000F9A109B01920E9A20
:104B00006344009212A82A00FFF7ACFE149A159B8A
:104B100012A804920593129A139B00960197029291
:104B20000393069A079B07F04FFE0C9A0D9B12A861
:104B3000049205930A9A0B9B02920393149A159B75
:104B400000920193129A139B07F03EFE4EE7C04677
:104B50000000F03F0000E03F182D4454FB210940C5
:104B600070EE000000002240FB211940F7B506005E
:104B70000F0014001D00FCF7ADFC002805D120003B
:104B80002900FCF7A7FC00280BD0200029003200E8
:104B90003B0008F067FB04000D002000290003B073
:104BA000F0BD22002B003000390007F0DFFD0028A7
:104BB000F3D1002200233000390007F0D7FD002890
:104BC0000CD0200029000022002307F0D5FD01248D
:104BD00000250028E1D080252D06DEE701236A4666
:104BE0003000137039000022002307F0D9FD00289F
:104BF00001D16B4618706A460123127830005A4082
:104C000001926A463900137022002B0007F0B4FDB0
:104C1000002801D16B4618706B466A461B781279E2
:104C2000934204D001240025A4197D41B5E7012455
:104C30006442E517F8E7F7B5071E21DA124C134D69
:104C400047420022124B01260092019312E03742A4
:104C500007D00098019922002B0009F029FA009052
:104C6000019122002B002000290009F021FA040004
:104C70000D007F10002FEAD10098019903B0F0BD1C
:104C80000024044DDDE7C0469A9999999999B93F56
:104C90000000F03F00002440F8B50D0017001E0092
:104CA000040009F0BFFF386009F0F2FF02000B00BA
:104CB0002000290009F06EFC0022104B09F0F8F9E1
:104CC00004000D00FBF75AFE09F0ACFF306009F05C
:104CD000DFFF02000B002000290009F05BFC00222E
:104CE000074B09F0E5F9FBF749FE09F09BFF0028A7
:104CF00000D10130069B1860F8BDC04600408F40CF
:104D00000000594030B50A4B652804DD0322873383
:104D10001A70002030BD000118180930FF300268F9
:104D200043688468C5680A604B608C60CD60F0E7BA
:104D3000A808001070B505000C0000220023280010
:104D4000210007F019FD002807D0280080252D0636
:104D50006119FDF729F9491970BD28002100FDF7F7
:104D600023F9F9E7F7B514001D0000900191002226
:104D7000184B2000290007F0FFFC002801D0002478
:104D8000144D0026134F009A019B2000290007F0C4
:104D9000FDFC002803D13000390003B0F0BD300025
:104DA000390022002B0009F083F906000F00FCF700
:104DB00081FB0028EFD130003900FCF78BFB002885
:104DC000E9D1200029000022024B08F04BFA040030
:104DD0000D00D8E70000F03FF7B506000D003000E9
:104DE0002900FCF777FB071E51D130002900FCF7A2
:104DF00061FB041E4DD1002200233000290007F082
:104E0000B5FC002837D1002200233000290007F02C
:104E1000B3FC002803D080231B06ED18DFE7002237
:104E20001D4B3000290007F0C5FC002815D00022DA
:104E30001A4B009201930098019932002B0007F061
:104E4000AFFC002817D1009801990022134B09F0FC
:104E50002FF9013400900191EDE7114C114B0093B3
:104E6000019401240098019932002B0007F08EFC78
:104E7000002802D064422000FEBD00980199002263
:104E8000064B08F00BFD013400900191EAE7002485
:104E9000F1E73C00EFE7C0460000F03F000024408F
:104EA0009999B93F9A9999990A4B10B51A007E328F
:104EB0001278002A0BD17F331B780022002B07D0F9
:104EC000054B09F0F5F8054A054B08F0E7FC10BD65
:104ED000044BF6E7A808001000007940182D445450
:104EE000FB2119400080764010B50122802806D8A9
:104EF000044980004358002B01D09847002210003D
:104F000010BDC04614F40000020008210300012077
:104F1000473A8A43D2B210B5824220D91A000424FB
:104F20006F3AA243D2B2002A19D01A00763A0A2A5E
:104F300015D9402218009043020001202B2A0ED0E0
:104F40009A1F82420BD9073AA243D2B20400002A28
:104F500005D000208B43433BDBB29C42404110BD57
:104F6000F8B501240C4D0D4E2F5D002F06D12B19E5
:104F7000013B1878FFF7C8FF00280AD03800FFF778
:104F8000C3FF431E98410019441CB442ECDDFA24CF
:104F9000E4002000F8BDC046D4000010CF07000098
:104FA00070B504000D00FFF7DBFF154B1A1AAA427B
:104FB00004DA0322134B87331A7070BD9C42FCDC69
:104FC0002919FAD4002DF8D00ADD00210E4BED1876
:104FD000A042F2DBC21816782E5411700138F7E7A0
:104FE000FA2200230848D200121B091824189A42FA
:104FF000E3DDE05CC8540020E0540133F7E7C0462D
:10500000CF070000A8080010D400001070B57C265F
:105010000C4D0D4BAC5B185DFFF776FF002807D0F9
:105020000A4B9C420AD9872303220120EA5470BD0F
:10503000074B9C42F7D80134AC53F8E70234AC5329
:105040000020F4E7A8080010D4000010CD070000ED
:10505000CE070000F7B5114C019123007C331B886B
:105060000F4D0700EA5C002A01D1002B01D1FFF7A8
:10507000CDFF7C3420880121FFF792FF268838007D
:10508000AF55FFF741FF002807D0701C0121FFF743
:1050900087FF2388ED18019B6B70F7BDA8080010EF
:1050A000D4000010F8B506000400064F351B002C94
:1050B00005DD013C385DFFF727FF0028F6D1012010
:1050C0002840F8BDD400001070B50A4E04B223B2D7
:1050D000002B01DC084809E0A5192B782B2B06D101
:1050E0002000FFF7DFFF002801D1687870BD013C88
:1050F000EDE7C046D4000010FFFFFF7FF8B57C2528
:10510000084E745B671E3800FFF7CCFF002805D1FE
:10511000002C01D07753F8BD0120FCE7023C74530A
:105120000020F8E7A808001030B5FA240023084949
:10513000E400CD5C5A1C2B2D04D18D5C854201D13D
:10514000981C30BD1300A242F3D10020F9E7C046FD
:10515000D400001010B5682802D8FFF7E5FF10BD95
:105160000A4BFE280CD1E922D2009B181868596816
:1051700009F058FD03004042002BF0DBD8B2ECE709
:10518000032287331A700020E9E7C046A808001000
:1051900083280DD80F290BD88423CA085343181825
:1051A0000723194079330B41024A115C0B43135416
:1051B0007047C046B8100010F0B587B003923C4A63
:1051C0000493D3780C00834204D21378019301989E
:1051D00007B0F0BD002153689278801A1A7888428F
:1051E0001ADC991C5B78009101938B1805930C9B3A
:1051F000002B02D0019BE41A0134049BE5B2002786
:10520000002B1BD10025E4B20295019B029A934228
:10521000DDDD082600273DE002329B180131DDE785
:10522000039B2800F118C9B2FFF7B2FF0136204BEB
:105230005B789E42F4DB01350137EDB2019BBB4246
:10524000E0DD0026F3E7082E08D1059B009A934283
:10525000BDD01300002601331578009301231D42B1
:1052600015D0039BF918049BC9B2002B1CD0832CCA
:105270000DD80F290BD88422CB0853437D3A0A401E
:10528000802111410B481B19C25C8A43C2546D1026
:1052900001370136064B5B789F42D4DB029B013419
:1052A00001330293E4B2B0E72000FFF771FFEEE7AD
:1052B00000000010B810001070B50D0004000122AD
:1052C000FBF71EF8290001222000FAF7F5FF70BD58
:1052D0000122F8B5082107001000FAF7EDFF0724B6
:1052E0000826002231000120FAF7E6FF3A000125E6
:1052F000224102212A400020FAF7DEFF2A00310075
:105300002800FAF7D9FF013CEBD2F8BD002210B516
:10531000040011000220FAF7CFFF2000FFF7D8FFAA
:1053200010BDF7B5012300245026134D00930194BE
:1053300076426A46A300D05800273043C0B2FFF738
:10534000E5FF0020FFF7E2FF1020FFF7DFFFE0207E
:10535000FFF7DCFF012200210220FAF7ADFFE85D34
:105360000137FFF7B5FF842FF4D18435012C00D12C
:10537000F7BD0124DDE7C046B81000107047704744
:105380000122024B80331A707047C046A8080010F3
:10539000054B002219007C310A80190086310A7001
:1053A000A43301321A707047A808001010B5074CDA
:1053B000230085331B78002B03D00C217620FFF7C8
:1053C00049FE0123A434237010BDC046A808001074
:1053D000044B84331A787F2A02D8FF221A70704750
:1053E0000022FBE7A808001010B5064C7C34238887
:1053F000002B02D0FFF782FE10BDFFF7B1FD208029
:10540000FAE7C046A808001010B5074C2300853302
:105410001B78002B03D00B217620FFF71BFE012306
:10542000A434237010BDC046A80800108022024B8F
:1054300052007E331A807047A80800100122024BE8
:105440007E331A807047C046A80800100022024B25
:105450007E331A807047C046A808001070470022AB
:10546000014B80331A707047A80800100122024BCC
:10547000A4331A707047C046A80800100122024BDE
:10548000A4331A707047C046A80800100022054BCC
:1054900084339A56002A02DC01221A7070470022D7
:1054A000FBE7C046A8080010F0B585B00090019158
:1054B0001000190014001D00FDF798F80B9B060062
:1054C0001A685B680F001000190002920393FDF741
:1054D0008DF802000B003000390007F04DF900286C
:1054E00007D00099019A0A9B19605A600B9B1C60B7
:1054F0005D6005B0F0BD054B00211A0081321170CE
:1055000082331A7851424A411A707047A808001035
:10551000054B00211A008232117081331A785142F2
:105520004A411A707047C046A808001070B5114C67
:10553000114923007C331A88885C002803D1002A93
:1055400001D0188070BD230085331B78002B02D05A
:10555000FFF75CFDF6E72500012386352B70FFF78A
:10556000C3FC2B78002B01D0FFF750FD00238634BD
:105570002370E7E7A8080010D4000010F0B585B04C
:105580000500019114008A4206DD0022002302601A
:105590004360002005B0F0BD1000FFF74CFB060093
:1055A0000F002868696807F047FE029003913000F9
:1055B000390007F023FE07F03FFE0B0002000298BF
:1055C000039908F06BF9FBF7D9F907F017FE019B77
:1055D00003C59C4203D10843411E8841DAE707F026
:1055E0002BFEFFF7F9FB019BC1171C1BE30FA04229
:1055F00059410800CEE773B51D00114B14001E0081
:105600001A00B836C83200900191106851683060B5
:1056100071609068D168B060F1601E00A833D83620
:10562000306871689C60DD6010605160B068F1683E
:105630009060D1600099019A19605A6073BDC046AC
:10564000A808001073B514000C4A009001911600D0
:105650001D000B4B983618685968103B1862596248
:105660009869D9699862D962B342F4D100980199D6
:10567000A8329460D5601060516073BDA808001016
:1056800070090010F8B51F00074B0400A4331B7805
:105690000D001600002B05D02000290032003B0031
:1056A000FFF7D0FFF8BDC046A8080010D0B5154CD4
:1056B000154A23000833DB6F13400CD1134AA5347D
:1056C000516E002902DD21705366D0BD23785366E8
:1056D00004232370F9E7230086331B78002BF4D0D2
:1056E0000A4B58690A4BE358A434C01A09F00AFB64
:1056F0000022084B08F0D2F800230022FFF7C2FF77
:105700000123E6E7A808001000FFFF0018000010C2
:105710007C07000000408F4010B50C4C0023210096
:10572000A83100228868C96807F020F8030001202A
:10573000002B09D0B8340023A068E168002207F0EC
:1057400015F843425841400010BDC046A80800105B
:1057500070B5FFF7E1FF03000020012B16D00C4BC2
:105760000022A8331C685D680A4B2000290007F05E
:105770000DF800280AD0084B00222000290007F06D
:1057800019F8431E984143420120184070BDC0469D
:10579000A80800100000F03F0000F0BFF8B55F4D12
:1057A0002B0087331B78082B07D1FBF779F80028EB
:1057B000FBD12B00072287331A70FBF771F8584F83
:1057C0000400031EBE6E3FD1032E2DD12B00853366
:1057D0001B78002B05D12B007A331B78002B00D1CE
:1057E00034002B0081331A78002A03D0052E01D013
:1057F00000221A702B0082331A78002A03D0092E57
:1058000001D000221A702B00002284339A56002AFD
:1058100005D02F2E0FD0572E0DD000221A703A2E01
:1058200009D1FFF743FF06E0532E02D12B00853349
:10583000D3E7002ED5D12A0000237A3279351370B0
:10584000BB662B70FB663DE02A0081321278002A8D
:1058500021D02834FB22053B134204D1200028210B
:1058600006F066FF0C00B44242D1032C2CD12B0071
:1058700085331B78002B15D00025FB6E022B32DD03
:10588000642D1FDC0120FAF7DFFCFBF709F8002884
:1058900010D00135F1E72A0082321278002AD9D0DF
:1058A0005034D7E71F4C0120FAF7CEFCFAF7F8FF87
:1058B000002801D1002405E0013C002CF3D1012394
:1058C0007A352B702000F8BD532CD5D0164D012011
:1058D000FAF7BAFCFAF7E4FF0028EBD0013D002DFF
:1058E000F5D1A034EEE7114A9542CBD10133A9E7B7
:1058F0002B000833DA6F0E4BBC661A42E2D1032C40
:1059000001D0532CDED1C820FAF79EFCFAF7C8FF6D
:105910000028CFD0012379352B70CBE7A8080010E1
:1059200018000010D1070000E90300005902000030
:1059300000FFFF00F8B51D4B1A6E002A35D1013269
:105940001A66FFF72BFF0028FBD172B68026802154
:1059500080208027164D174A2B68760013402B6055
:10596000154BC9004001DF67DE67D967D867FAF7D2
:10597000B9FD124A0F49136880200B401360AC2315
:105980000F4A5B0113608021C0220E4C5200C900F7
:105990004001A750A650A150A0502A6813432B6085
:1059A000276026602160206062B6F8BD18000010F4
:1059B000048204407FEAFFFF04E100E0008204402B
:1059C0000882044000E100E0F0B585B002900C00D0
:1059D00003921F0006F08AFB451E002D01DB002C00
:1059E00001DC05B0F0BD029B2100585D0123039A44
:1059F00000933B00FFF7E0FB241A002F02D1013C8B
:105A0000013DEAE70026B542F9D0064B5B789E429D
:105A1000F5DA039BE0B29919C9B2FFF7B9FB013679
:105A2000F3E7C04600000010F0B5264D85B02C000D
:105A30007034200006F05AFB0023C2B2A275E37551
:105A400023766376A376E3769A4201D001332376F8
:105A500070352B782D2B01D12C3BAB760022C3B2B5
:105A60000393160015001400110001230292019205
:105A70000398884212DC002D02D0124B7033DC7583
:105A8000002E03D00F4B019970335976002A03D0B2
:105A90000C4B029A7033DA7605B0F0BD09487030CD
:105AA0000F5C01312E2F07D0452FE1D1085CCCB21D
:105AB00001942D2803D01E001D001C00D8E71A00F9
:105AC0000293F8E7180000107FB51C4C0600230075
:105AD00070331B7E002B1DD1194D2B009C331B787E
:105AE000002B17D1174BA835196C5A6C00910192F5
:105AF0009A6CDB6C0098019902920393029A039BC3
:105B0000FFF7C0FD009A019B2A606B60029A039B1D
:105B1000AA60EB600A4970347831A07DE27D097893
:105B2000821A8A4204DB637E002B01D1452E02D10A
:105B3000024B70331E54FFF777FF7FBD1800001033
:105B4000A808001070EE000010B50B4C2300703355
:105B50001B7E002B06D13120FFF7B6FF0122074B39
:105B6000A4331A707034637E002B04D14520FFF7F4
:105B7000ABFFA37D637610BD18000010A8080010CD
:105B800010B5074B7033DA7D002A08D11B78002B43
:105B900002D13020FFF798FF2E20FFF795FF10BDB0
:105BA0001800001010B53920FFF78EFF10BD10B59A
:105BB0003820FFF789FF10BD10B53720FFF784FFAD
:105BC00010BD10B53620FFF77FFF10BD10B5352092
:105BD000FFF77AFF10BD10B53420FFF775FF10BD39
:105BE00010B53320FFF770FF10BD10B53220FFF75E
:105BF0006BFF10BD10B53120FFF766FF10BD10B56B
:105C00003020FFF761FF10BDF0B50123050085B01E
:105C10002800029306F06AFA2B7803902D2B09D006
:105C200000240194039B9C4208DB0298019B58438B
:105C300005B0F0BD029B01355B42E9E7039B581EAE
:105C4000001BFEF7F8FF06000F00285D0134303816
:105C500009F01EF832003B0008F02AFA060001980D
:105C60000F0009F015F802000B003000390007F0B2
:105C7000F9FA08F0D7FF0190D4E7F0B587B00190AA
:105C800006F034FA019B03901B782D2B26D1019846
:105C90000130FFF7F2FF80231B06C91807B0F0BDE3
:105CA000019AD25C2E2A17D0452A00D102930133E3
:105CB000039A9342F4DB8C4206D1029BA34212D199
:105CC000019806F013FA0400002500260027039B24
:105CD0009D420ADB002011E01C00E8E7214C002374
:105CE00002942100E4E7029CEEE7029BAB420CD158
:105CF0001800019B01301818FFF786FFFEF79BFF85
:105D000032003B0008F0D4F9C8E7AC4214DD0022B1
:105D1000154B3000390008F0CBF906000F00019B4D
:105D2000585D303808F0B4FF32003B0007F09AFAB3
:105D300006000F000135CAE7AC42FBDA601BFEF734
:105D40007AFF019B04900591585D303808F0A0FF60
:105D5000049A059B08F0ACF902000B0030003900F2
:105D6000E4E7C046E703000000002440F0B5060069
:105D700085B00F0006F0BAF9350000240390039AAD
:105D8000AB1B9A4201DD832C01DD05B0F0BD002381
:105D90002878210000933A00FFF70EFA2418013406
:105DA0000135ECE7802273B5002107252B4B2C4CE5
:105DB000920301912000DA67902206F05FF9019BBF
:105DC000284EA360284B1A68AA431A60012219685A
:105DD00011431960254B1968A943196019681143CB
:105DE0001960802322495B01086803430B60214B43
:105DF0001A6082323260204A126819681F4B186894
:105E0000504306F0B7F9E121090306F0B3F9102277
:105E10001B4B1C491A60030A0B6003231A4AC0B2C9
:105E200010603360194B1D60194B5935186801908B
:105E3000080011001A682A40602AFBD15F3A1D68E9
:105E4000154207D122708022124B92031A6005235B
:105E5000036073BD0D680195F1E7C04604E100E001
:105E6000281000100C800040A4400440A8400440CA
:105E7000808004409880044078800440180000101E
:105E800028800040048000400080004008800040DE
:105E90001480004000E100E0FA2110B50C4C8900AC
:105EA000206806F05FFB0B4B984209D800230A4A92
:105EB000013863611060094A13600722084B1A60B9
:105EC000FFF770FFFAF7FCF8FAF7B2FA10BDC04618
:105ED00018000010FFFFFF0014E000E018E000E0F1
:105EE00010E000E010B5002839D080211D4A136869
:105EF0008B43136001231C490A681A42FCD0032219
:105F00001A4B1A6001230021194A136011601360B3
:105F100011681942FCD0174A1749136080230C6896
:105F20005B0223430B601100002804D180230D4A3B
:105F3000146823431360114B9A6882420ED0986014
:105F4000431E98410E4B404218400E4B0968C01842
:105F500006F010F90C4B1860FFF79EFF10BD034BC5
:105F60001860CFE7388204400C8004407080044001
:105F70007480044078800440808004400000001059
:105F800000512502001BB7001800001010B504488E
:105F900016220021703006F071F8FFF745FD10BDA4
:105FA0001800001070B5FFF7F1FF084B08491A0000
:105FB0000C6C4D6C886CC96CA83214605560906094
:105FC000D1600022A4331A7070BDC046A80800102A
:105FD00070EE000070B50E4C23009C331B78002B34
:105FE00014D10C4D7035280006F080F800280DD033
:105FF0002800FFF742FE2300A833186059600022F2
:106000000023B03422606360FFF7C0FF70BDC0465C
:10601000A808001018000010F0B589B0FFF7DAFFEB
:10602000464B5C681B680093019400980199434BB0
:10603000DC689B6802930394029A039BFFF722FBA0
:106040003F4B1C6C5D6C9E6CDF6C200029003200A5
:106050003B00FFF7F7FA3B4B2933FF331C685D68C1
:10606000384B20003933FF331A685B680092019384
:10607000344B29004933FF331A685B680492059357
:10608000304B00225933FF331E685F682E4B08F0F7
:1060900081FA22002B0008F00BF82A4B02900391A2
:1060A0006933FF331A685B682000290008F000F8A4
:1060B0003200069007913B003000390007F0F8FFEE
:1060C00002000B000698079908F064FA029A039BF5
:1060D00007F0E4FBFBF70CFA00260027194BB83356
:1060E00018605960174B2000C0331E605F60049A2F
:1060F000059B290007F0DCFF009A019B04000D00BE
:106100001000190007F0D4FF02000B002000290046
:1061100008F040FA029A039B07F0C0FBFBF7E8F98E
:106120000122064B18605960064BB0331E605F6059
:10613000044BA4331A7009B0F0BDC04650090010DA
:1061400070EE0000A80800100000F03FF7B5FFF760
:1061500041FF204C2500A83528686968AA68EB68CB
:10616000FFF790FA1C4B1E6C5F6C9A6CDB6C009214
:106170000193009A019B30003900FFF763FA230076
:10618000210029335931FF33FF311A685B6826003B
:10619000086849680092019307F080FBB8363060C8
:1061A000716021002300002600273931C033FF3100
:1061B0001E605F6008684968009A019B07F06EFBEB
:1061C0002300B0331E605F600123A434286069603F
:1061D0002370F7BDA808001070EE000070B5FFF73F
:1061E000F9FE0B4C2500A835AA68EB682868696899
:1061F000FFF748FA2300E83319685A6829606A6093
:106200009A68DB68AA60EB600123A434237070BD38
:10621000A8080010F8B5FFF7DDFE084BD8331E685C
:106220005F689C68DD6830002B0039002200FFF7B2
:1062300029FA0123014CA4342370F8BDA8080010EA
:1062400070B5FFF7C7FE0B4C2500A835AA68EB68B0
:1062500028686968FFF716FA074BA434996ADA6A66
:1062600029606A601A6B5B6BAA60EB600123237084
:1062700070BDC046A8080010F0EE0000F0B587B071
:10628000FFF7A8FE484B1C685D68484B20001E685D
:106290005F68474B29007933FF331A685B6807F062
:1062A00007FF444B009001911A685B683000390089
:1062B00007F0FEFE02000B000098019908F06AF951
:1062C0003B4B029003914933FF331A685B6820000F
:1062D000290007F0EDFE320004000D003B00300005
:1062E000390007F0E5FE02000B002000290008F04D
:1062F00051F92F4E00900191A83630687168B2684C
:10630000F368FFF7BFF92C4B1C6C5D6C9A6CDB6C6F
:1063100004920593049A059B20002900FFF792F947
:10632000009A019B0298039907F0B8FA204C0022CA
:10633000B8342060616000211D4BC03319605A6081
:10634000009801991B4B1A685B6807F0B1FE174B68
:1063500004001A685B680D000298039907F0A8FE14
:1063600002000B002000290008F014F90E4B040075
:106370001A685B680D000098019907F099FE020009
:106380000B002000290007F089FA002230607160BC
:106390000021074BB03319605A600122044BA4332B
:1063A0001A7007B0F0BDC046D0090010E009001017
:1063B000A8080010000A001070EE0000F8B5FFF702
:1063C00009FE0D4C00222500A8352E686F680023B9
:1063D0003000390007F06CFE02000B00A868E96885
:1063E00006F040FF2300B0331E605F600123A43439
:1063F000286069602370F8BDA808001073B5FFF726
:10640000E9FD124B1E00A836B168F26800910192B6
:1064100034687568009801991A00F8321460556064
:106420009060D1601A00B8321068516814605560ED
:10643000306071609068D168B060F1600098019937
:106440009060D1600122A4331A7073BDA8080010B7
:10645000F7B5FFF7BFFD144C25002300F835A8332E
:1064600019685A6829606A609A68DB68AA60EB60FC
:106470002300B8331E685F689A68DB680092019356
:10648000009A019B39003000FFF7B5F829686A6867
:106490002300D83319605A60A968EA689960DA6005
:1064A0000123A4342370F7BDA8080010D0B52A4CEE
:1064B0008CB0220083321378002B07D0012B03D13C
:1064C0000B3313700CB0D0BD013BFAE7FFF782FD30
:1064D0002300A83319685A68069107929E68DF68FE
:1064E000069807990022002306F040F900280BD0F7
:1064F000002200233000390006F038F9002803D0CC
:10650000873401232370DDE723000699079AE833D7
:1065100019605A602300F0331E605F6013000A00A8
:1065200002920393002200230496059700920193A0
:1065300008A80022094B06F0BBFB0899099A230022
:10654000A83319605A600A990B9A2300B033196076
:106550005A60A434D5E7C046A80800100000F03FF8
:1065600010B5FFF737FD064B1A00A833E83218685C
:106570005968106051609868D9689060D16010BD0A
:10658000A8080010F7B5FFF7C7F8284E002803D079
:10659000022387363370F7BDFFF7E2FF3300A836DA
:1065A000B833776836681C685D6832003B002000AD
:1065B000290007F0EFFF0090019102000B0030006E
:1065C000390006F0E3F80022194B00282AD0009881
:1065D000019906F047FE02000B0020002900FEF79B
:1065E000C1FB009A019B04000D003000390006F049
:1065F000CDF8002801D1009E019F00220C4B3000F5
:106600003900FEF7AFFB02000B002000290007F065
:1066100045F900220023FEF7EEFF0122034BA433CD
:106620001A70B8E730003900D3E7C046A808001058
:106630000000F03FF0B589B0FFF76EF8394C0590D7
:10664000002804D002238734237009B0F0BD26004F
:106650002936FF36FFF784FF306871680022324B1D
:1066600007F098FF069007910B00210025002700F6
:1066700002003931F835A837FF312A636B630868A7
:1066800049683A687B680092019307F083FF009A9B
:10669000019B286469641000190007F009FD0B00D4
:1066A000224902000868496807F074FF2865696597
:1066B000210023005931B833FF311A685B6808683C
:1066C00049680292039307F065FF029A039B2866CC
:1066D00069661000190007F0EBFC0B00144902007A
:1066E0000868496807F056FF029A039B28676967A4
:1066F00000980199250007F0DBFC7935FF35020091
:106700000B002868696807F045FF069A079B286018
:1067100069603A607B60B268F368A434BA60FB6079
:10672000059B91E7A80800100000F03FF009001059
:10673000100A0010F7B5FFF713FF134C2500A8351A
:10674000A868E968FEF7F6FA2E686F680090019174
:1067500030003900FEF7EEFA06000F0000980199AC
:106760000022002307F0A4FC32003B0006F07AFD73
:106770002300B033286069600099019A19605A605B
:106780000123A4342370F7BDA808001070B5FEF7EC
:10679000C3FF104C012803D102238734237070BD3E
:1067A0002500A835FFF7DCFE2868696800220A4B3F
:1067B00007F07EFC094B0A4A07F070F823002860B6
:1067C000696000200021B03318605960A4340123AF
:1067D000E4E7C046A808001000807640FB2119407D
:1067E000182D4454F0B587B0FEF796FF334C0128BE
:1067F00004D102238734237007B0F0BD2500A835EB
:10680000FFF7AEFE2E686F6830003900FEF792FA8F
:106810000090019102000B003000390007F0BAFE31
:106820000022274B07F044FC0022264B07F040FCD7
:10683000FAF7A4F80022234B07F030F82300029067
:10684000039100200021B033186059600298039929
:1068500008F0E8F908F01CFA1B4A1C4B06000F0070
:1068600007F026FCFAF78AF83200049005910298A6
:1068700003993B0007F08EFE0022114B07F018FC35
:10688000134A144B07F014FCFAF778F802000B00D7
:106890000498059906F0E6FC00220F4B06F0FEFF77
:1068A00000220E4B06F0FAFF009A019B06F0DAFC7C
:1068B000A4342860696001239DE7C046A808001041
:1068C0000000594084D797415555555543DEA341A3
:1068D000E4388EE35831454180842E410088C3401E
:1068E00010B5084C230086331B78002B04D1853467
:1068F0002278002A01D0237010BDFFF731FE01235A
:10690000F9E7C046A8080010F0B587B0FFF728FEE9
:10691000144D02A82C00A834E3680193A3680093E7
:1069200022686368FDF790F8029E039F2660676007
:10693000049A059BA260E360FEF7EEFE01280BD0EF
:1069400030003900FEF7B0FA2B00206061600020B3
:106950000021B033186059600123A4352B7007B0B3
:10696000F0BDC046A8080010F0B58BB0FFF7F8FDE9
:10697000FEF7EEFE204E07003500A835A968E8684E
:106980002A686B680190009106A8FDF789F9089BB9
:10699000099C1A4802930394069A079B184907F02A
:1069A000F9FD00220490059102980399002307F055
:1069B0007FFB02000B000498059907F0EBFD340003
:1069C00028606960B034002F0CD1029A039B00202C
:1069D000002107F0DFFD206061600123A4363370E1
:1069E0000BB0F0BD0022002322606360FEF75CFA6A
:1069F00028606960F1E7C046A8080010182D4454CB
:106A0000FB21F93F70B586B0FFF7AAFDFEF7A0FEA7
:106A1000124E05003400A834E36802A80193A3686D
:106A2000009322686368FDF73BF9029803992060A0
:106A30006160049A059BA260E360002D09D03500D7
:106A400000220023B0352A606B60FEF72DFA20602B
:106A500061600123A436337006B070BDA808001031
:106A600070B5FFF77DFD0A4C2500A835AA68EB68D4
:106A700028686968FAF7F0FD230028606960002043
:106A80000021B033186059600123A434237070BD15
:106A9000A8080010F8B5FEF73FFE144C002803D0FC
:106AA000022387342370F8BDFFF75AFD2500230029
:106AB000A835B8331E685F682868696832003B00F3
:106AC00007F068FD00220A4B07F0F2FA3B003200A3
:106AD00006F0E4FE23002860696000200021B03346
:106AE00018605960A4340123DCE7C046A8080010F0
:106AF0000000594070B5FEF70FFE114C002803D07E
:106B000002238734237070BDFFF72AFD2500210082
:106B1000A835B8312A686B680868496807F0C8FA70
:106B2000084B002206F0BAFE2300286069600020AE
:106B30000021B03318605960A4340123E2E7C04655
:106B4000A808001000005940F0B58DB0FFF708FD0F
:106B50001D4C2500A835A968E8682A686B68019073
:106B6000009108A8FDF774F80A9A0B9B089E099FEC
:106B7000164906920793086C8A6BCB6B496C0090A0
:106B8000019108A8FDF764F80A9A0B9B08A80492E3
:106B90000593089A099B02920393069A079B009219
:106BA000019332003B0006F083F8089A099B2A60A3
:106BB0006B600A990B9A2300B03319605A60012365
:106BC000A43423700DB0F0BDA8080010F0EE000052
:106BD00030B587B0FFF7C4FC0C4D02A82C00A834D8
:106BE000E368A4350193A368009322686368FDF706
:106BF0002FF8029A039B22606360049A059BA260AF
:106C0000E36001232B7007B030BDC046A808001018
:106C100030B58BB0FFF7A4FC104C2500A835AA684E
:106C2000EB680492059328686968009201930290CA
:106C3000039106A82A686B6805F0C6FD069A079BB3
:106C40002A606B600899099A2300B03319605A6072
:106C50000123A43423700BB030BDC046A808001037
:106C6000D0B5FEF759FD134C002803D0022387341A
:106C70002370D0BDFFF774FC2300B8331E685F6833
:106C80002300A8331A685B683000390007F082FCE3
:106C90000022094B06F0E6FA02000B003000390032
:106CA000FEF760F800230022FEF7A5FCA4340123C0
:106CB000DEE7C046A80800100000F03FF0B591B034
:106CC000FFF74EFC644E33002933FF335C681B68CA
:106CD000009301940098019933003933FF335C68C5
:106CE0001B680293039433005933FF335C681B68BD
:106CF0000493059433007933FF331A685B6807F017
:106D0000D7F9049A059B04000D000298039907F037
:106D1000CFF902000B002000290007F03BFC3300F4
:106D20004933FF330A900B911A685B680098019908
:106D300007F0BEF9029A039B04000D001000190031
:106D400007F0B6F902000B002000290007F022FC32
:106D500033006933FF33069007911A685B68009827
:106D6000019907F0A5F9049A059B04000D00100095
:106D7000190007F09DF9370002000B0020002900E0
:106D800007F008FCA8373B687C6808930994BA6848
:106D9000FB680C900D9108980999FEF773FC2F4B36
:106DA0001C6C5D6C9A6CDB6C0E920F930E9A0F9BB1
:106DB00020002900FEF746FC0C9A0D9B06980799C7
:106DC00007F076F9FAF794FB340002000B000A98FA
:106DD0000B9906F063FDB834330020606160002237
:106DE0000021C03319605A60089A099B00980199E4
:106DF00007F05EF9029A039B07F0CCFB0A9A0B9B03
:106E000007F056F9069A079B04000D0004980599AF
:106E100007F04EF902000B002000290006F022FACC
:106E2000069A079B04000D000098019907F040F9AD
:106E300002000B002000290006F030FD330038600E
:106E4000796000220021B03319605A6033000122BA
:106E5000A4331A7011B0F0BDA808001070EE000045
:106E6000F0B587B0FFF77CFBFEF756FC244C0128F9
:106E700019D02500A8352E686F680022214B3000FC
:106E8000390005F079FC00280DD13900300007F0F9
:106E9000C9FE07F0FDFE02000B003000390005F0CE
:106EA00065FC00281DD12500A835286869680022E6
:106EB000144B06F0D7F902000B00E868A9680190AE
:106EC000009102A8FDF704FD029A039B2A606B6003
:106ED000049A059BAA60EB600123A434237007B0D9
:106EE000F0BD084B002230003900FDF73BFF2300C6
:106EF0002860696000200021B03318605960EBE71A
:106F0000A80800100000F03FF0B587B0FFF728FB9D
:106F10001A4C2500A835AE68EF6830002A686B6807
:106F2000390002920393FDF705FF0090019102984A
:106F30000399FDF7FFFE0022049005910098019946
:106F4000002307F0B5F8049A059B06F08BF90200C0
:106F50000B000298039907F01DFB009A019B286023
:106F6000696025003000390007F014FB0123B035BB
:106F7000A43428606960237007B0F0BDA808001031
:106F8000F8B5FEF7C9FB194C012803D10223873459
:106F90002370F8BD2500A835FFF7E2FAA868E96874
:106FA0000022134B06F07AFC02000B0006F05AF99F
:106FB000104A114B07F07CF8002206000F002868E9
:106FC00069680B4B06F06AFC02000B0006F04AF9F8
:106FD000094B084A07F06CF82300B0331E605F606D
:106FE00028606960A4340123D2E7C046A8080010D5
:106FF00000807640182D4454FB210940F0B585B03F
:10700000FEF78AFB3D4C012804D10223873423700C
:1070100005B0F0BDA834FFF7A3FA65682468200026
:107020002900FDF787FE0090019102000B0020006F
:10703000290007F0AFFA0022314B07F039F80F00B2
:10704000060007F0EFFD040007F022FE02000B002F
:107050003000390007F09EFA0022294B07F028F88B
:107060000022284B07F024F8F9F788FC0022254B72
:1070700006F014FC0022224B06000F0005F09AFBDC
:10708000002808D03000390000221D4B07F082FA9A
:1070900006000F0001343B2C08DD00980199002206
:1070A000194B06F0DFF8009001913C3C64206043EE
:1070B00007F0EEFD00220290039100980199134B16
:1070C00006F0F6FF02000B000298039906F0CAF8DA
:1070D00032003B0006F0C6F80C4B002206F0DEFB47
:1070E000064D0B4B186059602B0000200021B03377
:1070F000186059600123A4352B7089E7A808001097
:1071000000004E4080842E410000F03F0088C340C4
:1071100050090010F7B5154C23009C331B78DB0693
:1071200003D52B22124BE254F7BD25002600B835BB
:10713000A836FFF715FA326873682868696806F0A0
:1071400091F8B268F36800900191A868E96806F0C8
:1071500089F806000F00009801993B003200FEF705
:107160004AFA0123A4342370DEE7C046A8080010C1
:1071700076070000F0B589B0FEF7CEFA394C0590DD
:10718000002804D002238734237009B0F0BD260004
:107190002936FF36FFF7E4F9306871680022324B78
:1071A00006F060F8069007910B00210025002700EB
:1071B00002003931F835A837FF312A636B6308685C
:1071C00049683A687B680092019306F04BF8009A90
:1071D000019B286469641000190006F069FF0B0028
:1071E000224902000868496806F03CF8286569658C
:1071F000210023005931B833FF311A685B680868F1
:1072000049680292039306F02DF8029A039B2866C0
:1072100069661000190006F04BFF0B0014490200CC
:107220000868496806F01EF8029A039B2867696798
:1072300000980199250006F03BFF7935FF350200E3
:107240000B002868696806F00DF8069A079B28600D
:1072500069603A607B60B268F368A434BA60FB602E
:10726000059B91E7A80800100000F03FF00900100E
:10727000100A0010F7B5154C23009C331B78DB0671
:1072800003D52D22124BE254F7BD25002600B83558
:10729000A836FFF765F9326873682868696807F0EF
:1072A00079F9B268F36800900191A868E96807F07D
:1072B00071F906000F00009801993B003200FEF7BB
:1072C0009AF90123A4342370DEE7C046A808001011
:1072D00076070000D0B5184C8AB023009C331B7889
:1072E000DB0604D52A22154BE2540AB0D0BDFFF7C5
:1072F00037F923002100B83318001E685F68A831F1
:107300008A68CB68049205930A684B6802920393DB
:107310008268C36806A80092019332003B0005F022
:1073200053FA089A099B06980799FEF764F9012316
:10733000A4342370D9E7C046A808001076070000DF
:10734000F0B5A1B0FFF70CF97B4D2B002C00843376
:107350001B78A8345BB20693012B4CD1226863687A
:10736000A668E7681000190005F07CFF08900991F5
:10737000FBF740F932003B000C900D9130003900D2
:1073800005F070FF0A900B91FDF7F4F902000B0075
:107390000C980D9905F066FF06000F000A980B99EE
:1073A000FDF7A2F932003B0006F078FA0A900B9143
:1073B00008980999FBF7B6F932003B0006F06EFA1F
:1073C000002206000F000A980B99002306F070FEB9
:1073D00002000B003000390005F044FF2B00B033F1
:1073E000206061600A990B9A19605A60069BA43567
:1073F0002B7021B0F0BD069B27686668013338D139
:1074000000224E4B18A804920593002200230292FA
:107410000393A268E368009201933A00330005F0F9
:10742000D3F91A99189A00911B99199B019118A8E0
:10743000FCF70AFB0022424B18A804920593802314
:1074400000221B06029203931A9A1B9B009201933F
:10745000189A199B05F0B8F9189A199B2260636075
:107460001A991B9A2B00B03319605A60A435012376
:10747000BEE7FEF751F901286ED02B007E331B7852
:10748000002B34D02F4A73005B08934208DC0123A1
:1074900000220093380000233100FCF753FD08E080
:1074A000294A934213DD3A0033003800310007F0D7
:1074B00071F82B00A83318605960B0350023002400
:1074C0002B606C6001221C4BA4331A7091E71CAA3C
:1074D00031003800FCF728FF1E9A1F9B0221400054
:1074E00008400139081A00901C981D99D5E72B0017
:1074F0007F331B78B0350022002B1BD0134B380094
:10750000310006F0CBF906000F00FAF71BFB320042
:10751000069007913B0000200D4907F03BF8FAF771
:1075200011FB02000B000698079906F0B7F92060DE
:107530006160C3E7074BE2E7A80800100000F03FD6
:107540000000F0BFFB21E93FFFFFEF7F0000694033
:107550000000E03F008066403A00E568A468330020
:107560003800310005F07EFE06900791FDF702F924
:10757000220006000F002B002000290005F072FEFB
:1075800008900991FBF736F802000B003000390033
:1075900005F068FE06000F00FBF728F800229C4B60
:1075A00005F0EAF8002800D1F7E006980799FBF704
:1075B0001DF80A900B9108980999FBF717F8954A5E
:1075C0000C900D910A980B99934B06F067F90022E5
:1075D000002304000D0005F0EDF800228F4B002879
:1075E00000D10BE12000290005F03CFE07F01AFB5A
:1075F00007F04EFBA822884BD20506000F0006F0CC
:1076000057FD02000B000A980B9906F0C3FF802279
:1076100004000D005205824B3000390006F048FD91
:1076200002000B002000290006F0B4FF7D4A040090
:107630000D007D4B3000390006F03AFD02000B00D2
:107640002000290006F0A6FF02000B0006F030FD26
:107650000C9A0D9B00260027109011911000190024
:1076600006F026FD002234003D00704B129013916D
:107670000E920F930C920D930A920B9300226B4B78
:107680002000290005F0EEFD0A9A0B9B04000D0076
:1076900006F00EFD00220A900B91644B2000290099
:1076A00005F0E0FD04000D0002000B000A980B99A4
:1076B00006F0FEFC0C9A0D9B0A900B911098119904
:1076C00006F0F6FC0E9A0F9B0C900D9112981399F0
:1076D00006F0EEFC02000B000E900F910C980D9935
:1076E00005F0C0FD0A9A0B9B06F0D8F832003B006B
:1076F00005F0B8FD0022169017914C4B2000290090
:1077000005F0B0FD04000D0002000B000A980B9973
:1077100006F0CEFC002206000F00444B200029009A
:1077200005F0A0FD02000B0004000D003000390040
:1077300006F0BEFC0C9A0D9B0A900B9110981199C3
:1077400006F0B6FC0E9A0F9B0C900D9112981399AF
:1077500006F0AEFC0C9A0D9B0E900F9106F01AFFEE
:107760000A9A0B9B06F09AF802000B0014901591F0
:107770001698179905F076FD02000B0006000F0021
:107780001498159906F08AF8FAF730FF284A294B21
:1077900005F006F8002800D070E700220023300032
:1077A000390004F0E3FF00282DD108980999FAF771
:1077B000B9FF32003B0006F071F804000D00069896
:1077C0000799FCF791FF32003B0006F067F80022B2
:1077D00006000F0000232000290006F069FC0200CB
:1077E0000B003000390005F03DFD134B1A00B0339B
:1077F000A832106051601C605D6063E620002900C3
:1078000006F0C8FEF2E600240C4D00200C49ECE71F
:107810000000D03F182D4454FB2109400000E03FF8
:10782000460B213E6EC0453163626A3C0000F03F6A
:107830004F64A14091B49F3CA80800100000F07F65
:107840000000F87FF0B5842597B0FEF789FE824BE3
:10785000814C5D57A834012D42D126686768A26823
:10786000E3683000390006920793FAF75BFF08904F
:10787000099106980799FCF737FF02000B0008985A
:10788000099906F015FC0890099130003900FAF7C3
:10789000B1FE06000F0006980799FCF76BFF020087
:1078A0000B003000390006F003FC002206000F0038
:1078B00008980999002306F0FBFB02000B0030003A
:1078C000390005F0CFFC644B206061600899099A8B
:1078D000B03319605A60604BA4331D7017B0F0BD0F
:1078E00022686368069207936B1C5AD10698079921
:1078F000E36800220893594B05F0B4FCA768089D83
:1079000002000B0001950EA80097FBF701F80E9AF4
:107910000F9B069807990A920B93109A119B0C9251
:107920000D9300224D4B06F035FE01950B00020031
:1079300000970EA8FAF7ECFF109A119B0EA804927C
:1079400005930E9A0F9B029203930C9A0D9B009243
:1079500001930A9A0B9B04F037FF069A079B0E9837
:107960000F9905F07FFC089B06000D0010981199F7
:107970003A0005F077FC32002B00019100900EA830
:10798000FCF766F90E9A0F9B226063601099119ABA
:10799000314BB03319605A6001222F4BA4331A7057
:1079A0009CE7FDF7B9FE2C4DB035012825D02A4BB8
:1079B00000267E331B780027002B08D006980799F5
:1079C000FCF7D8FE206061602E606F60E4E7224B18
:1079D00000227F331B78002B0DD0214B069807998E
:1079E00005F05CFF02000B0000201E4906F0D2FDEE
:1079F000FAF7A8F8E6E71C4BF0E714AB12AAA06868
:107A0000E168FAF743FF06980799FCF76DFE149AB0
:107A1000159B06F04DFB07000E000891069807998C
:107A2000FCF7A8FE129A139B06F042FB0022069078
:107A3000079100233800089906F03AFB0B0002007A
:107A40000698079906F0A6FD80231B06F61820600D
:107A500061602F606E609FE7A80800100000F03F93
:107A6000000069400000E03F00806640F0B591B042
:107A7000FEF776FD684D2B002C0084331B78A8346C
:107A80005BB20893012B42D126686768A268E3685D
:107A90003000390006920793FAF7ACFD0A900B917B
:107AA00006980799FCF720FE02000B000A980B9934
:107AB00006F0FEFA0A900B9130003900FAF732FE18
:107AC00006000F0006980799FCF754FE02000B0011
:107AD0003000390006F0ECFA002206000F000A9888
:107AE0000B99002306F0E4FA02000B003000390085
:107AF00005F0B8FB2B00B033206061600A990B9A47
:107B000019605A60089BA4352B7011B0F0BD6368F2
:107B100026680693089B013344D1A268E368089263
:107B20000993049205933200069B0CA802920393DA
:107B3000089A099B009201933200069B04F044FED0
:107B40000C980D990022354B05F08CFB0B000E991B
:107B5000020000910F990CA80191FAF7D9FE0C9838
:107B60000D993200069B05F07DFB089A099B0600E3
:107B70000F000E980F9905F075FB32003B00019144
:107B800000900CA8FCF764F80C9A0D9B22606360CF
:107B90000E990F9A2B00B03319605A600122A43558
:107BA0002A70B2E72F00FDF7B7FDB037012823D0C8
:107BB0002B007E331B78002B0ED030000699FCF78B
:107BC00093FD20606160002300243B607C602B00FB
:107BD0000122A4331A7098E72B007F331B78002210
:107BE000002B07D00E4B3000069905F057FEF9F731
:107BF000A9FFE6E70B4BF6E7E068A1683200069BB9
:107C0000019000910CA8FCF7F7FD0C9A0D9B2260E7
:107C100063600E9B0F9CD8E7A80800100000F03F9F
:107C20000000694000806640D0B5224C8CB0230033
:107C30009C331B78DB0604D52F221F4BE2540CB07B
:107C4000D0BDFEF78DFC2300A83319685A68069151
:107C500007929E68DF68069807990022002304F0C7
:107C600085FD00280BD0002200233000390004F0ED
:107C70007DFD002803D0873401232370DFE7230034
:107C8000B8331868596804960597069E079F0296B0
:107C900003979A68DB680092019302000B0008A822
:107CA00005F006F8089809990A9A0B9BFDF7A3FCC2
:107CB000A434E1E7A80800107607000070B58AB088
:107CC000FEF74EFC154C2100B83188680A684B68F5
:107CD0000090C96801912100A8310D684E68029595
:107CE00003968868C9680490059106A8FCF77CF89B
:107CF0000699079A2300F83319605A600899099A7F
:107D00009960DA60089A099B06980799FDF773FC59
:107D10000123A43423700AB070BDC046A808001027
:107D200070B58AB0FEF71CFC134C144925002600E0
:107D3000086C8A6BCB6B496CA83500900191286860
:107D4000696802900391F836A868E9680490059183
:107D500006A8FCF749F8069A079B0898099932602B
:107D600073602A606B600123A434B060F160A86086
:107D7000E96023700AB070BDA8080010F0EE0000A2
:107D800030B587B0FEF7ECFB0C4D02A82C00A834F0
:107D9000E368A4350193A368009322686368FCF745
:107DA00061FD029A039B22606360049A059BA260B6
:107DB000E36001232B7007B030BDC046A808001057
:107DC00030B587B0FEF7CCFB0C4D02A82C00A834D0
:107DD000E368A4350193A368009322686368FAF707
:107DE00097FD029A039B22606360049A059BA26040
:107DF000E36001232B7007B030BDC046A808001017
:107E0000842210B552000021014804F037F910BD5A
:107E1000B810001010B508210120FDF74DFA02211D
:107E20000020FDF749FA00210220FDF745FA06215E
:107E30000220FDF741FA03210800FDF73DFA032176
:107E400000220800F8F738FA002206210220F8F78D
:107E500033FA012206210220F8F72EFAFFF7D0FFAD
:107E6000FDF75FFAA220FDF751FAA020FDF74EFAC8
:107E7000C020FDF74BFAF820FDF748FA0020FDF787
:107E800045FA0A20F8F7E0F94020FDF73FFA2C20E8
:107E9000FDF73CFA3220F8F7D7F92E20FDF736FA35
:107EA0003220F8F7D1F92F20FDF730FA0A20F8F741
:107EB000CBF92520FDF72AFA0A20F8F7C5F9812029
:107EC000FDF724FA0020FDF721FAAF20FDF71EFA96
:107ED000A420FDF71BFA10BD70B50A20F8F7B4F91D
:107EE000FDF75CFC0128F8D01D4D2C0048342379A7
:107EF000002B19D0002323712372E3706379002BC8
:107F000007D1C122022152000E20F8F773FA012393
:107F100063710C22012148352B7908001A43AB7993
:107F20005B001A43F8F766FAAC20FDF7EFF9AE20D4
:107F3000FDF7ECF9A520FDF7E9F900200121F8F79C
:107F4000F1FA0020F8F772FC002802D10121F8F7BD
:107F5000E9FAFFF75FFFFFF753FFFDF7E2F970BDA6
:107F600018000010CC2270B5D20000210C4804F09B
:107F700085F8EB230B4CDB00E5181033E05806F0D6
:107F8000C1FE094A094B05F089FCEC23DB00E4182B
:107F900000220023286069602260636070BDC046D3
:107FA000B0090010A80800100000C0FFFFFFDF416B
:107FB0001B4B1C491A002932FF3270B50C6C4D6CFA
:107FC000886CC96C146055609060D1601A003932B9
:107FD000FF32146055609060D1601A004932FF3260
:107FE000146055609060D1601A005932FF321460FD
:107FF00055609060D1601A0079336932FF33FF32E7
:108000009860D960146055609060D1601C605D60BC
:10801000FDF7BCFF40220021034804F02FF870BD9B
:10802000A808001070EE00005009001070B50F4C49
:108030000F2223000E4E78331A70300005320021D3
:1080400004F01CF8230000259C330A4A1D700A4BDB
:108050000C320A493000E55404F005F8230083345B
:10806000A0331D602570FDF791FF70BDA8080010BA
:10807000300900100000001076070000C8F700006B
:10808000F7B56F4C260083363378002B16D02300CB
:1080900085331B78002B10D06A4D7035280004F012
:1080A00025F8012804D12800FDF7AEFD013030701D
:1080B000833421787620FCF7CDFFF7BD230086338B
:1080C0001B78002B00D1A2E0FDF784FF23007C3356
:1080D0001A885D4B9B185D78FDF71EFB01280BD1BC
:1080E0000C2D05D8594BEB409843C0B2002809D05D
:1080F000022387342370E0E7022803D12B00083BDA
:10810000032BF5D92300A8331E685F682300681E7F
:10811000B8331A685B68009201930B2819D804F0F1
:108120000BFB061B262D343B4E5D60636669210008
:10813000A83100228868C968002304F017FB0028D2
:1081400012D0002200233000390004F00FFB002879
:108150000AD0FCF75BFF07E0002200233000390063
:1081600004F01EFB0028F4D0A4340123C2E700224F
:1081700000233000390004F0FFFAF3E70022002367
:108180003000390004F016FBECE700220023300039
:10819000390004F0FBFAE5E721002300A831B833E9
:1081A0009A68DB688868C96804F0E0FA0028D0D0D3
:1081B000009A019B3000390004F0D8FAD2E7210080
:1081C0002300A831B8339A68DB688868C96804F06E
:1081D000CDFA0028C8D0009A019BB4E7009A019B11
:1081E000BCE7009A019BC4E7009A019BC8E7009A8C
:1081F000019BCCE72100A83100228868C9680023D0
:1082000004F0B4FA0028A4D000220023D2E723000F
:1082100085331B78002B00D14FE7FFF707FF2200C3
:1082200020219C321170220001230949A0321160E3
:108230007834084908483370237003F014FF3CE792
:10824000A808001018000010D4000010C210000090
:1082500081800000A0F7000030090010F7B5384C0D
:1082600023009C331D78002D56D03648364D030030
:1082700070331B78002B0FD12300A0331B68AB4257
:1082800002D0324A93421DD1314BE35C002B19D10D
:108290007030304903F0E7FE2300A0331A68AA4289
:1082A00022D12B4AA25C2B2A12D12B4A1A6023001E
:1082B000A0331B68873498472378002B29D0FDF71B
:1082C00065FE04E0230083331B78002BE4D1F7BD67
:1082D0002D2A01D1214AE9E72A2A01D1204AE5E7DE
:1082E0002F2AE4D11F4AE1E718498A42DFD1184A10
:1082F000A25C2B2A01D11C4AD8E72D2A01D11B4AA6
:10830000D4E72A2A01D11A4AD0E72F2ACFD1194A15
:10831000CCE7FFF78BFEDAE7FDF75CFE2300A8331E
:108320001E685F689A68DB6800920193009A019B5F
:1083300030003900A434FDF785F92570C7E7C04641
:10834000A808001018000010ED9600009D9700008E
:1083500076070000A6F70000F1980000459900009C
:1083600099990000FD990000619A0000A99A000007
:10837000F19A0000459B0000F0B56D4C91B02300D0
:108380009C331B785B070BD56A4B70331B7E002B2D
:1083900002D14920FDF798FBFFF760FF11B0F0BD57
:1083A000FDF718FEFDF7B8F9012835D12500A835ED
:1083B000AA68EB6806920793230080331B78B034D9
:1083C00000260027002B22D02A686B6808920993A8
:1083D00008980999069A079BF9F73EF9089A099BAC
:1083E0000A900B9106980799FBF77CFA0A9A0B9B67
:1083F000266067602A606B60FCF756FD32003B0028
:10840000FDF720F901224A4BA4331A70C6E7266013
:10841000676006980799F1E7022802D18734207037
:10842000BCE72200B832106851689568D66822000F
:108430002300089009910695079680321278A83398
:108440001868596800260027002A4CD023007E3384
:108450001B78002B0FD17F3423780022002B40D0D3
:10846000354B05F01BFA02000B0004F0FBFE334A0B
:10847000334B05F01DFE2E4B324C1A00B0331E60FC
:108480005F600023A83210605160049305940200DD
:108490000B000CA8029603970096019704F094F93C
:1084A0000E990C9A00910F990D9B01910CA8FCF765
:1084B000D9F90E9B0F9C0CA8049305940C9B0D9C62
:1084C00002930394069B079C00930194089A099BCE
:1084D00004F07AF90C980D990E9A0F9BFDF78BF822
:1084E00090E7194BBDE70024164D029603970494BC
:1084F00005950200DC689B680CA8009301940B00B2
:1085000004F062F9089A099B0C980D9904F0AAFEF0
:10851000069A079B04000D000E980F9904F0A2FE26
:1085200006000F002000290032003B00D6E7C046BD
:10853000A80800101800001000007940182D4454BD
:10854000FB2109400000F03F008076401FB5124C2F
:1085500023009C331B789B070AD510487030037E9C
:10856000002B02D10E4903F07EFDFFF777FE1FBD01
:10857000FDF7F6FF23008021A8339A6809060292CE
:10858000DA68A434521803920299039A9960DA6067
:1085900001232370EBE7C046A80800101800001064
:1085A000AAF70000F0B5384B89B004930023374E8A
:1085B0000D00745C02A903900B739A4204D015223B
:1085C000334904A803F04FFD2000FCF79DFC070091
:1085D0002800FCF767FD002F1ED000281ED12F00B9
:1085E0007619767806AD05220021280003F046FDB5
:1085F000FE2E17D12749280003F035FD762C2DD10A
:108600003A00254BB6009E19B36C2449009304AB85
:10861000039803F028FD2CE000282CD06F1EF45D99
:10862000765DDFE7FF2E01D11D49E4E71D49FD2EF0
:10863000E1D0632E0FD923004F3B012B04D92B2C03
:1086400002D0A31F012B06D832001149233A28007B
:1086500003F009FDD2E732001349F8E7134BA400F9
:10866000E358019500933A0004AB1149039803F0D5
:10867000FAFC09B0F0BD0D4BA400E3582A000093AA
:108680000C4904ABC4E7C04620200000D400001011
:1086900091F8000055F80000F0EE0000B7F7000078
:1086A000AAF70000AEF70000B4F7000010F20000D7
:1086B000C0F70000CBF7000010B509280BD9094B13
:1086C000FE2809D1E922D2009B181868596806F0E3
:1086D000A9FA03F0E7FE10BD032287331A700020C9
:1086E000F9E7C046A808001010B503000E280CD901
:1086F0000F20FE2B09D1E922044BD2009B181868E9
:10870000596806F08FFA03F0CDFE10BDA8080010DE
:1087100010B5682802D8FCF707FD10BD094BFE28EC
:108720000AD1E922D2009B181868596806F07AFA33
:1087300003F0B8FEC0B2EEE7032287331A700020C0
:10874000EBE7C046A808001010B5030063280CD959
:108750006420FE2B09D00130FD2B06D0094CFF2BE5
:1087600004D0032300208734237010BDE923DB00ED
:10877000E3181868596806F055FA03F093FE632869
:10878000EFDCF2E7A8080010F0B50D0085B004009A
:108790001700026843681000190000920193FCF76B
:1087A0001BFB534A28601300A5331B780600012BDE
:1087B00030D1A6321378BB4200DB7B1E0F2F00DDC9
:1087C0000F27BE4203DA5B429E4200DB82E03000AC
:1087D000FCF731FA02000B000098019905F05EF8F1
:1087E00001262060616020686168FCF7F5FAB042FC
:1087F0004FDB3F4B2F68A5331B78032B00D06CE079
:10880000032E00D069E000223A4B033722606360F8
:108810002F603EE0022BDAD0032B4DD10098019956
:108820000022354B03F0C6FF002807D100980199BC
:108830000022304B03F0AAFF00284BD03000FCF799
:10884000FAF902000B000098019905F027F8206062
:108850006160300003F026FE032103F069FF0E1E65
:1088600017D02B6800932268636802920393009BE1
:10887000002B10DD0800FCF7DEF9029A039B05F0DF
:1088800017FC009B206061609F1B01362F60002E4B
:10889000A9D105B0F0BD03277F1A3800FCF7CBF94A
:1088A000029A039B05F004FC206061600420009B99
:1088B000861BDF1B2F6096E7042BEAD10E20801B5E
:1088C000FCF7B9F902000B000098019905F0F0FBE4
:1088D0002060616000232B60DBE7701EFCF7ABF9C2
:1088E00004F08CFC04F0A8FC0137206061608FE785
:1088F000A80800100000F03F00408F40F0B58BB09A
:10890000FDF72EFE3B4C08A823002600A83319686B
:108910005A68089109929A68DB68069207930223C5
:10892000A53635780F2205A93370FFF72DFF0F22EA
:1089300006A804A9FFF728FFA63435702078FCF7B5
:108940007AF904F05BFC032D03D10A22002303F023
:108950009DFC04F071FC089A099B04000D0005F0D1
:10896000A7FBF8F70BF822002B0004F097FF069AFC
:10897000079B06000F002000290005F099FBF7F780
:10898000FDFF22002B0004F089FF040005980D0074
:10899000FCF751F902000B003000390005F088FBAC
:1089A000029003910498FCF746F9124E0090019151
:1089B000002200232000290005F07AFB009A019B89
:1089C00005F076FB029A039B370004F04BFC009AFB
:1089D000019BA8373860796037002000290005F036
:1089E00067FB0123B037A4363860796033700BB071
:1089F000F0BDC046A8080010F0B597B0019019006E
:108A000010000892099315001C00F8F763FDC34994
:108A1000049000280ED16300C14A5B08D3420ED4F3
:108A2000210000220023280003F0BAFEBD490028DF
:108A300000D1BD49019803F016FB17B0F0BD00222C
:108A400000232800210003F097FE00280FD0B74B29
:108A5000A5331B780895043B1A00531E9A418023C6
:108A60001B06E4181C9B0492013B09941C931C9A5E
:108A70000BA908A8FFF788FE089B099C1800210095
:108A80000693079404F0BAFB03000C0002900391D4
:108A90000E930F9404F0D0FB0D000400FCF79CF93A
:108AA000220005902B00461C0698079905F072FDE0
:108AB000029B039A0690079113430F27002B00D1C6
:108AC0001027BF1B3800FCF7B6F802000B000400AB
:108AD0000D000698079905F0EBFAF7F74FFF04F041
:108AE0008DFB0C900D9104F0A7FB22002B0003F0EE
:108AF00061FE002820D000220023012000210C92DA
:108B00000D93029A039B12184B41100019000B9C05
:108B10000E900F9104F090FBFCF75EF9B0420BDB76
:108B2000002C00D1B4E00598FCF785F804F066FB52
:108B30000E900F9101340B940B9C002C07D0200059
:108B400006F0A6F8FCF748F9E40F24180234774B36
:108B50001A00A533A63215781B782A00032B02D100
:108B6000AA1BAE4200DC0F25002F00D193E03B0092
:108B7000974200DD13001C9A141BA11B1A008B42A4
:108B800000DD0A00D143C9170A400292BA4200DB55
:108B900086E0BA1A39000CA8FCF7F0FC00281DD0BA
:108BA00000220023012000210C920D930E9A0F9BAE
:108BB000801859410E900F9104F03EFBFCF70CF920
:108BC000B0420BDB0B9F002F68D0701EFCF733F810
:108BD00004F014FB0E900F9101370B97002C00DC72
:108BE0000124A6425EDD341B220031000EA8FCF7F2
:108BF000C5FC002809D00E980F990B2364220B9313
:108C0000002303F043FB0E900F910B9B1C190B9458
:108C10001422002111A803F031FA029A444911A844
:108C200003F021FA049B012B08D1019803F05EFAAE
:108C3000019B2D2218183F4903F015FA019803F003
:108C400055FA019B3C4918180E9A0F9B03F00BFA3A
:108C5000029B002B4EDD019803F048FA019B11A9FD
:108C600018180C9A0D9B03F0FEF90B9B002B00D1FA
:108C7000E3E62E4B0198A5331B78042B47D103F074
:108C800035FA2E22019B2B49181803F0ECF9D4E693
:108C9000059E023650E701235B426CE701369DE7F3
:108CA00002939BE7AE42B3DD771B3800FBF7C3FFAF
:108CB0003A0004000D000EA83100022E0EDCFCF775
:108CC0005DFC0E980F9904F0B7FA22002B0005F016
:108CD000EFF904F093FA0E900F9199E7FCF74EFC30
:108CE0000028EED0002301220E920F930B9B03333A
:108CF0000B938DE7029B002BB7D1019803F0F6F997
:108D0000019B2E2218180B4903F0ADF9ADE703F0D3
:108D1000EDF9019B0B9A18180849B6E7D3F7000044
:108D200000001080D8F70000D7F70000A808001056
:108D3000DCF7000091F80000E6F70000EBF7000018
:108D400082B0F0B593B019931C9B1892023BDA0FD6
:108D5000D3185B100390162200210CA8029303F095
:108D60008DF91622002106A803F088F91A9C1B9D94
:108D7000404E330080331B78002B5DD01898199932
:108D800022002B00F8F768FC189A199B04900591B3
:108D900020002900FAF7A6FD33007E367F331A78CB
:108DA000337804000D00134338D10022324B05F014
:108DB0007FF9324A324B04F071FD1E2604000D008B
:108DC000029B0CA80093049A059BFFF715FE0CA8C4
:108DD00003F08CF9029B984206D20CA803F086F9A6
:108DE000029B5B001B1A0293029B06AF00932200BA
:108DF0002B003800FFF700FE1E4B1A00A532127838
:108E0000042A1FD133001F4900970CAA039803F0CE
:108E10002AF913B0F0BC08BC02B018471E26002A7D
:108E2000CED00022184B05F043F9144A144B04F03D
:108E300035FD04000D00C3E7189A199B69260492BA
:108E40000593BDE780331B78002B04D000973300D7
:108E50000CAA0E49DAE7002200232900200003F0C3
:108E60009FFC00963B000CAA09490028CED1094975
:108E7000CCE7C046A808001000807640182D445466
:108E8000FB211940F0F7000000007940F7F70000DF
:108E900000F800000AF8000070B5214C23009C3354
:108EA0001B785B060AD51F487030037E002B02D169
:108EB0001D4903F0D8F8FFF7D1F970BD2500A8359A
:108EC000FDF788F8AA68EB6828686968FCF7DAFBA0
:108ED000EB23DB00E618154A154B3068716805F086
:108EE000E7F804F06DF9ED23DB00E050114803F0E2
:108EF000DDFA05F0CDFE0D4A0D4B04F0CFFCEC235E
:108F0000DB00306071600022E6180023326073607D
:108F1000AA60EB600123A434286069602370CCE769
:108F2000A808001018000010A6F700000000C0FFFD
:108F3000FFFFDF411010001010B5284C2849703495
:108F4000200003F0E5F8002802D1FDF71FF810BD5E
:108F5000200003F0CBF800280FD0200003F0C6F863
:108F60000023201801380370200003F0BFF8002808
:108F7000EDD11C4BA4331870E9E71A4B1A009C3250
:108F80001278002A02D0FFF751F8E0E71A00853284
:108F90001278002A1AD07C331C88002CD7D0124BB0
:108FA000185DFBF7B1FF002802D0A01C022107E0EA
:108FB0002000FCF777F801210300601C002BF5D19D
:108FC0004942FBF7EDFFFCF799F8C0E7200003F0FA
:108FD0008DF80028BBD1FCF7E5FFB8E718000010BA
:108FE000AAF70000A8080010D400001010B50F4C1C
:108FF000FE2070342378492B13D00D49200003F054
:1090000087F80300FF20002B0BD00A49200003F053
:109010007FF80300FD20002B03D02078402801D9E1
:10902000233010BD2000FCF7EFFDFAE71800001018
:10903000AAF70000A6F7000070B5FCF7CBFF1E4CA6
:1090400025009C352B78002B0AD08534FFF7CEFF06
:109050002378002B03D0C1B27320FBF7FBFF70BD58
:10906000230086331B78002B15D023007C331A880D
:10907000124B9B185878FFF71FFB230087331B7890
:10908000002BECD10E4B2418E4182378002BE6D1EA
:10909000FBF7BCFFE3E7FEF7C9FF05232B702300B6
:1090A000084AA0331A60012378340749074823701F
:1090B00002F0D9FFD3E7C046A8080010D400001082
:1090C0006C0700003990000013F800003009001010
:1090D00070B5FCF77FFF224C25009C352B78002BC8
:1090E00016D0FFF783FF230085331D78C0B2002D13
:1090F00004D001006F20FBF7ADFF70BDFFF7DCFA75
:10910000184B2018C01805700123A4342370F4E70D
:10911000230086331B78002B11D023007C331A8860
:10912000114B9B185878FFF7C7FA230087331B7839
:10913000002BE2D10B4A201880180370E4E7FEF7F9
:1091400075FF05232B702300084AA0331A60012302
:10915000783407490748237002F085FFCDE7C04601
:10916000A80800106C070000D4000010D190000087
:109170001FF800003009001070B5FCF72BFF204CE1
:1091800025009C352B78002B16D0FFF72FFF2300EE
:1091900085331B78C0B2002B04D001006B20FBF795
:1091A00059FF70BDFFF788FA164B2018C01801232D
:1091B000A43403702370F4E7230086331B78002B5C
:1091C0000DD023007C331A880F4B9B185878FFF77B
:1091D00073FA230087331B78002BE2D1E4E7FEF714
:1091E00025FF05232B702300084AA0331A600123B2
:1091F000783407490748237002F035FFD1E7C046AD
:10920000A80800106C070000D4000010799100003D
:109210002BF8000030090010F8B5FCF7DBFE1D4C00
:1092200025009C352B78002B23D0FFF7DFFEC0B242
:10923000FBF77AFF184B984217DC0222012103004A
:109240009446164F091AFA22CD18D200934206D03E
:10925000FA5C562A03D066460133B243F3D10221A9
:109260004942491B4019FBF79BFE00237C342380B5
:10927000F8BDFEF7DBFE08232B702300084AA0335D
:109280001A600223783407490748237002F0EBFE86
:10929000EEE7C046A8080010CF070000D400001079
:1092A0001992000035F8000030090010F0B5334C79
:1092B00089B025009C352B78002B0BD08534FFF727
:1092C00095FE2378002B03D0C1B24B20FBF7C2FEE2
:1092D00009B0F0BD230086331B78002B3CD0FCF78F
:1092E00079FE23007C331A88254B9B185878FFF7AA
:1092F0002BFA05002D0165192F00224E0937310088
:10930000FBF700FD3068716807AB009305AA06AB58
:10931000FBF7C2FC059A079BFF379E180798BA68AF
:10932000FB6805960292039305F0B2FC02000B0065
:109330003868796803F096FF029A039BF835AA61B2
:10934000EB61069B286169619E4201DDFBF75EFED1
:109350000123A4342370BBE7FCF73CFEFEF766FE56
:1093600007232B702300084AA0331A6002237834A5
:1093700006490748237002F076FEA9E7A808001006
:10938000D4000010A0090010AD92000042F80000C7
:1093900030090010F0B5334C89B025009C352B788E
:1093A000002B0BD08534FFF721FE2378002B03D050
:1093B000C1B24720FBF74EFE09B0F0BD2300863353
:1093C0001B78002B3CD0FCF705FE23007C331A8869
:1093D000254B9B185878FFF7B7F905002D01651943
:1093E0002F00224E09373100FBF78CFC3068716882
:1093F00007AB009305AA06ABFBF74EFC059B079A4B
:10940000FF379E1A0798BA68FB6805960292039385
:1094100005F03EFC02000B003868796805F0BAF8E8
:10942000029A039BF835AA61EB61069B286169618A
:109430009E4201DCFBF7EAFD0123A4342370BBE765
:10944000FCF7C8FDFEF7F2FD07232B702300084A46
:10945000A0331A600223783406490748237002F0CB
:1094600002FEA9E7A8080010D4000010A00900100F
:109470009593000046F800003009001070B52D4C9F
:1094800025009C352B78002B19D0FFF7AFFD23006A
:1094900085331B78C0B2002B1ED001004320FBF7A0
:1094A000D9FD70BD2D0165190935FF353268736826
:1094B0002A606B60B268F368AA60EB6023E0230067
:1094C00086331B78002B22D0FCF784FD23007C33ED
:1094D0001A88194B9B185878FFF736F92600210097
:1094E000F836A8310A684B680500326073608A68F4
:1094F000CB68B260F360FBF705FC652DD2DD23007D
:10950000032287331A700123A4342370C9E7FCF7C0
:1095100061FDFEF78BFD07232B702300074AA03364
:109520001A600223783406490648237002F09BFD36
:10953000B7E7C046A8080010D40000107D940000D2
:109540004AF800003009001070B51F4C25009C350A
:109550002B78002B12D0FFF749FD230085331B78B1
:10956000C0B2002B15D001004C20FBF773FD70BD7D
:1095700001221A700323A5342370F8E723008633F1
:109580001B78002B0DD023007C331A880F4B9B18BF
:109590005878FFF7A9F82300A6330028E8DD1870F3
:1095A000E8E7FCF717FDFEF741FD230002227833C0
:1095B000074908481A7002F056FD074BA034236093
:1095C00005232B70D3E7C046A8080010D400001074
:1095D0004FF80000300900104995000070B51C4C90
:1095E00025009C352B78002B0CD0FFF7FFFC2300C7
:1095F00085331B78C0B2002B0FD001004820FBF749
:1096000029FD70BD230086331B78002B0ED023006C
:109610007C331A880F4B9B185878FFF765F82300A6
:10962000A63318700223A5342370EAE7FCF7D2FCB6
:10963000FEF7FCFC230002227833074907481A7022
:1096400002F011FD064BA034236005232B70D8E7F0
:10965000A8080010D400001053F8000030090010D2
:10966000DD95000070B51C4C25009C352B78002B37
:109670000CD0FFF7BBFC230085331B78C0B2002B56
:109680000FD001004420FBF7E5FC70BD23008633BA
:109690001B78002B0ED023007C331A880F4B9B18AD
:1096A0005878FFF721F82300A63318700123A5345A
:1096B0002370EAE7FCF78EFCFEF7B8FC23000222D9
:1096C0007833074907481A7002F0CDFC064BA034E6
:1096D000236005232B70D8E7A8080010D4000010E1
:1096E00057F80000300900106596000070B5264C50
:1096F00025009C352B78002B1BD0FFF777FC23002F
:1097000085331B78C0B2002B20D001000D20FBF761
:10971000A1FC70BD2300000120180930FF30A833E0
:1097200019685A68016042609A68DB688260C360A9
:1097300014E0230086331B78002B13D0FCF74AFC7F
:1097400023007C331A88114B9B185878FEF7FCFFD6
:109750006528DFDD2300032287331A700123A43438
:109760002370D6E7FCF736FCFEF760FC56232B701F
:109770002300074AA0331A600223783405490648BB
:10978000237002F070FCC4E7A8080010D400001099
:10979000ED9600005BF800003009001030B5314C48
:1097A00085B025009C352B78002B26D0FFF71EFCBA
:1097B000230085331B78C5B2002B05D0290011206A
:1097C000FBF748FC05B030BD274B196C5A6C009173
:1097D00001929A6CDB6C0098019902920393029AB1
:1097E000039BFBF74FFF2800FEF7AEFF1F49FBF777
:1097F00089FA0123A4342370E4E7230086331B781D
:10980000002B1CD0FCF7E6FB23007C331A88184B96
:109810009B185878FEF798FF0500134B196C5A6C8B
:10982000009101929A6CDB6C00980199029203936B
:10983000029A039BFBF726FF0C492800D7E7FCF7A9
:10984000C9FBFEF7F3FB56232B702300094AA03314
:109850001A600223783408490848237002F003FC98
:10986000B0E7C046A808001070EE000050090010D4
:10987000D40000109D9700005FF800003009001030
:1098800070B5174C01222300A4331A7023008633CD
:109890001B780500002B0ED07C34FCF79BFB228844
:1098A000104B9B185878FEF74FFF04000E4920001C
:1098B000FBF728FA10E023009C331B78002B0DD017
:1098C000FFF794FB85342378C0B2002BEBD0010066
:1098D0002800FBF7BFFB054C200070BD034CE5E7FB
:1098E000A8080010D4000010A0090010FFFFFF7F9F
:1098F000F7B57920FFF7C4FF050064281FDC104C82
:109900002D0127002600A837F836326873683868BA
:10991000796803F0A7FCBA68FB6800900191B06811
:10992000F16803F09FFC009A019B6419F8343260DF
:109930007360B060F16022616361A061E161F7BDB5
:10994000A8080010F7B57A20FFF79AFF05006428F1
:109950001FDC104C2D0126002700F836A8373A6886
:109960007B683068716804F015FEBA68FB68009087
:109970000191B068F16804F00DFE009A019B641932
:10998000F83432607360B060F16022616361A0619D
:10999000E161F7BDA808001070B57B208AB0FFF721
:1099A0006FFF0500642824DC134C2D0123002600E2
:1099B000A8339968DA68049105921A685B68029284
:1099C0000393F836B268F368009201936419326821
:1099D000736806A8F83402F0F7FE06980799089A0B
:1099E000099B30607160B260F36020616161A261C7
:1099F000E3610AB070BDC046A808001070B57C20B5
:109A00008AB0FFF73DFF0500642824DC134C2D01CC
:109A100023002600A8339968DA68049105921A6831
:109A20005B6802920393F836B268F3680092019380
:109A300064193268736806A8F83403F039F9069897
:109A40000799089A099B30607160B260F3602061E9
:109A50006161A261E3610AB070BDC046A808001050
:109A600073B57D20FFF70CFF642819DC0D4C250031
:109A70002600A835F836B268F368A868E96803F0EC
:109A8000F1FB32687368009001912868696803F0FF
:109A9000E9FB009A019BB034286069602260636032
:109AA00073BDC046A808001073B57E20FFF7E8FE1E
:109AB000642819DC0D4C25002600A835F836B2685C
:109AC000F368A868E96804F065FD3268736800907F
:109AD00001912868696804F05DFD009A019BB0342B
:109AE000286069602260636073BDC046A8080010EA
:109AF00030B57F208BB0FFF7C3FE64281EDC104C0E
:109B000006A823002500F8339968DA6804910592C5
:109B10001A685B6802920393A835AA68EB68009202
:109B200001932A686B6802F04FFE069A079BB034D7
:109B30002A606B60089A099B226063600BB030BD9D
:109B4000A808001030B580208BB0FFF799FE64287C
:109B50001EDC104C06A823002500F8339968DA684B
:109B6000049105921A685B6802920393A835AA686B
:109B7000EB68009201932A686B6803F099F8069AE3
:109B8000079BB0342A606B60089A099B226063606F
:109B90000BB030BDA808001070B5114C114E250057
:109BA000A0352B68B3420DD1FFF720FAC0B2FBF706
:109BB000D1FA002803D104238734237001E07C34D8
:109BC000208070BDFEF732FA230002227833064966
:109BD00006481A709C3402F046FA2E600923ECE71E
:109BE000A8080010999B000063F8000030090010DD
:109BF00070B5FCF7EFF9244C25009C352B78002B31
:109C00000AD085342378002B05D0FFF7EFF9C1B2D5
:109C10000720FBF71FFA70BD230086331B78002B4B
:109C200019D0230001222500A4331A707C352A881C
:109C3000164B9B185878FBF78DFA002807D12300A4
:109C4000042287331A700123A4342370E3E72880A9
:109C5000FBF754FAF7E7230085331B78002B0FD06E
:109C6000FEF7E4F90C232B702300094AA0331A6095
:109C70000223783407490848237002F0F4F9CAE750
:109C8000FFF78AFFC7E7C046A8080010D4000010FD
:109C9000F19B00006EF800003009001070B5184C00
:109CA000184E2500A0352B68B34213D1FFF79EF95B
:109CB000061E00D10136FBF753F90500B04200DD66
:109CC00035002800FBF7EEF9431E98417C342D182F
:109CD000258070BDFEF7AAF9FBF742F904F0D8FF22
:109CE000FBF77AF8230001307833187006490748EB
:109CF00002F0B9F901239C342E602370E9E7C046D5
:109D0000A80800109D9C000077F8000030090010A2
:109D1000F7B5304C220083321378002B08D00C2B7F
:109D200004D10B3B1370FBF77FFEF7BD0133F9E75E
:109D3000294D70352B7E002B17D06E7EA97E744284
:109D400074410C40E97E701C2818AB19AA7D0C43A5
:109D500004D00100180002F0B4F9E4E7190002F0A1
:109D6000B0F92D236C75AB55DDE723000122A43338
:109D70001A702300A8331A685E6801929F68DD6834
:109D8000002200230198310002F0F0FC002802D1EB
:109D900080231B06F618002200233800290002F059
:109DA000E5FC002802D180231B06ED1800220023C9
:109DB0003800290004F07CF9019A330003F052FACC
:109DC000064B3A00186059602B00B0342260636083
:109DD000A9E7C046A808001018000010500900109C
:109DE000F0B5504D89B0280002F080F94E4E009039
:109DF00028220021300002F041F94C4F4C4CE35D29
:109E0000002B0FD0280002F071F92018873003785A
:109E10002B2B39D1280002F069F9444B2018E35C60
:109E200087300370230083331B78424F002B4AD0C6
:109E3000414A9B00D3189A6C390002A802F013F92A
:109E400023009C331B78DB0603D53C49300002F02D
:109E500061FB02A9300002F05DFB23009C331B78FC
:109E6000002B55D02200A032354B126800259A42B3
:109E700008D0344F7037230078331B78BA7D9B1A93
:109E8000AB423FDC09B0F0BD280002F02FF92018EA
:109E9000873003782D2BBDD0280002F027F9201839
:109EA000873003782A2BB5D0280002F01FF920183C
:109EB000873003782F2BADD0280002F017F9201837
:109EC0008830E35DADE71222009BD31A1D4A01934F
:109ED00070320092937D019A93420CDD1A4A1B491D
:109EE0000F32300002F0BFF8009B9A7D019BD21A1E
:109EF000009B9A18A0E72A003900300002F0B3F85E
:109F0000009A99E71249300002F004FB0135B2E7EC
:109F10000C4B70339B7D0E2BB4D80D49300002F0F2
:109F2000F9FAAFE730090010D008001076070000FA
:109F3000A8080010C8F70000F0EE000035F9000096
:109F400081800000180000100000001083F800005D
:109F500087F80000F0B5CD4E89B0282200213000EE
:109F600002F08CF8CA4D28220021280002F086F861
:109F7000C84C14220021200002F080F81422002195
:109F8000C54802F07BF8330085331B78002B05D1E0
:109F9000330079331B78002B00D1E6E033007C33AB
:109FA0001988002904D0013900223000FEF7FAFA9E
:109FB00037007C37012239882800FEF7F3FA388809
:109FC000FBF782F80200692807DCB449632801DD49
:109FD000B349233A200002F046F89C363378002B30
:109FE00001D0FFF7FDFEA94C230087331B78002B1F
:109FF00044D0012B03D1AB49200002F034F82300F8
:10A0000087331B78022B03D1A749200002F02BF8DD
:10A01000230087331B78042B03D1A449200002F0CE
:10A0200022F8230087331B78052B03D1A049200099
:10A0300002F019F8230087331B78032B03D19D49C5
:10A04000200002F010F8230087331B78062B03D181
:10A050009949200002F007F8230087331B78072B6B
:10A0600003D19649200001F0FEFF230087331B78BF
:10A07000092B03D19249200001F0F5FF23007A3328
:10A080001B78002B03D08F49200001F0ECFF230048
:10A0900086331B78002B14D12300A5331B78042BA7
:10A0A0000FD0230084331B7887495BB2012B00D18A
:10A0B000E7E0013300D0D7E01D228449764801F063
:10A0C000D2FF230085331B78724D002B28D123004B
:10A0D000A5331B78042B23D023007E331B78002B61
:10A0E00003D07B49280002F015FA23007F331B7848
:10A0F000002B03D07749280002F00CFAEF23DB0095
:10A10000E35C002B03D07449634802F003FA230098
:10A1100080331B78002B03D07049280002F0FAF935
:10A12000FDF76EFE20000021FBF720FE08215848B5
:10A13000FBF71CFE002383211A0028008334FBF761
:10A1400043FC2378002B00D1E0E0012308226821A2
:10A150006348FBF739FC0123082252216148FBF7D1
:10A1600033FCFBF7DEF809B0F0BD330086331B7813
:10A17000002B0FD033007C331B885B4AD35C2A2B27
:10A1800008D05A49300001F06EFF5949280001F00B
:10A190006AFF28E73300A53356481B780C30042BA0
:10A1A00050D101F0A3FF16245349241A300001F0C6
:10A1B0005AFF374F5149380001F055FF300001F088
:10A1C00095FF3300B8331A68351805929E685A68AF
:10A1D000DB6806920793002200233000079902F003
:10A1E000C5FA002832D10799059A069B029401917D
:10A1F00000962800FEF7A4FD380001F077FF234BFE
:10A200003F18A8331A689D68DE6805925A682800CE
:10A21000069200230022310002F0A8FA00281CD187
:10A22000059A069B0294019600953800FEF788FD7A
:10A23000334B70331B7E002B00D0D2E6134B9C3384
:10A240001B78CCE601F052FF1224ADE70094059A8A
:10A25000069B2800FEF7D0FBCEE70094059A069BEC
:10A260003800FEF7C9FBE3E7230082331B7825495A
:10A27000002B06D1230081331B78002B00D120E76F
:10A280002149054802F046F91BE7C046A80800101E
:10A29000D0080010F80800100C09001094F8000015
:10A2A00089F80000B3F80000BFF80000CCF8000007
:10A2B000D5F80000E2F80000EDF80000FFF800001B
:10A2C0000CF9000014F900001AF900001CF9000054
:10A2D00022F9000026F9000029F900002CF90000FD
:10A2E0002FF9000033F90000D40000109FF800009F
:10A2F000A7F8000000000010ADF80000B0F8000062
:10A3000018000010A5F8000020F9000008228321A1
:10A31000004824E70C090010F0B5434B83B005005A
:10A320000191160098423DDC019B002B59D000287A
:10A3300040D07C21862301223C4CADB26552E254D0
:10A340002800FAF7AFFE002840D1002E44D0384E46
:10A35000384F0EE098478623E35C002B54D08723C8
:10A36000E35C002B0ED1FAF751FE00280AD17C23C2
:10A37000E55A735D9A00002B44D0802B02D8D35944
:10A38000002BE7D1012586230022E254FBF722FEB1
:10A390008723E35C072B39D0019B002B07D1F6F70D
:10A3A00015FA04E0872203210125204B9954280047
:10A3B00003B0F0BD012386217C221C4C013528000E
:10A3C0006354A352FAF76EFE0028BED0FAF71EFEC1
:10A3D0007C23E55A002EBAD1174B184A5B69A3506B
:10A3E000B5E7FBF7A7FA002D16D0862201217C23C2
:10A3F0000E4CA154E552124BE35C002B09D07C2398
:10A40000E55A9DE7FAF77AFE0025BCE7FAF7FEFD6C
:10A41000C2E7FFF79FFDF2E7012386217C22034C70
:10A420006354A352E7E7C046CF070000A808001016
:10A43000D400001014F40000180000107C07000085
:10A4400077070000F8B5254C25009C352B78002BAC
:10A4500026D0FEF7CBFDC5B22800FEF759F9230040
:10A4600085331F780600002F0AD0002803D005236B
:10A470008734237003E029002B20FAF7EBFDF8BDA9
:10A4800000280AD0FDF7D2FD0123A4343A00390098
:10A4900030002370FFF740FFF1E787340423E8E73B
:10A4A000230086331B78002BE9D1FBF793FDFDF7E2
:10A4B000BDFD08232B702300094AA0331A60230036
:10A4C000022278331A708534237806480649002B17
:10A4D00000D1064901F0C7FDD1E7C046A808001029
:10A4E00045A400003009001037F9000041F90000D0
:10A4F00070B5194D2B009C331B781A0709D5174BE3
:10A5000070331B7E002B03D1FBF7DEFAFDF7A6FEAE
:10A5100070BD002BFCD12B0085331E782330C4B2D4
:10A52000002E04D021000720FAF794FDF0E7FBF796
:10A5300051FD2B000122A43320001A70FEF7E8F829
:10A54000002804D032003100FFF7E6FEE0E70422E5
:10A5500087352A70DCE7C046A808001018000010F4
:10A5600010B54520FFF7C4FF10BD10B54420FFF71C
:10A57000BFFF10BD10B54320FFF7BAFF10BD10B5E7
:10A580004220FFF7B5FF10BD10B54120FFF7B0FF27
:10A5900010BDF8B50B4C060025001000002300226A
:10A5A0000F000949E8350E604F608A60CB601031BA
:10A5B000A942F8D10122A8341100FFF7ADFE2068AE
:10A5C0006168F8BDA808001050090010F8B5174CD4
:10A5D0001D00230006000F00A8331E605F602300EB
:10A5E00000200021B0331860596030003900FFF7B7
:10A5F000D0FF02000B002A606B60250087352B78A6
:10A600000120002B07D18140C1401800084BD942DE
:10A610000AD409202870210000220023A831B03478
:10A620000E604F6022606360F8BDC046A80800104D
:10A6300000001080F0B58DB00292039380239B0040
:10A640000990089302980399F7F7D0FF00900191C1
:10A6500014981599F7F7CAFF04000D0002000B00CB
:10A660000098019902F09CF8002801D1009401950E
:10A67000009801990022524B02F07EF8002803D086
:10A6800000234F4C00930194149A159B0298039950
:10A6900002F0E8FD00224B4B03F00AFD0AAB099AD9
:10A6A00004000D00FFF792FF0590002806D0464BEE
:10A6B00087331B78059305980DB0F0BD0A9E0B9F5C
:10A6C000002200233000390002F050F800280AD0A0
:10A6D0003D4B00211A00A832146055600022B033AF
:10A6E00019605A60E7E7029A039B1498159903F0E2
:10A6F00051FFF7F77BFF0022069007910098019920
:10A70000324B03F0D5FC02000B000698079902F0CB
:10A710003DF80028DCD1129813990022002302F0A2
:10A720002BF8002807D0002200233000390002F067
:10A7300037F8002834D1129813990022002302F030
:10A740002FF8002807D0002200233000390002F043
:10A7500013F8002824D1169817990022002302F03C
:10A760000BF8002807D0002200233000390002F047
:10A7700017F800280FD1169817990022002302F02D
:10A780000FF8002816D0002200233000390001F015
:10A79000F3FF00280ED0129613970294039503E05E
:10A7A0001696179714941595089B013B0893002B58
:10A7B00000D047E70924044B059487331C707AE7DF
:10A7C0000000F03F0000E03FA80800100000D03C6F
:10A7D000C54BF0B51A00A9B0A832116852680691AD
:10A7E00007921A00B832116852680A910B9200223F
:10A7F00087331190069807991A70F7F7F7FE04004F
:10A800000D000A980B99F7F7F1FE06000F00020001
:10A810000B002000290001F0C3FF002801D0260012
:10A820002F000A9A0B9B0698079903F0B3FEF7F7DF
:10A83000DDFE002208900991AC4B3000390003F096
:10A8400037FC02000B000898099901F09FFF0028CF
:10A8500035D00022A64B2000290001F08DFF0028F2
:10A8600001D00024A24D0022A24B2000290003F0B9
:10A870001FFC002206000F009F4B2000290003F060
:10A8800017FC04000D0002000B003000390001F03D
:10A8900073FF002801D026002F0006980799320088
:10A8A0003B0003F077FE320004000D000698079984
:10A8B0003B0002F0D7FC069407950A900B9106988E
:10A8C000079922AB119AFFF781FE0890002804D067
:10A8D000854B87331B78089313E000242298239933
:10A8E000002522002B0001F041FF00280CD0069823
:10A8F00007997D4B1A00A832B033106051601C607C
:10A900005D60089829B0F0BD20AB119A0A980B99A8
:10A91000FFF75CFE08900028DAD1209A219B0E9266
:10A920000F930E980F990022002301F01FFF0028BB
:10A9300005D00A980B996C4B1A00A832DCE7229BD1
:10A94000239C180021000C930D94F7F74FFE06008E
:10A950000F000E980F99F7F749FE02000B00040054
:10A960000D003000390001F011FF069A079B002806
:10A9700001D10A9A0B9B1E921F93300022002B00DC
:10A98000390001F003FF0C9A0D9B002801D10E9AAB
:10A990000F9B0C980D991C921D930022002301F02F
:10A9A000EBFE002808D00E980F990022002301F03A
:10A9B000F7FE002800D072E00C980D9900220023C9
:10A9C00001F0EEFE002807D00E980F990022002318
:10A9D00001F0D2FE002862D10A9A0B9B06980799D3
:10A9E00001F0DEFE00286DD10A9B0B9C129313949C
:10A9F000069B079C1493159480235B001893149A6C
:10AA0000159B1298139903F0C5FD06000F00F7F788
:10AA1000EDFD1690179114981599F7F7E7FD0400CE
:10AA20000D0012981399F7F7E1FD02000B002000CA
:10AA3000290002F017FC00222D4B02F013FC00222B
:10AA40002E4B03F035FB02000B001698179901F00E
:10AA50009DFE002800D0B3E00022294B30003900D1
:10AA600002F01CFF149A159B04000D0002F0FAFB83
:10AA7000220016901791129813992B0003F08AFD6B
:10AA800026AB06000F0016981799119AFFF79EFD46
:10AA9000041E37D0144B87331C78089431E70E9B83
:10AAA0000F9C049305940A9B0B9C029303940C9BAC
:10AAB0000D9C00930194069A079B1198FFF7BAFD2D
:10AAC00008901EE70C9A0D9B0E980F990E920F930B
:10AAD000069A079B0C900D910A980B990A920B937A
:10AAE0000690079180E7C046A80800100000E03CEF
:10AAF0000000F03F0000D03F0000503D0000D03C7F
:10AB0000000008401CAB1EAD019316981799269AB9
:10AB1000279B0095FAF7C8FC269827990022002366
:10AB200001F024FE00280CD0B74B169817991A0094
:10AB3000A8321060516000210022B03319605A60C1
:10AB4000ABE724AB119A30003900FFF73FFD041E3C
:10AB5000A0D11CAB01933000249A259B39000095AD
:10AB6000FAF7A2FC249A259B1A921B931A981B9918
:10AB70000022002301F0FAFD002805D0A24B1A00A4
:10AB8000A83216605760D6E726982799F7F72EFD6A
:10AB900004000D001A981B99F7F728FD02000B001E
:10ABA0002000290001F0E8FD002848D1169B179CE1
:10ABB00014931594189B013B1893002B00D01EE7AB
:10ABC000069A079B0A980B9903F0E4FC18901991D8
:10ABD0001C981D99F7F70AFD00228C4B01F0D6FD59
:10ABE00000282FD018981999894A8A4B03F060FAE7
:10ABF000069A079B1E9E1F9F04000D00300039001F
:10AC000003F0C8FC22002B0001F0CAFD002819D077
:10AC10000A980B9932003B0003F0BCFC22002B0089
:10AC200001F0BEFD00280DD0774B1A00A832166047
:10AC3000576000210022B03319605A6061E6129615
:10AC40001397B7E70A9A0B9B0698079902F00AFB3D
:10AC5000714B002203F02CFA189B199C1293139449
:10AC600080231A901B919B001693129A139B1A989B
:10AC70001B9903F08FFC1A9A1B9B06000F00129879
:10AC8000139902F0EFFA26AB14901591119A300047
:10AC90003900FFF79BFC0890002800D018E61CAB99
:10ACA00001931EAB00933000269A279B3900FAF7D8
:10ACB000FBFB269C279D002200232000290001F099
:10ACC00055FD0028B0D1002200232000290001F00A
:10ACD00053FD002807D00C980D990022002301F0A5
:10ACE0005FFD002835D1002200232000290001F05B
:10ACF00057FD002807D00C980D990022002301F081
:10AD00003BFD002825D11498159924AB119AFFF723
:10AD10005DFC0890002800D0DAE5149815991CAB6A
:10AD200001931EAB0093249A259BFAF7BDFB249C4C
:10AD3000259D002200232000290001F017FD002896
:10AD400014D0314B149815991A00A8321060516034
:10AD50006FE70C9A0D9B0094019504920593069A57
:10AD6000079B0292039332003B00A6E600220C9858
:10AD70000D99002301F000FD002807D000220023D8
:10AD80002000290001F00CFD00282FD10C980D990E
:10AD90000022002301F004FD002807D00022002338
:10ADA0002000290001F0E8FC00281FD1189A199B07
:10ADB0001298139902F056FA169B12901391013BC8
:10ADC0001693002B00D050E70F4B1E981F991A00C6
:10ADD000A832106051601A0000200021B0321060CB
:10ADE0005160092287331A7008928AE50494059508
:10ADF000149B159C029303940E9B0F9C009301944B
:10AE00000A9A0B9B59E6C046A80800100000503D66
:10AE1000BBBDD7D9DF7CDB3D0000E03FF0B53C4B4C
:10AE2000A5B01590A6331B78181C0F2B00D90F2046
:10AE3000C0B24042F9F7FFFE354C1890199123003B
:10AE4000A8331A685B680092019300980199230067
:10AE5000B8331E685F6832003B0001F0A1FC002897
:10AE60000CD000220023F83426606760A260E36003
:10AE7000009A019B0096019716001F00009A019B03
:10AE80003000390003F086FB32001A901B910098C5
:10AE900001993B0002F0E6F91E4B002203F008F98D
:10AEA0000023002405931493002320902191029302
:10AEB0000394059B0C2B2FD1029C039D144E1498D8
:10AEC000370003F0E5FEC8373300386079600022B0
:10AED0000021D03319605A60029A039B2000290098
:10AEE00003F058FBF7F782FB3300B8331860596062
:10AEF000330000210022C03319605A603300002063
:10AF0000A833B0361C605D603160726025B0F0BD62
:10AF1000A80800100000E03F059BC14C584203F018
:10AF2000B7FE0B0080210200C9050020F7F740FEA4
:10AF3000059B1C901D915A1E9341DAB201331E935A
:10AF4000DB009B181F9301235B4216931794002389
:10AF500000240A930B94069307940492049803F038
:10AF600097FE1C9A1D9B03F0A3F804000D00F7F751
:10AF7000D9FB0890099120002900F7F73BFBA94A6B
:10AF80002290239108980999A74B03F091F8C023C8
:10AF900000221B0603F08CF8F5F778FF002200234F
:10AFA00004000D0001F0E2FB002800D0CEE00022FA
:10AFB0009E4B2000290002F055F9089009910200EB
:10AFC0000B002000290002F069FC02000B00129027
:10AFD00013911A981B9903F06BF8009A019B0E903D
:10AFE0000F9102F03FF90E9A0F9B0C900D913000DB
:10AFF000390003F0CFFAF3230E900F9112981399B2
:10B0000000229B0501F0C2FB00281FD00C9A0D9B6B
:10B010000098019901F0CEFB002807D00098019913
:10B0200032003B00F9F7A2FD0C900D910E9A0F9B98
:10B030003000390001F0AAFB002807D0009A019BDC
:10B0400030003900F9F792FD0E900F911A981B9974
:10B05000744A774B03F02CF8229A239B03F028F8CC
:10B0600022002B0003F024F8089A099B04000D002D
:10B070001000190003F01CF802000B00200029004A
:10B0800002F00CFC049B04000D00159A002B00D06C
:10B090008EE020982199FFF77CFA664A4B005B0806
:10B0A000D34207D502000B002000290003F000F86E
:10B0B00010901191149B013314935F4B87331B78CD
:10B0C000002B43D1109A119B0698079902F0CAF8F9
:10B0D0000690079110981199F7F788FA02000B0073
:10B0E00004000D000A980B9902F0BCF81F9B049A0B
:10B0F0000A900B91934200DD7EE01698179922008A
:10B100002B0001F04DFB002800D178E0069807994C
:10B11000F7F76CFA00220890099118981999474B93
:10B1200002F0C6FF0A9A0B9B0C900D9108980999A2
:10B1300002F098F802000B000C980D9902F0B8FF8D
:10B1400022002B0001F02CFB002858D03A4B87330B
:10B150001B78002B00D0AFE61C9A1D9B0698079920
:10B1600002F0A6FF059B04000D00002B1AD00298E8
:10B1700003990022324B02F09BFF02000B002000DB
:10B18000290002F06FF8029A039B04000D0003F0FF
:10B1900001FAF7F72BFA189A199B01F0EDFA00283B
:10B1A00000D08BE6059B029403950133059380E65E
:10B1B0000C980D99FFF7EDF9159A0C9008910E98DF
:10B1C0000F99FFF7E6F9089B1A4A5B005B08D34228
:10B1D000BCD54B005B08D342B8D502000B000C98DD
:10B1E000089902F03FF82B00220002F061FF149B47
:10B1F0001090119102335FE7049B002B07D0129847
:10B20000139900220F4B01F0C1FA00289ED11E9A1B
:10B21000049B944663440493169417959EE6C04697
:10B22000FFFFEF7F182D4454FB21F93F0000F03F52
:10B23000FB21094000001080A80800100000D03F4A
:10B240000000E03F0000A03CF7B5FAF7C3FE274C32
:10B2500025009C352F78002F0AD085342378002BC9
:10B2600005D0FDF7C3FEC1B20620F9F7F3FEF7BD26
:10B27000260086363378002B1FD025007C352A889F
:10B280001B4B9B185878FDF743FA002803D1042381
:10B2900087342370EBE72B883900019323000124C6
:10B2A000A43322001C70FFF737F8002801D0377054
:10B2B000DDE7019B34702B80D9E7230085331B78B1
:10B2C000002B0FD0FCF7B2FE0C232B702300094A91
:10B2D000A0331A600223783407490848237000F02D
:10B2E000C2FEC4E7FEF7DAFCC1E7C046A8080010BA
:10B2F000D400001049B200004AF9000030090010E3
:10B3000010B5FAF767FE084B1A008632117800294B
:10B3100004D000231370F9F779FE10BD7C33188830
:10B320000A00FEF7F9FFF8E7A808001010B5064B71
:10B3300086331B78002B05D0FEF70CFEFA20800028
:10B34000F4F782FF10BDC046A8080010F8B5FAF760
:10B3500041FE2D4C26009C363378002B2BD0FDF778
:10B3600045FEC5B22800FDF7D3F9230085331E78CA
:10B370000700002E04D029004F20F9F76BFEF8BD1E
:10B38000FCF754FE002F11D02500012386352B70C9
:10B39000FEF7E0FDFAF7CEFA3800FFF73FFDF5F7CC
:10B3A00015FA2E700123A4342370E8E72300042249
:10B3B00087331A70F6E7250086352B78002B13D0DB
:10B3C00026007C363788114BDB195878FDF7A0F939
:10B3D000002806D0FFF722FD012337802B70A4340C
:10B3E000E2E787340423DFE7FCF720FE092333700C
:10B3F0002300074AA0331A6002237834054906481F
:10B40000237000F030FEBAE7A8080010D400001046
:10B410004DB3000053F9000030090010F7B5FAF7FA
:10B42000D9FD364C26009C363578002D2BD0FDF703
:10B43000DDFDC5B22800FDF76BF9230085331E78CA
:10B440000700002E04D029005020F9F703FEF7BDB5
:10B45000FCF7ECFD002F11D02500012386352B7061
:10B46000FEF778FDFAF766FA3800FFF7B1F9F5F75D
:10B47000ADF92E70A43401232370E8E723000422E1
:10B4800087331A70F6E71E4B1B78002B25D0260059
:10B490007C3632881B4B27009B185878FDF738F90B
:10B4A0008737002816D033880193FFF791F9019B65
:10B4B000012233802300A4331A703B78092B04D176
:10B4C000F9F7A4FD3D708634D5E7002BFBD00C4B7B
:10B4D0001D70BCE704233B70B9E7FCF7A7FD092307
:10B4E00033702300084AA0331A60022378340749D6
:10B4F0000748237000F0B7FDA9E7C046A808001070
:10B500002E090010D40000101DB4000062F90000E4
:10B51000300900104F4B10B51A694F4901321A61BA
:10B520004E4A1268D2B2302A66D01AD8182A0ED0E3
:10B5300005D8082A36D0102A44D008234EE0202A05
:10B5400069D0282AF9D1D8689A69904248D2DA6835
:10B55000501CD86001339B18DB7F414ADBB213607B
:10B56000EBE7482A57D009D8382A4DD0402AE4D1F1
:10B57000DA690423012A4BD10B60DEE7502A53D04D
:10B58000582ADAD1364A12689868D2B2441C9C60B4
:10B590001C00383422540222FF325A608023F13AD0
:10B5A000DB0552E00022DA60D868421CDA605A1CDF
:10B5B0001218D27F2A48D2B2026028220A60273AA3
:10B5C0005A6010BD00229A60DA68501CD8600133BE
:10B5D0009B18DB7F224ADBB2136028230B60F0E765
:10B5E0008022D869D205002801D02023B7E70220A5
:10B5F000FF3058601023B2E780221020D20510607F
:10B6000008220A60FA32DBE7822252005A6094E78D
:10B610008022D205A3E780221020D20510600822E4
:10B620000A600422FF32CBE70D4A12689868D2B252
:10B63000441C9C601C0038342254DA699868531EFC
:10B640000422834203D98023DB051A6075E70A6070
:10B6500073E7C046180000101800004004000040C6
:10B6600008000040202130B5064A074C0378002B23
:10B6700001D1180030BD013015680D42FCD02360A7
:10B68000F4E7C04614800040008000400E22174BB3
:10B6900010B51B681340062B12D1154B90321B6856
:10B6A000134205D0134ADBB25360134B1B6810BD25
:10B6B000DB07FCD5104B1868C0B2F4F7B5FDF6E710
:10B6C000042BF7D00C2B05D10A4AF43351680B43F5
:10B6D0005360ECE7022BEAD1054B1A68054B920642
:10B6E00002D500229A60E2E70122FBE708800040D1
:10B6F0001480004028100010008000400122034BFD
:10B700001A60034AD3680133D36070470080014058
:10B71000980000100122034B1A60034A1369013399
:10B720001361704700400140980000100122034B54
:10B730001A60034A536901335361704700000140A6
:10B74000980000100122034B1A60034A93690133E9
:10B750009361704700C0004098000010074A084BF2
:10B760005169013102D1D9690131D9615169013180
:10B7700051611A6A01321A627047C04618000010FF
:10B78000980000101B4B10B59A6D002A2AD0DA6D74
:10B790000132DA65184B9868FAF7A4FB8022174B40
:10B7A0000121DA679218DA678022D200DA678022F4
:10B7B0005201DA6780221201DA6780229200DA678A
:10B7C00000230F4A494213600E4A11600E4A13606B
:10B7D0000E4A136001220E4B1A60F4F771FCC0464A
:10B7E000C04610BD08220B4B87331A70F4F7EEFFEA
:10B7F000F7E7C046180000100000001004E100E068
:10B80000048204400882044004C000403CC0004060
:10B8100000C00040A8080010F7B5F4F72BFDC04A9F
:10B82000012413681B0B1B031360BE4A13681B0B18
:10B830001B031360BC4A13681B0B1B031360BB4A3A
:10B8400013681B0B1B0313600022B94B1A60B94B22
:10B850001C601A601C601A682242FCD02322B64B7E
:10B8600001201A60FAF73EFBF4F704FD40213F2067
:10B87000B24B1A688A431A60B14A1060B14A146028
:10B880001A688A431A60FCF7C5FAFCF7B9FAFAF7A6
:10B8900003FBF4F777FF0021AB48F4F7F9FC002134
:10B8A000AA48F4F7F5FCF4F7F3FDF4F7C1FDA84C52
:10B8B000092248340021200000F0E0FB0020E07164
:10B8C000F4F7B4FFA34D002822D0F4F775FD0C2344
:10B8D000184002D02378184320709D4C48342378B8
:10B8E0005B0711D5F4F732FDA378002B03D0237A40
:10B8F000012B02D80133237201E02B6A6B62002313
:10B90000934A2B624832D3700022914B48331A700D
:10B910008F4B4833DB79002B01D1F4F717FDFA2365
:10B9200000269B002E626B62FAF73CFAF0228A4CEA
:10B93000D2003100200000F0A1FB23000222A4333A
:10B94000FF321A802300FD3AA6331A7023000B320F
:10B9500078331A70814A82490C32824800F083FBA6
:10B96000FAF714FBFAF760F8FEF7F4FAF9F716FFA6
:10B97000061E00D143E1EF22D200A35C002B04D0CD
:10B980000023A35422007C32138000222300AA61EA
:10B9900087331F78974216D01A70FAF745F8AA69CC
:10B9A000714B9A4203D9FCF797FA0023AB61FEF77B
:10B9B000D1FAEF23DB00E35C002BD7D103210A206F
:10B9C000F4F7B0FDD2E7A02E66DDA021300000F034
:10B9D000AFFE0D2927D1FCF729FBFA27634800F0B9
:10B9E00037FB0126FF00624B6248995D013600F08B
:10B9F0002FFBBE42F7D1CC270026FF0033000933CE
:10BA0000FF33E15C5B48013600F022FBBE42F5D11A
:10BA1000594800F01DFB594E300000F019FB300072
:10BA200000F016FBB9E7112914D1FCF7FFFAFA224E
:10BA30003900D2004E4800F021FB2300EF227C3376
:10BA40001F800123D2004E48AF62A35400F000FBD8
:10BA50004A48E5E7072907D1230086331B78002BE6
:10BA60009BD1FEF799F898E7062907D12300863382
:10BA70001B78002B91D1FEF711F98EE732298CD17A
:10BA8000FA223900D2003A4800F0F8FA23007C3359
:10BA90001F80FCF7CBFA80E723009C331B78002B38
:10BAA00074D033003D3B012B21D92821300000F018
:10BAB0003FFE12291BD004230A009A43012A16D004
:10BAC0003200153A132A03D82E4BD340DB070ED48D
:10BAD00033000422143B934304D1230083331B78A7
:10BAE000002B04D133000422373B93430FD1F0B233
:10BAF000F9F7FAF91648703000F0F8FA23007833B5
:10BB00001B78984200D048E7FCF7A8FB45E71429CA
:10BB1000F0D81D4BCB40DB07ECD52831C8B2E7E7A6
:10BB200000800050008001500080025000800350CF
:10BB3000408004404480044008800440388204402F
:10BB400024800440D8800440984004409C40044035
:10BB50001800001098000010A80800100000001045
:10BB6000C8F70000300900105702000077F9000004
:10BB7000D40000106DF9000000FB00007EF9000009
:10BB800071F90000F3EE0F001091190023008533C6
:10BB90001B78F6B23000002B29D0F9F7B5F9002850
:10BBA00024D1202332009A43122A1FD033000222CC
:10BBB0009343012B1AD03300523B012B16D9612E2F
:10BBC00014D02633DBB2102B03D84E4ADA40D30709
:10BBD0000CD42821300000F053FBFB230539194217
:10BBE00004D033007F33DBB21E2B03D83000F9F7CB
:10BBF0007BF9D2E600213000F9F72CFACDE6EF23ED
:10BC0000DB00E35C002B00D1C9E63F4A917B537B0C
:10BC1000994200D1AAE6937BD318DE7B937B013354
:10BC2000DBB293735BB2002B01DA002393730D2E0A
:10BC300003D00A2E01D0202E28D12F002C37380017
:10BC4000F9F7E2FF0A2201900021380000F016FA0D
:10BC50002E4B5F612E4BE35C002B03D131002D484E
:10BC600000F0F6F9019BFF2B00D97FE622007C3221
:10BC7000138829498B4238D9AB6A28498B423BD873
:10BC8000274A0199D1540133AB626FE6082E01D0E7
:10BC90007F2E18D11E4BE35C002B14D12B001B4FC1
:10BCA0002C337A699A420ED908211A4800F0D0F94B
:10BCB0002021184800F0CCF90821164800F0C8F9F6
:10BCC0007B69013B7B613300303B092B9DD8104BD6
:10BCD000E35C002B03D131000E4800F0B9F90B4AA8
:10BCE0005369591C51611E708FE701339BB2138059
:10BCF00001990C4AD15439E600231380EF22D20077
:10BD0000A35433E611310100281000100000001088
:10BD10007707000091F80000CE0700005F060000E2
:10BD2000B0090010D400001070B500241E5D051984
:10BD3000002E08D1121B1300002B07DCD043C017C4
:10BD40001040001970BD06550134EFE72970013B22
:10BD50000135F1E7F8B505000C001E00571E092B50
:10BD600016D90A21180000F005FA210003003A0054
:10BD70002800FFF7EFFF04002D1830000A2100F023
:10BD80007FFA30312970601CF8BD2C70013F0135FD
:10BD9000002FFADC141E00DC0124013CEDE7F0B5B5
:10BDA00085B00B9E040003910A9F551E002E01D101
:10BDB000092F1DD90A2200233800310000F066FA4D
:10BDC0002A000090019120000399FFF7E8FF050089
:10BDD0002418380031000A22002300F057FA681CAA
:10BDE0003032227005B0F0BD039B013D2370013459
:10BDF000002DF9DC151E00DC0125013DE9E7F7B552
:10BE00000F00D9171E005B184B4004000193551E0C
:10BE1000092B16D918000A2100F0ACF90300002EF6
:10BE200000DA43422A0020003900FFF7E8FF05004E
:10BE3000241801980A2100F023FA3031681C21707F
:10BE4000FEBD002E00DA951E23006119CA1A002AD1
:10BE50000BDCE843C017054064196B1C002EE8DAC0
:10BE60002D221D0022700134E3E71F700133EDE73E
:10BE700073B5069E04001D0010003309013A002B23
:10BE800011D0009320002B00FFF7F2FF24180F239E
:10BE90001E40F3B2092E0DD830330130237076BD29
:10BEA0002170013A0134002AFADC002800DC01206C
:10BEB0000138ECE7002D01D03733EEE75733ECE7DC
:10BEC000F0B585B0040003911D00002801D00023C7
:10BED0000370002630001378002B00D092E0039A04
:10BEE000B24200D99AE00023013C2370013E96E063
:10BEF0005178252902D1217002328CE0302924D0DA
:10BF0000531C029320239C46029B1B782D3B5A42D4
:10BF10005341029AD31800220293029B1B781F0000
:10BF2000303F092F15D9039997198F4201D98A1BE0
:10BF3000D2B2692B46D015D8632B5ED0642B41D08A
:10BF4000582B4ED00126764269E0931C02938C4612
:10BF5000DAE70A214A439A18029B303A0133D2B2F7
:10BF60000293DAE7732B41D01FD86C2BEAD1029BE6
:10BF70005B786C2B14D1029B9B78752B10D1029BA4
:10BF800007350233072102932B008B431D001868ED
:10BF9000596800900191614620000835FFF7FFFEC7
:10BFA000029A24180132361895E7752B12D0782B97
:10BFB000C8D12B682F1D0093002361462000FFF796
:10BFC00057FF05E02B68614620002F1DFFF717FF84
:10BFD0003D00E5E72B68614620002F1DFFF7BAFE04
:10BFE000F6E72B682F1D00930123E6E72B686146D7
:10BFF00020002F1DFFF798FEEAE72B680120237031
:10C000000435CDE70399B14200D86CE7252B00D168
:10C010006EE701322370013601345CE72370300093
:10C0200005B0F0BD10B513000A006421FFF748FF0A
:10C0300010BD00B59BB00A00010001A8FFF7F2FF98
:10C04000632800DDFEE701A8FFF70CFB1BB000BD75
:10C050000FB407B504A901C90191FFF7EAFF03B0C6
:10C0600008BC04B018470EB403B503AA02CA019273
:10C07000FFF7D8FF02B008BC03B01847F0B50500C1
:10C08000830704D003009A189A4217D1F0BD030029
:10C09000032AF8D9131F0F049B080C063C439E008B
:10C0A00036180C430F0204363C4310C5B542FCD190
:10C0B000032401339B00C3182240E4E719700133C5
:10C0C000E2E710B5814208D20139431E002A00D1AF
:10C0D00010BD8C5C9C54013AF8E700238142F7D9EB
:10C0E0009A42F5D0CC5CC4540133F9E70200030056
:10C0F000981A0133591E09780029F9D170470300B5
:10C100000A781A70002A00D1704701310133F7E72D
:10C11000002210B5835C8C5CA34201D0181B10BDBB
:10C120000132002BF6D11800F9E7FEE7FEE7000028
:10C13000002370B50A480B490B4C1A188A4207D3E2
:10C1400000210A4B0A4A934206D3FFF765FBFEE73C
:10C15000E55C01331570F0E719700133F3E7C04671
:10C160000000001018000010CCFB000018000010A8
:10C17000C0110010002243088B4274D303098B4284
:10C180005FD3030A8B4244D3030B8B4228D3030CA7
:10C190008B420DD3FF22090212BA030C8B4202D349
:10C1A0001212090265D0030B8B4219D300E0090A71
:10C1B000C30B8B4201D3CB03C01A5241830B8B427A
:10C1C00001D38B03C01A5241430B8B4201D34B0363
:10C1D000C01A5241030B8B4201D30B03C01A5241C8
:10C1E000C30A8B4201D3CB02C01A5241830A8B424D
:10C1F00001D38B02C01A5241430A8B4201D34B0236
:10C20000C01A5241030A8B4201D30B02C01A524199
:10C21000CDD2C3098B4201D3CB01C01A524183094D
:10C220008B4201D38B01C01A524143098B4201D387
:10C230004B01C01A524103098B4201D30B01C01AB2
:10C240005241C3088B4201D3CB00C01A524183082C
:10C250008B4201D38B00C01A524143088B4201D359
:10C260004B00C01A5241411A00D2014652411046B9
:10C270007047FFE701B5002000F006F802BDC04698
:10C280000029F7D076E770477047C046002B11D1E0
:10C29000002A0FD1002900D1002802D00021C94373
:10C2A000081C07B4024802A14018029003BDC04612
:10C2B000D9FFFFFF03B4684601B5029800F006F805
:10C2C000019B9E4602B00CBC7047C046F0B54F467D
:10C2D0004646D646C0B5040082B00D009146984649
:10C2E0008B422FD82CD04146484600F0B1F82900A7
:10C2F0000600200000F0ACF8331A9C46203B9A461A
:10C3000000D576E04B46524693401F004B466246AE
:10C3100093401E00AF4228D825D05346A41BBD41F0
:10C32000002B00DA7BE0002200230092019301231E
:10C33000524693400193012362469340009318E0D4
:10C340008242D0D900220023009201930A9B002B45
:10C3500001D01C605D600098019902B01CBC904641
:10C360009946A246F0BDA342D7D9002200230092ED
:10C3700001936346002BE9D0FB07984641467208BB
:10C380000A437B0866460EE0AB4201D1A2420CD8BC
:10C39000A41A9D41012024196D410021013E241859
:10C3A0004D41002E06D0AB42EED9013E24196D411D
:10C3B000002EF8D100980199534600196941002BCD
:10C3C00023DB2B005246D3402A006446E2401C0087
:10C3D00053461500002B2DDB26005746BE40330088
:10C3E00026006746BE403200801A994100900191B4
:10C3F000ACE7624620239B1A4A46DA4061461300A6
:10C4000042468A4017001F4380E7624620239B1A5A
:10C410002A0066469A402300F3401343D4E762465D
:10C42000202300219B1A0022009101920122DA4070
:10C43000019280E72023624626009B1ADE402F00EF
:10C44000B0466646B74046463B003343C8E7C04661
:10C4500010B5002903D100F007F8203002E0081CD5
:10C4600000F002F810BDC0461C2101231B049842B5
:10C4700001D3000C10391B0A984201D3000A083975
:10C480001B09984201D30009043902A2105C40182C
:10C490007047C046040302020101010100000000D0
:10C4A00000000000C317C0185840704770B50568F9
:10C4B0000400002D22D01349280000F053F8C201D7
:10C4C000121A9200131ADA00D21A92001218D3002C
:10C4D000D2180D4BAA1A5A4303051B1A9B001B18AE
:10C4E0009B001B181B011B1A9B00181A8000801848
:10C4F00005D5064BC3185800400801E00448030066
:10C50000236070BD1DF30100A7410000FFFFFF7F06
:10C5100067B7E12A70B50400830717D102680F4B93
:10C52000D31893430E4A150013420FD1043002680A
:10C530000A4BD31893432B4208D104300268074BAF
:10C54000D31893432B42F1D000E001300378002B45
:10C55000FBD1FFF7D4FD200070BDC046FFFEFEFEFC
:10C560008080808003460B437FD4002243088B42A7
:10C5700074D303098B425FD3030A8B4244D3030B6A
:10C580008B4228D3030C8B420DD3FF22090212BA2F
:10C59000030C8B4202D31212090265D0030B8B42AB
:10C5A00019D300E0090AC30B8B4201D3CB03C01A95
:10C5B0005241830B8B4201D38B03C01A5241430B70
:10C5C0008B4201D34B03C01A5241030B8B4201D360
:10C5D0000B03C01A5241C30A8B4201D3CB02C01ACB
:10C5E0005241830A8B4201D38B02C01A5241430A43
:10C5F0008B4201D34B02C01A5241030A8B4201D332
:10C600000B02C01A5241CDD2C3098B4201D3CB01D8
:10C61000C01A524183098B4201D38B01C01A524187
:10C6200043098B4201D34B01C01A524103098B428B
:10C6300001D30B01C01A5241C3088B4201D3CB0076
:10C64000C01A524183088B4201D38B00C01A524159
:10C6500043088B4201D34B00C01A5241411A00D209
:10C6600001465241104670475DE0CA0F00D0494272
:10C67000031000D34042534000229C4603098B42E2
:10C680002DD3030A8B4212D3FC22890112BA030A6A
:10C690008B420CD3890192118B4208D389019211EC
:10C6A0008B4204D389013AD0921100E08909C30971
:10C6B0008B4201D3CB01C01A524183098B4201D373
:10C6C0008B01C01A524143098B4201D34B01C01A5E
:10C6D000524103098B4201D30B01C01A5241C308D6
:10C6E0008B4201D3CB00C01A524183088B4201D345
:10C6F0008B00C01A5241D9D243088B4201D34B0060
:10C70000C01A5241411A00D20146634652415B10A1
:10C71000104601D34042002B00D549427047634682
:10C720005B1000D3404201B50020FFF7ADFD02BD14
:10C730000029F8D016E7704702B47146490849004D
:10C74000095C49008E4402BC7047C0468446101CF8
:10C7500062468C46191C634600E0C0461FB501F0D6
:10C760003FFC002801D40021C8421FBD10B501F0D4
:10C7700097FB4042013010BD10B501F031FC00289C
:10C7800001DB002010BD012010BDC04610B501F036
:10C7900027FC002801DD002010BD012010BDC0468F
:10C7A00010B501F0B9FB002801DC002010BD01200C
:10C7B00010BDC04610B501F0AFFB002801DA002023
:10C7C00010BD012010BDC046F0B5DE4657464E46AE
:10C7D00045469446E0B595B09B461E9B65469946F6
:10C7E0001F9B04009846209B60460293219B029A5F
:10C7F0009A46594653460A9501F05AFC239F229EB9
:10C800000490059132003B004846414603960B9741
:10C8100001F04EFC3D0006000F00039A2B000A9821
:10C8200059460C960D9701F043FC4A460690079135
:10C8300043460298514601F03BFC32003B00089011
:10C8400009910498059901F0A5FE089A099B060034
:10C850000F000698079900F005FD32000090019145
:10C860003B0030003900FFF781FF00280DD0009A0F
:10C87000019B200026606760A260E36015B03CBCAD
:10C8800090469946A246AB46F0BD00980199020039
:10C890000B00FFF76BFF0028E9D10A995B468C4635
:10C8A0000A0060465946654601F074FE4A461090FB
:10C8B000119143464846414601F06CFE0B000200D0
:10C8C000FFF754FF3822434258416B469B181870BB
:10C8D0004A46434641464846FFF748FF3822431E32
:10C8E00098416B469B181B782A0003400E93280042
:10C8F0005B465946FFF73AFF002800D123E1109824
:10C90000119902000B00FFF731FF002800D01AE157
:10C9100059460022D34B002900DAD34B9B460E9B8D
:10C920000A925A425341D14A5B421340CD4A94463F
:10C930006344424600215B00D20FD2075B081343D9
:10C9400089469846029A534602985146FFF70EFFD1
:10C95000002800D168E10B99039D8C460B002A004A
:10C9600028006146FFF702FF002800D150E10123B3
:10C970000E93029A53460298514601F00BFE129014
:10C9800013910B99039D8C462A000B0028006146E9
:10C99000654601F0FFFD0B000200FFF7E7FE4022B5
:10C9A000434258416B469B181870039A2B0029008C
:10C9B0000398FFF7DBFE4022431E98416B469B180D
:10C9C0001B78029A03401093029853465146FFF792
:10C9D000CDFE002868D01298139902000B00FFF7D3
:10C9E000C5FE002860D1524600259E4B002A00DA81
:10C9F0009D4B9A46109B9D4A013B1340994A0295D4
:10CA0000944663440B9A5B00D70F00220A9E5B0892
:10CA1000FF073B4303920B9332005B4630005946BD
:10CA2000FFF7A4FE002800D138E14A4643464846B5
:10CA30004146FFF79BFE002800D125E1029A5346AC
:10CA40000A98594601F034FB0B9D06000F00039A2B
:10CA50002B004846414601F02BFB02000B00300042
:10CA6000390001F097FD0022814B01F021FB039A70
:10CA70002B0006000F000A98594601F019FB029A94
:10CA80000090019153464846414601F011FB0200D7
:10CA90000B000098019900F0E5FB0022744B01F0B7
:10CAA00007FB00900191E2E6109B002B00D0A4E070
:10CAB0000E9B002BC2D10498059902000B0001F0D7
:10CAC00069FD0E900F910498059902000B00FFF785
:10CAD0004DFE002846D00E980F9902000B00FFF77C
:10CAE00045FE00283ED10A9E5B4632003000594682
:10CAF000FFF73CFE002800D1A0E04A4643464846E6
:10CB00004146FFF733FE002800D1B3E0029A5346B6
:10CB100002985146FFF72AFE002800D198E0039FB3
:10CB20000B9E3A00330038003100FFF71FFE00284B
:10CB300084D100220B991300914201DA80231B0655
:10CB400003920B937AE70E9B002B00D111E7002292
:10CB500059461300914201DA80231B069B460A9234
:10CB6000404BE6E60C980D9902000B0001F012FD17
:10CB7000049005910C980D9902000B00FFF7F6FD4B
:10CB8000002807D00498059902000B00FFF7EEFD7E
:10CB90000028A8D00698079902000B0001F0FAFCC3
:10CBA000049005910698079902000B00FFF7DEFD3F
:10CBB000002807D00498059902000B00FFF7D6FD66
:10CBC000002890D00898099902000B0001F0E2FCBF
:10CBD000049005910898099902000B00FFF7C6FD23
:10CBE000002800D143E60498059902000B00FFF7E6
:10CBF000BDFD002800D03AE675E7002552462B001F
:10CC0000AA4201DA80231B069A460295154BF9E6E3
:10CC100000220B991300914201DA80231B060B932B
:10CC2000012303920E93A4E652464D464B464A45D5
:10CC300001DA80231B0602959A468CE600265A46A6
:10CC40003300B24201DA80231B060A969B4654E762
:10CC5000002552462B00AA4201DA80231B060295CA
:10CC60009A465CE70000F03F0000F0BF000010C0F3
:10CC70000000F07F002241461300914201DA802338
:10CC80001B069146984641E7002241461300914217
:10CC900001DA80231B0691469846CFE600265A46C5
:10CCA0003300B24201DA80231B060A969B46BCE69B
:10CCB000F0B557464E464546DE46E0B58BB0169970
:10CCC000824689461799189888461999149E8B466A
:10CCD00041464C005946159F4900019203930500B7
:10CCE000059002004B084846610802960497FFF73A
:10CCF00043FD00284BD02A005B4648464146059537
:10CD000000F0CCFD04000D0002000B004846414637
:10CD100001F0CEF9059A5B4600F0A4FA22000690D5
:10CD200007912B000198039901F0C2F932003B00F2
:10CD30000296049700F096FA069A079B00F0AEFD63
:10CD400022002B0006000F000298049901F0B0F9B0
:10CD5000019A039B01F01EFC069A079B00F09EFDC2
:10CD6000320004000D003B0030003900FFF7FEFCEC
:10CD700000283ED0534650461E605F609C60DD60D8
:10CD80000BB03CBC90469946A246AB46F0BD059E12
:10CD90004A4643463000594600F080FD04000D002D
:10CDA00002000B003000594601F082F94A46434622
:10CDB00000F058FA06000F00029A049B2000290098
:10CDC00001F076F9019A039B00F04CFA32003B0027
:10CDD0000696079700F062FD019A039B06000F007C
:10CDE0002000290001F064F902000B000298049968
:10CDF000B0E722002B0020002900FFF7B7FC002835
:10CE0000B8D10022002348464146FFF7AFFC002876
:10CE100028D00022002305985946FFF7A7FC0028D8
:10CE200020D00399019A0B000198FFF79FFC00287E
:10CE300000D176E143460024DE4D002B01DA0024C8
:10CE4000DD4D019A039B2000290001F031F9029A7F
:10CE500006000F0020002900049B01F029F90400BE
:10CE60000D0087E7019803990690079102000B00D7
:10CE70000698079901F08EFB089009910399019A91
:10CE80000B000198FFF772FC00287ED008980999E2
:10CE900002000B00FFF76AFC002876D14A464346A1
:10CEA0004846414601F076FB02000B00FFF75EFCAE
:10CEB000002800D146E105995B460A000800594662
:10CEC00001F068FB02000B00FFF750FC002800D1C6
:10CED00095E0BA4B039A029FD20F049ED2071343E8
:10CEE00001933A0033003800310001F053FB3A005F
:10CEF00004000D00330038003100FFF737FC002834
:10CF000000D153E122002B0020002900FFF72EFC66
:10CF1000002800D04AE1A94C049B0022DB0FDB076C
:10CF20001C434846019B414601F0C2F8230006001D
:10CF30000F0000220598594601F0BAF802000B00D4
:10CF40003000390000F08EF900229A4B01F0B0F861
:10CF50002300002206000F004846414601F0A8F8D1
:10CF6000002204000D00019B0598594601F0A0F82D
:10CF700002000B002000290001F00CFB00228D4B69
:10CF800001F096F804000D00F4E60298049906906A
:10CF9000079102000B000698079901F0FBFA069032
:10CFA00007910499029A0B000298FFF7DFFB002813
:10CFB00000D1C7E00698079902000B00FFF7D6FBE7
:10CFC000002800D0BEE04A4643464846414601F0AC
:10CFD000E1FA02000B00FFF7C9FB002800D1B1E025
:10CFE00005995B460A000800594601F0D3FA0B0088
:10CFF0000200FFF7BBFB0023984200D06AE70599C7
:10D000005B4689460A000800594601F0C3FA4A46C1
:10D01000069007915B4648465946FFF7A7FB002854
:10D0200000D1A7E60698079902000B00FFF79EFBC8
:10D03000002800D09EE60898099902000B00FFF72F
:10D0400095FB002800D195E6029989460A000499CB
:10D0500048460B0001F09EFA0B000200FFF786FB2A
:10D060000023984200D185E64246D70F059EFF0770
:10D070003B433200994630005B46594601F08AFA3C
:10D08000320004000D005B4630005946FFF76EFB8E
:10D09000002800D18CE022002B0020002900FFF79F
:10D0A00065FB002800D083E0444E5B46DB0FDB07C6
:10D0B0001E4300224B460198039900F0F9FFB04649
:10D0C0003300049E04000D0000223100029800F09D
:10D0D000EFFF02000B002000290000F0C3F800223F
:10D0E000002300F0E5FFB34600224B4606000F0088
:10D0F0000298594600F0DCFF002204000D00434670
:10D100000198039900F0D4FF02000B0020002900D1
:10D1100001F040FA0022002300F0CAFF04000D00D5
:10D1200028E60499029A0B000298FFF71FFB0028DB
:10D1300000D07FE60399019A0B00019801F02AFACA
:10D14000089009914A4643464846414601F022FA72
:10D150004A4606900791434648464146FFF706FB7C
:10D16000002800D14BE70698079902000B00FFF753
:10D17000FDFA002800D042E70898099902000B0048
:10D18000FFF7F4FA002800D1F4E5029989460A0075
:10D19000049948460B0001F0FDF902000B00FFF76F
:10D1A000E5FA002800D1E5E5044B5DE70024B3E68D
:10D1B00000267AE70000F07F0000F0FF0000F03F5B
:10D1C00070B500220C4B04000D00FFF7F3FA0028A5
:10D1D00004D12000290001F025FD70BD064B00227E
:10D1E0002000290001F0D6F901F01CFD80231B0668
:10D1F0009C466044F1E7C0460000E04170B5002263
:10D200000B4B0D00040000F053FFFFF7D9FF0600A1
:10D2100001F078FD0022074B00F04AFF02000B00EE
:10D220002000290001F0B6F9FFF7CAFF310070BDF8
:10D230000000F03D0000F04170B50600080001F06C
:10D2400061FD0022064B00F033FF0D0004003000AA
:10D2500001F058FD2B00220000F004F870BDC0461C
:10D260000000F041F0B54F464646D6460C00090393
:10D27000C0B5490A470F5E0039431F03DB0F9C46C8
:10D2800065007B0A570F1F436D0DE40F760DA14615
:10D29000C000B846D200AB1B64457BD0002B5FDDDD
:10D2A000002E00D0A4E03E00164300D112E15E1E25
:10D2B000002E00D09EE1871A4346B84280410125E6
:10D2C000C91A4042091A0B0200D431E149024E0A40
:10D2D000002E00D16EE13000FFF7C6F80300083BD6
:10D2E0001F2B00DD61E120223900D21A9E40D1407F
:10D2F0009F400E439D4200DD51E15D1B6B1C1F2BC7
:10D3000000DD7CE12021C91A3D0030008F408840BB
:10D31000DD40791E8F41310007222843D940002586
:10D3200007433A40002A09D00F233B40042B05D085
:10D330003B1DBB42BF417F42C9191F000B0200D4F5
:10D3400026E26A1CC64B55056D0D9A4200D106E1D6
:10D35000C44AFF080A40530752023B43120B8EE0B7
:10D36000002B00D0B8E06B1C5B055B0D012B00DCD3
:10D3700030E1871A4346B842B641CB1A76429E1B2B
:10D38000330200D54CE13B003343A1D100220024FD
:10D39000002570E0002B00DCE5E0002E00D183E0EA
:10D3A000AF4EB54260D0802636043743B846382B9E
:10D3B00000DC3EE1434613431F007A1E97413F18AD
:10D3C00087428041404209180B0200D4B0E0A44BD0
:10D3D00001359D4200D1C3E0A24A7B080A400121E9
:10D3E0000F401F435108D30707221F433A4099E7D4
:10D3F0009B4EB54238D0802636043743B846382B8A
:10D4000000DDDCE01F2B00DC30E11E004746203E43
:10D41000F740BC46202B04D04026F31A46469E40D7
:10D420003243170063467A1E97411F43CCE0002B1E
:10D4300000D104E24346134300D159E14B07C00831
:10D4400018438023C9081B03194208D04546ED083C
:10D450001D4204D14346D008590708432900420F12
:10D46000C9007F4D1143C0004B07CA087C49C00862
:10D4700003438D4268D012036D05120B6D0D002120
:10D4800012031800130B0A0D12051A43764B2D05D3
:10D4900013402B435B00E4075B08234319001CBCCB
:10D4A00090469946A246F0BD3E00164312D05E1E3D
:10D4B000002E00D000E1871887428041414440425D
:10D4C000091801250B0233D5022585E76446330090
:10D4D000414610001D00C7E7002D00D0DAE00C0027
:10D4E0000443F3D05C1C00D19FE15D4CA64200D107
:10D4F0002FE1DB43382B00DD66E11F2B00DD83E1EC
:10D5000020240500E41A0F00DD40D940A040434626
:10D51000A7405B1A441EA04198462F433843171A70
:10D52000BA42924143465242991A64463500CAE6CD
:10D5300007223A40002A00D0F6E64B07CA084849BD
:10D54000FF083B438D4296D11900114300D19EE163
:10D55000802109030A431203120B414D8FE7150086
:10D56000002200238BE7002B00D0C7E06B1C5F0577
:10D570007F0D012F00DCF1E0394DAB4200D1B9E065
:10D5800085180A00854289414244494251180722C0
:10D59000CF076D082F4349083A401D00C2E6072215
:10D5A0003049ED1A31403A40BCE63E00283886400A
:10D5B00000279FE63800FEF757FF20308EE64346EF
:10D5C00013431F007A1E9741C71BB8428041404257
:10D5D000091A78E60E003B0006431343002D61D183
:10D5E000002E00D0F4E0002B00D11BE1644639008E
:10D5F000100039E71A4FBB427AD03300FFE6300003
:10D600001F3DE840202B03D04021CB1A9E403743DA
:10D610007B1E9F41072207433A400021002589E7EE
:10D62000171A4346BA42B641591A76428E1B6446CF
:10D630004EE61F2B00DDADE020264746F61AB74028
:10D64000B9461700B246DF404E463E4337005646C5
:10D65000B240561EB24117434246DA408918AEE640
:10D66000FF070000FFFF7FFFFFFF0F8020264746D8
:10D67000F61AB740B9461700B246DF404E463E4361
:10D6800037005646B240561EB24117434246DA4072
:10D69000891A99E77F4CA6425BD0802424045B4220
:10D6A000214327E7002E0CD1002B00D1CBE06446AC
:10D6B00039001000774DD7E6764FBB4218D03300C3
:10D6C00075E6002B14D04B07C00818438023C90807
:10D6D0001B03194207D0FC081C4204D17907D0086B
:10D6E0000843E14621004C46420FC9001143C000E7
:10D6F000684DB9E61D0000220023C0E6002D5BD175
:10D700000D00054300D1E2E65D1C00D1B0E0614DA3
:10D71000AE421FD0DB43382B71DC1F2B00DD96E0BF
:10D7200020250F00ED1AAF40B9460700AA46DF409A
:10D730004D463D432F005546A840D940451EA841BF
:10D7400088440743BF1897429241514241443500F3
:10D750003AE6644635004146100085E60B00034377
:10D76000002D00D063E6002BF5D04346134300D1D3
:10D770007AE68718874280410722414440420918CF
:10D780003A400B0200D4D5E6434B01351940C9E5B8
:10D79000380069E61E004746203EF740BC46202B75
:10D7A00004D04026F31A46469E4032431700634693
:10D7B0007A1E97411F4302E6364DAE42CAD08025FD
:10D7C0002D045B422943A6E70843411E8841A6E693
:10D7D000002B00D148E6871A4346B842B641CB1A1F
:10D7E00076429E1B33024BD5171A4346BA429241EA
:10D7F000591A5242891A072264463A4092E5014377
:10D800000F00791E8F419DE71C000F00203CE74070
:10D81000202B03D04024E31A99400843411E88413D
:10D8200038437CE60022002425E6171A4346BA4214
:10D830009241591A5242891A6446350043E54146DD
:10D840001000144D10E680220024120380E61D0013
:10D850000F00203DEF40BC46202B03D04025EB1AA3
:10D860009940084307006346781E87411F4369E7D4
:10D87000871897429B4141445B42C9183500A3E594
:10D880003B003343CED0072231003A4052E600231A
:10D890001A00F4E5FF070000FFFF7FFFF0B55746D1
:10D8A000DE464E464546E0B5834607000E03480077
:10D8B00085B092461C00360B400DCD0F002800D1DC
:10D8C0009DE0954B984239D08023F6001B041E43FF
:10D8D000924A7B0F33439946944603006344009376
:10D8E00000230026FF00029323031B0B98466300CE
:10D8F000E40F52465B0D019400D1B3E086498B42A0
:10D9000000D19EE04246D100802212040A435146D3
:10D91000490F11438B46814952468C460099634416
:10D92000CB1A0021D20000932B0063409A460F2EA1
:10D9300000D905E17A4BB6009B599F465B463343BD
:10D94000994600D0B8E002230826002700900293F1
:10D95000CAE7CB463A0002990195019B9A460229F3
:10D9600027D0032900D180E2012944D06D49009BD2
:10D970008C4663441C00002C38DD530700D013E2B2
:10D98000D2085B46DB0109D55946674B19408B46E7
:10D990008021C9008C46009B63441C00634B9C4261
:10D9A00007DC5B4664055F075B0217431B0B620DD8
:10D9B00002E000230027584A00211B031C0B0B0D1B
:10D9C0001B05234314055A4A380013401C43534691
:10D9D0006400DB0764081C43210005B03CBC904692
:10D9E0009946A246AB46F0BD0122524201231B1BC1
:10D9F000382B00DCADE1002200230027DCE75B468A
:10DA0000334399465ED0002E00D18AE13000FEF704
:10DA10002BFD03000B3B1C2B00DD7BE11D22D31AE9
:10DA20005A460100DA4008398E4013005F463343FE
:10DA300099468F403F4B00261B1A00930023029308
:10DA400052E7414653460B433B499B468C46009B5D
:10DA5000634400935B46002B3BD1022300221E430C
:10DA6000022161E7434613439B4637D04346002BD0
:10DA700000D162E14046FEF7F7FC03000B3B1C2B94
:10DA800000DD53E102004146083A914088461D21DD
:10DA9000CB1A5146D9400B0041460B439B46534697
:10DAA00093401A00009B25499C46604403008C4625
:10DAB00063440093002137E70323B14600900C260E
:10DAC000029311E7002300930133042600270293F9
:10DAD0000AE70323C3461E43032125E701331E4300
:10DAE0000022012120E700239A46802300271B0300
:10DAF000094A61E7802349461B03194200D1E2E04D
:10DB00005946194200D0DEE00B431B0317001B0BE4
:10DB1000A246014A50E7C046FF07000001FCFFFF94
:10DB200044FB0000FF030000FFFFFFFEFE070000B4
:10DB3000FFFF0F800DFCFFFF01F8FFFFF303000064
:10DB4000D94500D9CBE000D1C6E03C0048460027CB
:10DB5000009B013B00935B46160E1B021E43130203
:10DB6000984633041B0C9946310C0191FEF788FB53
:10DB70004A4642430B04210C050019438A4207D947
:10DB80008919013D8E4203D88A4201D9851E89191F
:10DB9000881A0199FEF774FB09048C464A46210451
:10DBA00064464243090C030021438A4204D989197F
:10DBB000013B8E4200D8F1E02D041D43AB464346A5
:10DBC000891A4246280C12041D0C5B46140C2200D4
:10DBD0001B041B0C5A4303946B4344430295684354
:10DBE0001B19150CEB189C4203D980246402A4462F
:10DBF00060441C0C15041B042D0C20185D19814277
:10DC000077D373D00C1AA24A7D1BAF42BF41944612
:10DC1000009B7F426344E01B1C00864200D1DBE096
:10DC20000199FEF72DFB4A4642430B04290C0700DD
:10DC300019438A4207D98919013F8E4203D88A4283
:10DC400001D9871E8919881A0199FEF719FB090461
:10DC50004A46894629044D464243090C030029439C
:10DC60008A4207D98919013B8E4203D88A4201D9D9
:10DC7000831E89193F04891A3A00039F1A4338000A
:10DC800013041B0C584381460298150C6F43434301
:10DC900045434846000C8446DB1963449F4203D940
:10DCA000802040028446654448461F0C00041B0443
:10DCB000000C7D191818A94200D284E000D17FE041
:10DCC00001231A4357E680234A461B0313431B03D1
:10DCD0001B0BAA466F4A6FE6BA4200D935E74B469E
:10DCE000DC0758087B081C43FF0734E70024AF42D9
:10DCF00089D247444745A4415B466442A41964184D
:10DD0000013BA6421ED2A0426DD800D1B6E0241A33
:10DD10009B4678E703005A46283B9A4000279146E5
:10DD200088E65846FEF7A0FB203072E60300524614
:10DD3000283B9A4093460022B4E65046FEF794FBF7
:10DD400020309AE6A642E2D1B845DCD9341A9B4687
:10DD500059E71F2B65DC504C0099A4465C46614492
:10DD600008008C4011008240D940501E82410C4373
:10DD700014435A46DA401300620709D00F222240AA
:10DD8000042A05D02200141D9442894149425B189F
:10DD90001A0262D50122002300270DE68A4200D82C
:10DDA0000AE7831E891907E70F231340042B00D1CC
:10DDB000E6E5171D9742924153429B44FA08E0E57D
:10DDC000002800D1D7E57118531EB14227D3A942CC
:10DDD00015D358D01A0073E7002B00DC04E60123AA
:10DDE00000229B44CDE502234744474589415B42DD
:10DDF0009C46494289190C19E344241A03E7434617
:10DE00005F0047459B41B8465B429E19023A89191B
:10DE1000A94200D054E7404500D051E7ABE51A00D5
:10DE2000F6E71F215F4649420C1BE740202B07D035
:10DE30001A49009B8C46634418005B4683401A4392
:10DE4000501E82413A4307270023174009D00F2173
:10DE5000002311401400042995D122005F075B02C2
:10DE60001B0BD20817430022A6E5802359461B034B
:10DE70000B431B0317001B0B064A9DE5BD42B2D89E
:10DE80009B460024BFE68045B9D31A00C3E7C046CD
:10DE9000FF030000FF0700001E0400003E04000016
:10DEA000F0B54F464646D6468446C0B58046194E24
:10DEB00018030F034D00000B5C0082463F0B6D0DF5
:10DEC000C90F9146640DDB0F0120B5420AD0B44260
:10DED00003D0A54201D157450CD01CBC90469946B1
:10DEE000A246F0BD66463E43F7D1AC42F5D154465A
:10DEF0001443F2D10120C845EFD1994207D0002D3B
:10DF0000EBD163461F433800471EB841E5E70020C8
:10DF1000E3E7C046FF070000F0B54F464646D64649
:10DF20004D00C0B50E03C90F8A462C491F035C0083
:10DF30008046360B6D0D91463F0B640DDB0F8D4215
:10DF40001ED08C4216D0002D1ED130438446002CAA
:10DF500001D13A4323D06246002A1AD09A4529D0EB
:10DF6000514602200139084001381CBC90469946B0
:10DF7000A246F0BD39001143E5D002204042F4E74B
:10DF80003043FAD1AC420FD0002C0FD13A43E7D046
:10DF90000CE00122013B934318000130E5E76346A2
:10DFA0000020002BE1D0DBE73A43E6D19A45D7D1F8
:10DFB000A542D5DCA54205DBBE42D1D808D0002061
:10DFC000BE42D2D250460123013898430130CCE7FB
:10DFD000C845C5D80020C845F4D3C6E7FF070000F0
:10DFE000F0B54F464646D6464D00C0B50E03C90FA4
:10DFF0008A462E491F035C008046360B6D0D914604
:10E000003F0B640DDB0F8D4218D08C4211D0002DD8
:10E0100018D130438446002C1ED13A431CD16346AC
:10E020000020002B30D05146022001390840013831
:10E030002AE039001143EAD0022025E03043FBD129
:10E04000AC4226D0002C26D13A4324D1514602209E
:10E0500001390840013817E06246002A0FD09A457E
:10E06000E1D1A54205DBBE42DDD819D00020BE4279
:10E070000AD25046012301389843013004E00122BE
:10E08000013B9343180001301CBC90469946A246C0
:10E09000F0BD3A43D0D19A45C5D1A542C3DCE0E7F3
:10E0A000C845C0D80020C845E3D3EDE7FF0700000E
:10E0B000F0B55746DE464E464546E0B58346060077
:10E0C0000F03480087B092461D003F0B400DCC0F58
:10E0D000002800D16FE0DE4B984238D08023FF004B
:10E0E0001B041F43730F3B430193DA4B00279946F0
:10E0F00000239B46F60081442B0369001B0B52460C
:10E100009846490DED0F002900D185E0D04B99428A
:10E1100000D173E04346DA0080231B0413435246C8
:10E12000CC48520F84461343524600206144D2002B
:10E1300089442100694000918C46012149448A4666
:10E140000F2F00D990E0C449BF00CF59BF465B46AE
:10E150003B43019300D06AE1022308270026814651
:10E160009B46C9E732005846019B61460091022850
:10E1700000D175E0032800D1FEE1012800D02CE198
:10E1800000230027002600253F032A0D3F0BB3483C
:10E1900012053A4302401B051343009A5B00D10766
:10E1A0005B080B433000190007B03CBC9046994611
:10E1B000A246AB46F0BD5B463B43019300D12FE145
:10E1C000002F00D1A5E13800FEF74EF903000B3B0C
:10E1D0001C2B00DD96E11D22D31A5A460100DA40BD
:10E1E0005E4608398F4013008E403B4301939C4BA1
:10E1F00000271B1A994600239B467DE7414653465C
:10E200000B4393498C46E144002B00D01AE10222D3
:10E210000220174300228CE7134300D10DE143464F
:10E22000002B00D181E14046FEF71EF902000B3AB7
:10E230001C2A00DD72E10100434608398B409846F4
:10E240001D239A1A5346D3401A004346134352469D
:10E250008A404946081A824989468144002068E775
:10E260007B4B002700268EE7140C1204120C1100C1
:10E27000370C3604350C794328008C462E00604359
:10E280006044834656432100300C8046584679430B
:10E2900040440291844506D98846802149028C4633
:10E2A000E044414602913604010C360C00048B46D2
:10E2B00081191E0C1B041B0C0391190079438C4619
:10E2C000280075436544A8465843050C45447743E8
:10E2D000A94203D9802149028C466744290C8C4607
:10E2E00039000004000C2D042D186144AB44059145
:10E2F0005946049101990F043F0C080C3900514311
:10E300004243904602008C46090C8B4662437C4394
:10E3100044445C44A04503D98021490288464244D4
:10E32000210C884661460904090C8C463900594382
:10E33000434370437E430F0CF6182404BE19644413
:10E3400042448C46B34203D980235B029846404442
:10E35000029B61469846049B370443449B46AB4569
:10E36000AD416B420D0405992D0C8C467F19674415
:10E37000FD18A8465D462D19A542A4419346644266
:10E38000A446C344DC448F42BF4198459B4193451A
:10E390009241A445A4415B427F421F43360C524246
:10E3A0006442BF192243BF18624638184302D20D97
:10E3B000039913436A020A43501E82416146ED0DE0
:10E3C0002A434E023243D90100D4B3E0012650085B
:10E3D00032400243DE0732435B08224C5444002C97
:10E3E00062DD510709D00F201040042805D0101D10
:10E3F0009042924152429B180200D90104D58024D8
:10E400001948E400034054441848844200DD27E7DB
:10E410005E075B02D2081F0B630516435B0DB2E675
:10E42000002399460133042700269B4664E6032314
:10E43000019781460C279B465EE601220120174387
:10E44000002276E6032303201F43434671E6C046BD
:10E45000FF07000001FCFFFF84FB0000FFFF0F80AF
:10E460000DFCFFFFFF030000FFFFFFFEFE070000A3
:10E470000023802700933F030026434B83E6019B44
:10E480003200A446584670E6AC466EE680270199F5
:10E490003F0339422DD03B422BD11F433F033F0B5B
:10E4A00000951600384B6EE601252D1B382D00DD3A
:10E4B00066E61F2D40DC35481C00504416008240A3
:10E4C0008440EE40501E824134431443EB406207C7
:10E4D00009D00F222240042A05D02200141D9442A4
:10E4E000804140421B181A023ED501230027002616
:10E4F00049E68027019B3F031F433F033F0B0094E6
:10E50000214B40E603005A46283B9A4000260192E0
:10E510006DE65846FDF7A8FF203057E60300524647
:10E52000283B9A401300002293E65046FDF79CFFDB
:10E5300020307BE6CA4650E71F201E004042041BE5
:10E54000E640202D03D0124C5444A3401A43501EE1
:10E550008241324307260027164009D00F200023AE
:10E56000104014000428B9D122005E075B021F0B83
:10E57000D2081643002306E680273F031F433F03CC
:10E580003F0B1600004BFEE5FF0700001E040000D5
:10E590003E040000F8B557464E464546DE460C00A0
:10E5A0000903E0B5490A460F5F0031431E03DB0F44
:10E5B000760A9B46530F3343C84E6500C000E40FF4
:10E5C000D2006D0DA24681467F0D9C469046B74213
:10E5D00000D1B9E05B46012673409B46EE1BA34584
:10E5E00000D183E0002E63DD002F00D0B1E0634650
:10E5F000134300D123E1731E002B00D0BAE1861A29
:10E600006346B04280410125C91A4042091A0B02F3
:10E6100000D447E149024B0A98464346002B00D1FB
:10E6200089E14046FDF720FF0300083B1F2B00DD7A
:10E630007CE120223000D21A4146D04099400200AD
:10E640009E400A439D4200DD6AE15D1B6B1C1F2B4F
:10E6500000DD94E1202110003500C91A8E40DA4017
:10E660008840DD40711E8E4111000722284300259D
:10E6700006433240002A09D00F233340042B05D033
:10E68000331DB342B641764289191E000B0200D4F5
:10E690003DE26A1C914B55056D0D9A4200D119E17E
:10E6A0008F4AF6080A40570752023743120B9BE085
:10E6B000002E00D0C5E06E1C7605760D012E00DC24
:10E6C00048E16746861ACB1BB042BF417F42B8463D
:10E6D0001F004346FF1A3B00B8461B0200D55FE10E
:10E6E00037439AD100220024002579E0002E00DC77
:10E6F000FAE0002F00D18DE0784B9D4267D0802357
:10E7000067461B041F43BC46382E00DC52E16346BB
:10E7100013435A1E93411E188642804140420918F5
:10E720000B0200D4BEE06D4B01359D4200D1D2E01A
:10E730006B4A73080A4001210E401E435108D3075B
:10E7400007221E43324095E71E00164300D045E7DE
:10E7500040E7624B9D423AD0802367461B041F432B
:10E76000BC46382E00DDEBE01F2E00DC3AE1330022
:10E770006746203BDF403B00202E05D04027BF1BD3
:10E780006646BE40324390464646721E964133432B
:10E79000DAE0002B00D114E26346134300D168E1B4
:10E7A00080234E07C008C9081B030643194208D03E
:10E7B0006046C008184204D163460100D2085E07D3
:10E7C0001643F3009946C900720F444D11434B465E
:10E7D000DE08424B4F073743CA089D4200D16EE026
:10E7E00012036D05120B6D0D00211203130B0A0DA0
:10E7F00012051A433B4B2D0513402B435B00E407E6
:10E800005B082343380019003CBC90469946A24659
:10E81000AB46F8BD6346134311D0731E002B00D0E6
:10E8200007E186188642804161444042091801256B
:10E830000B0237D502257BE73E0061469146350045
:10E84000C5E75C46002D00D0E1E00B000343F3D0A8
:10E85000731C00D1ACE1214B9F4200D13AE1F3435C
:10E86000382B00DD6FE11F2B00DD8CE120250E0031
:10E87000ED1AAE40B0460600AA46DE404546354396
:10E880002E005546D940A8406346451EA8415B1A54
:10E890009C463043161AB242924163465242991A3C
:10E8A0003D00B4E607223240002A00D0E4E60B4BDC
:10E8B000F6084F073743CA089D4200D090E73B0057
:10E8C000134300D1A6E180231B031A431203120B4A
:10E8D000024D89E715000022002785E7FF070000A9
:10E8E000FFFF7FFFFFFF0F80002E00D0C7E06B1CF3
:10E8F0005E05760D012E00DCF0E0C84DAB4200D184
:10E90000B9E085180A00854289416244494251189C
:10E910000722CE076D082E43490832401D00A9E6A4
:10E92000BF49ED1A114007223240A3E632002838D1
:10E930008240002686E63000FDF796FD203073E623
:10E94000634613435A1E9341C61AB0428041404267
:10E95000091A5CE60E00674606431743002D5ED198
:10E96000002E00D0F3E0002F00D11EE15C4661468E
:10E9700091462CE7A94FBE427BD01E00F1E6100065
:10E980001F3DE840202B03D04021CB1A9A4016436C
:10E99000731E9E410722064332400021002583E773
:10E9A000161A6346B2428041591A40420B1A9846E1
:10E9B0005C4632E61F2E00DDABE02027BB1B9A46EB
:10E9C00063465746BB40994613004F46F3401F43EA
:10E9D0003B005746BA40571EBA4113436246F240C5
:10E9E000891898E62027BB1B9A4663465746BB40CA
:10E9F000994613004F46F3401F433B005746BA4029
:10EA0000571EBA4113436246F240891A9CE7834B72
:10EA10009F425FD080252D047342294320E7002EBA
:10EA20000CD1002F00D1D0E05C46614691467B4D71
:10EA3000CDE67A4FBE421CD01E0065E6002F18D0EE
:10EA4000C0084E0706438020C9080003014208D0D1
:10EA50006346DC08044204D12100DA46D2085E078E
:10EA60001643F300994601245346C900720F11431F
:10EA70001C406A4DABE61D0000220027B4E6002DC5
:10EA800059D10B00034300D1D6E6731C00D1B2E08C
:10EA9000624B9F421ED0F343382B6FDC1F2B00DDEF
:10EAA00097E020250E00ED1AAE40B0460600AA46BB
:10EAB000DE40454635432E005546A840D940451E08
:10EAC000A8418C440643B618964292415142614493
:10EAD0003D0025E63D006146914678E60B00034384
:10EAE000002D00D055E6002BF5D06346134300D12E
:10EAF0006DE6861886428041614440420918002232
:10EB00000B0200D4D0E6464B01351940B2E5B146C0
:10EB10005DE633006746203BDF403B00202E05D0FA
:10EB20004027BF1B6646BE40324390464646721E93
:10EB300096413343EFE5394B9F42CBD080252D04DE
:10EB400073422943A8E70843411E8841A2E6002FEB
:10EB500000D13CE66346861ACF1AB0429B415B4225
:10EB6000FB1A98461B024ED5161A6346B2429241D2
:10EB7000591A5242891A5C4600227BE501430E0075
:10EB8000711E8E419FE71D000E00203DEE40B046F5
:10EB9000202B04D04025EB1A994008438146484673
:10EBA0004346411E8841184374E60022002417E6BC
:10EBB000161A6346B2429241591A5242891A3D00CE
:10EBC00025E561469146154D01E680220024120399
:10EBD00079E61D000E00203DEE40B046202B04D00B
:10EBE0004025EB1A9940084381464E464346711E24
:10EBF0008E411E4367E7861896429B4161445B4203
:10EC0000C9183D008CE547463743CED00722414620
:10EC1000324049E600273A00E6E5C046FF0700001B
:10EC2000FFFF7FFF30B5144D0A034B00120B5B0D45
:10EC3000C90F0024AB4211DD104CA34210DC80242C
:10EC4000640322430E4CE41A1F2C0CDD0D48C31A3A
:10EC5000DA4013005C42002900D11C00200030BDC6
:10EC6000094BCC18FAE7094DE040AC4663449A40A2
:10EC700013000343EEE7C046FE0300001D0400003E
:10EC80003304000013040000FFFFFF7FEDFBFFFFD4
:10EC900070B500282DD0C317C5185D40C40F2800DB
:10ECA000FDF7E2FB154B1B1A5B055B0D0A2815DD12
:10ECB0000B38854000222D032D0B002110002D0361
:10ECC0000A0D2D0B12052A430D4D1B052A40134337
:10ECD0005B00E4075B082343190070BD02002900B4
:10ECE000153291400A000B21081AC5402D032D0B47
:10ECF000E3E70024002300250022DEE71E040000D5
:10ED0000FFFF0F8010B5041E25D0FDF7ADFB144B9F
:10ED10001B1A5B055B0D0A2812DD0B3884400022AC
:10ED20002403240B0021100024030A0D240B1205D8
:10ED300022430C4C1B05224013435B00590810BDB5
:10ED400002002100153291400A000B21081AC4402C
:10ED50002403240BE6E7002300240022E2E7C04658
:10ED60001E040000FFFF0F80A30000000000000051
:10ED7000FC3F0150FC3F0250FC3F0350008001501B
:10ED800000800250008003502024282C383C40444E
:10ED9000484C0207020802010003010903040204AF
:10EDA00002050305000600070008000A0100000034
:10EDB0000000E0FE422EE63F0000E0FE422EE6BFED
:10EDC000763C7935EF39EA3D763C7935EF39EABD65
:10EDD000000000000000E03F000000000000E0BF75
:10EDE00000000000000000000000000000000080A3
:10EDF00000000040FB21F93F000000002D44743E5C
:10EE0000000000809846F83C0000006051CC783B40
:10EE100000000080831BF0390000004020257A3874
:10EE2000000000802282E336000000001DF36935F7
:10EE3000000000000000F03F000000000000F83F6C
:10EE4000000000000000000006D0CF43EBFD4C3E68
:10EE500000000000000000000000004003B8E23F96
:10EE60004FBB610567ACDD3F182D4454FB21E93FE2
:10EE70009BF681D20B73EF3F182D4454FB21F93FD1
:10EE8000E2652F227F2B7A3C075C143326A6813C57
:10EE9000BDCBF07A8807703C075C143326A6913C02
:10EEA000000000000000F87F000000000000F07F7C
:10EEB0000000000000000000000000000000000052
:10EEC000010000000000F03F8A1EBD726654B6408B
:10EED0004E543EF2A6EFCCC078844D13BFE9CB4030
:10EEE0004FFA050429CCB8C06C5C8AE26E56944097
:10EEF000CC5CF6234F0B5BC0563BD76877D80440F9
:10EF0000AC5913DC0D687EBFA38C9F98E6E76C3E7E
:10EF10005610B1E5EB4731BE182D4454FB21094092
:10EF2000000000000000000000000000000024407D
:10EF3000000000000000000000000000FCFA0000DB
:10EF400002FB000008FB00000EFB000014FB0000A9
:10EF50001AFB000020FB000026FB00002CFB000039
:10EF600032FB000038FB00003EFB000006061038B4
:10EF70007C101010050554341C1615060611514A54
:10EF80002A2410060610242A4A5111080804423E79
:10EF900002023E42200505007F3E1C080303403E5E
:10EFA00001070760584641465860040463554941CB
:10EFB000020225520505080C7E0C08050510307E5E
:10EFC000301006061010107C381004040404000EE3
:10EFD000050560506844400505600060006000025F
:10EFE00001015F03030600060505147F147F140565
:10EFF00005042A7F2A1005052313086462050536D7
:10F000004951225001010602023E410202413E05E1
:10F01000054428102844050510107C1010020240F9
:10F020003005051010101010020260600303601814
:10F030000605053E5149453E050500427F40000555
:10F0400005625149494605052241494936050518D9
:10F0500014127F100505274545453905053C4A49E9
:10F060004930050501710905030505364949493649
:10F070000505064949291E020242000202402205F6
:10F08000050814142222050514141414140505226D
:10F09000221414080505020151090608083C02392A
:10F0A00045453D417E05057E0909097E05057F49E7
:10F0B00049493605053E4141412205057F4141222E
:10F0C0001C05057F4949494105057F0909090105D5
:10F0D000053E4141513205057F0808087F03034181
:10F0E0007F410505304040403F05057F081422411F
:10F0F00005057F4040404005057F020C027F050565
:10F100007F0408107F05053E4141413E05057F090A
:10F1100009090605053E4151215E05057F091929AA
:10F120004605052649494932050501017F010105CA
:10F13000053F4040403F0505071860180705057F5B
:10F140002018207F0505631408146305050304785F
:10F1500004030505615149454302027F410303064B
:10F1600018600202417F05050804020408050540F5
:10F170004040404002020204040420545478040435
:10F180007F44443804043844444404043844447FED
:10F190000404385454580303087C0A040418A4A433
:10F1A0007C04047F0404780303447D400202847DD0
:10F1B00004047C10284401017F05057C0438047C8C
:10F1C00004047C0404780404384444380404FC44F3
:10F1D00044380404384444FC04047C080404050551
:10F1E00008545454200303047E4404043C40407CEF
:10F1F00005050C3040300C05053C403C403C050505
:10F200004464384C4404041CA0A07C030364544CA4
:10F2100081F900000000000087F9000000000000F4
:10F220008BF900000000000090F9000094F9000044
:10F2300098F90000000000009CF900009FF9000010
:10F24000A3F900005BF80000A8F90000AEF9000087
:10F25000B2F900005FF8000000000000B6F90000FD
:10F26000BAF90000BEF90000BEF90000C4F90000C0
:10F27000C8F9000000FB0000CCF90000CEF9000046
:10F28000D0F90000ABF8000062FA0000D2F90000EB
:10F29000D4F90000D6F90000D9F90000DBF900002C
:10F2A000DDF90000D7F90000BBFA0000F5FA000014
:10F2B000FAFA000000000000DFF90000E3F90000A6
:10F2C000E7F9000000000000E9F90000F1F9000092
:10F2D00092F900000000000000000000F5F90000B5
:10F2E000FCF90000F9F90000FEF9000008FA00003E
:10F2F00049FA00000000000012FA00001AFA0000AB
:10F3000048F80000AEF70000AEF7000023FA000056
:10F310002AFA000031FA000034FA00001FFA000057
:10F3200057F8000037FA00003BFA000046F80000EA
:10F3300053F8000041FA000046FA000042F80000CD
:10F340004FF800004BFA000050FA000058FA000095
:10F350005AFA000000000000000000000000000059
:10F3600060FA00000000000064FA000068FA000083
:10F370006EFA00000000000071FA000074FA00004C
:10F380007AFA00007EFA0000A6F7000082FA000078
:10F3900094FA00000000000088FA00008DFA0000D6
:10F3A00093FA000096FA000096FA00009DFA000019
:10F3B0009FFA0000A3FA0000A8FA0000ABFA0000D0
:10F3C000BEFA0000AEFA0000B4FA0000B7FA00007E
:10F3D00047FA0000BAFA0000BDFA0000C2FA0000C5
:10F3E000C5FA0000CAFA0000CFFA000000000000D1
:10F3F00000000000D4FA0000D9FA0000DEFA000094
:10F40000E3FA0000E8FA0000EDFA0000F2FA00006A
:10F41000F7FA000000000000D97E000001B30000F0
:10F420002D550000C17D00001155000049B20000BB
:10F43000F19B0000817D0000F75400005164000042
:10F440006D7A0000217D0000ED960000FD63000054
:10F4500045780000BD7C00009D970000398F0000BA
:10F4600041730000AD6400005D8200005D82000019
:10F47000495B0000119D0000FF5B0000F55B000090
:10F48000D75B0000B95B0000815B0000EB5B000014
:10F49000CD5B0000AF5B000075710000E15B000018
:10F4A000C35B0000A55B00001571000075720000D1
:10F4B000D5720000297C0000D97E00002DB3000029
:10F4C00045A4000089A5000000000000B17F0000F5
:10F4D0008D5400007FA5000000000000199200007C
:10F4E0006D54000075A50000096F0000657F0000E5
:10F4F0004D8500006BA500005D540000AD56000076
:10F500007983000061A50000998E0000998E0000AB
:10F510007D5400007D530000616E00005F540000C8
:10F520007D94000065960000BD6C0000FD6F00003A
:10F5300095930000DD9500007D620000816F000062
:10F54000AD92000049950000616C0000BD630000B1
:10F550004DB300001DB40000D97E0000E16800003A
:10F56000E9530000116C00000000000091530000FE
:10F57000D1530000D16B00000000000015620000B4
:10F58000056A0000496B000035670000FD88000037
:10F5900069690000F56A00007F530000A55F000064
:10F5A00009690000956A0000DD610000DD6100006E
:10F5B00041620000616A00004D610000815300005B
:10F5C000799100004D54000019600000E5670000CB
:10F5D000D19000003D540000356600008D670000AA
:10F5E000399000002D5400008565000081800000E6
:10F5F000AD53000009540000F19800004599000047
:10F6000099990000FD990000619A0000A99A0000F4
:10F61000F19A0000459B0000FB21F93FFB210940C6
:10F620007CD91240FB2119407A6A1F407CD92240C4
:10F63000BBFD2540FB2129403A462C407A6A2F40E9
:10F640005C4731407CD932409C6B3440BBFD354037
:10F65000DB8F3740FB2139401BB43A403A463C40EF
:10F660005AD83D407A6A3F404C7E40405C4741401A
:10F670006C1042407CD942408CA243409C6B444079
:10F68000AC344540BBFD4540CBC64640DB8F4740D0
:10F69000EB584840FB21494083F9A200444E6E00DC
:10F6A000FC291500D1572700DD34F50062DBC000CE
:10F6B0003C999500419043006351FE00BBDEAB00D6
:10F6C000B761C5003A6E2400D24D42004906E00001
:10F6D00009EA2E001C92D100EB1DFE0029B11C008E
:10F6E000E83EA700F535820044BB2E009CE984006B
:10F6F000B4267000417E5F00D691390053833900F3
:10F700009CF439008B5F840028F9BD00F81F3B0092
:10F71000DEFF97000F980500112FEF000A5A8B00AB
:10F720006D1F6D00CF7E360009CB2700464FB70016
:10F730009E663F002DEA5F00BA277500E5EBC70023
:10F740003D7BF100F739070092528A00FB6BEA001B
:10F750001FB15F00085D8D00300356007BFC460042
:10F76000F0AB6B0020BCCF0036F49A00E3A91D007B
:10F770005E619100081BE60085996500A0145F009A
:10F780008D40680080D8FF0027734D0006063100C9
:10F79000CA561500C9A873007BE260006B8CC000DC
:10F7A000544553543A00524E4400286929005241AE
:10F7B0004E202300257500256425732025733F0006
:10F7C0002564257320257320257300256425732067
:10F7D0002573004E414E002D494E46002E25253002
:10F7E00025646C6C7500256C6C75002045256400E3
:10F7F0002573256325730025732020256325730059
:10F800002573202B25732025630025732025732065
:10F81000256300436865636B20466C61673A00436B
:10F820006C65617220466C61673A005365742046CE
:10F830006C61673A0044656C657465205072676D51
:10F840003A004953470044534500582019200045C9
:10F850004E4700534349004649580053544F005205
:10F86000434C00476F20546F204C424C3A004754A1
:10F870004F204C424C3A00476F20546F204C696E29
:10F88000653A00257320005F0050726F6772616DEA
:10F890002025630050726F6772616D2025640052ED
:10F8A000756E6E696E67002E202E202E00593A006C
:10F8B000583A0044697669646520627920300049CD
:10F8C0006E76616C69642074797065004E6F206C8F
:10F8D0006162656C004C6162656C20657869737467
:10F8E00073004F7574206F66204D656D004D617813
:10F8F00020497465727320526561636865640055C0
:10F900007365722061626F72746564004E6F20725D
:10F910006F6F740041626F72740068006825630045
:10F9200066007261640067720020100020500020A1
:10F930001C2000201020005069636B204C424C3A80
:10F940000052756E204C424C3A00475342204C42C4
:10F950004C3A00494E54454752415445204C424C84
:10F960003A00534F4C5645204C424C3A00256420F7
:10F97000005061737465204D656D6F72793A0D0AA0
:10F9800000456D70747900522F530053515254004A
:10F990004753420047544F00655E5800521B0053C6
:10F9A000494E0031305E5800582019205900434F0D
:10F9B0005300595E580054414E00312F5800454EB7
:10F9C0005445520045455800434853003100340027
:10F9D000370035003800182B00330036003900504E
:10F9E0005345004C424C004100434C4541522018C5
:10F9F000004859500044494D004652414300434C91
:10FA00004541522052454700436F6D7020636F6E31
:10FA10006A0072756E54696D650059202B20695813
:10FA2000201900524553554C54004D4154524958E9
:10FA3000007821001C5200792C72001C482E4D5376
:10FA4000004C2E522E001C5241440050792C78005C
:10FA50005265201920496D001600534F4C56450041
:10FA6000585E320052544E00485950201D004C4EF2
:10FA700000521A0053494E201D004C4F4700494E7A
:10FA80005400434F53201D00434C20580054414E16
:10FA9000201D001725004C415354205800140041EC
:10FAA0004253004D45414E001C50005346005354F4
:10FAB000444556001C4800434600182D001C444590
:10FAC0004700463F00475241440043792C78005498
:10FAD0004553540053544F2B0053544F2D0053544F
:10FAE0004F2A0053544F2F0052434C2B0052434C8B
:10FAF0002D0052434C2A0052434C2F005820112015
:10FB0000300058203E20300058203C203000582043
:10FB10001220300058201320300058203D2059007A
:10FB200058201120590058203E20590058203C20D0
:10FB300059005820122059005820132059005820ED
:10FB40003D20300040DB0000B2D90000F6D90000B3
:10FB50005AD90000F6D90000E6DA0000F6D9000014
:10FB60005AD90000B2D90000B2D90000E6DA00008C
:10FB70005AD9000052D9000052D9000052D90000D1
:10FB8000F4DA000068E200006AE100006AE10000C7
:10FB900088E4000064E1000064E1000070E400001B
:10FBA00088E4000064E1000070E4000064E100000B
:10FBB00088E400007EE400007EE400007EE40000B3
:04FBC0008CE40000D1
:08FBC40008C7FF7F01000000EB
:10FBCC000508107A6CEF00004D000000583A001F39
:08FBDC002C000000C400001021
:040000030000C13107
:00000001FF
